:1000000000C80120090900000509000005090000D9
:1000100005090000050900000509000000000000B6
:1000200000000000000000000000000005090000C2
:100030000509000000000000050900000509000096
:100040000509000005090000050900000509000078
:100050000509000005090000050900000509000068
:100060000509000005090000050900000509000058
:100070000509000005090000050900000509000048
:100080000509000005090000050900000509000038
:100090000509000005090000050900000509000028
:1000A0000509000005090000050900000509000018
:1000B0000509000005090000050900000509000008
:1000C00005090000050900000509000005090000F8
:1000D00005090000050900000509000005090000E8
:1000E00005090000050900000000000000000000F4
:1000F000000000008D050000050900000509000052
:1001000005090000050900000509000005090000B7
:10011000050900000509000061080000CD08000085
:10012000D5080000DD0800000509000005090000F1
:100130000509000005090000050900000509000087
:100140000509000005090000050900000509000077
:100150000509000005090000050900000509000067
:100160000509000005090000050900000509000057
:100170000509000005090000050900000509000047
:100180000509000005090000050900000509000037
:100190000509000005090000050900000509000027
:1001A0000509000005090000050900000509000017
:1001B0000509000005090000050900000509000007
:1001C00005090000050900000509000005090000F7
:1001D00005090000050900000509000005090000E7
:1001E000050900000509000005090000E50E0000F2
:1001F00005090000050900000509000005090000C7
:1002000005090000050900000509000005090000B6
:1002100005090000050900000509000005090000A6
:100220000509000005090000050900000509000096
:100230000509000005090000050900000509000086
:100240000509000005090000050900000509000076
:100250000509000005090000050900000509000066
:100260000509000010B5054C237833B9044B13B1D0
:100270000448AFF300800123237010BD78000020F4
:10028000000000002847020008B5034B1BB10349DA
:100290000348AFF3008008BD000000007C00002090
:1002A0002847020070B50D461646044610B1081ED8
:1002B00018BF01200549064B34229847236832466F
:1002C00029462046BDE87040184700BF8C630100F6
:1002D000150600004309012200F01F0002FA00F099
:1002E0004033024A42F82300704700BF00E100E0BB
:1002F0007723584302300323B0FBF3F07047772392
:10030000584302300323B0FBF3F04FF47A735843A1
:1003100070477047000000000139FDD8704700BFEA
:10032000F0B505681DB90F4BBDE8F0401847D1F88E
:1003300008C02C460026C2F1010ED4E901379342D1
:1003400095BFDB1973449B1ADB199C4507D92368B9
:10035000264613B9044B3046E6E71C46EDE7A542B6
:10036000E1D0F7E7D5050000010600002DE9F047D0
:10037000D0E90465037E0136DA07044606611FD41E
:10038000037E9B071CD4DFF84480DFF8449000F123
:100390001407CDB16B68AA68F31A934214D3384698
:1003A000C0472B7C012B04D16E603246294638466B
:1003B000C847D4F814A0EB68284698475546E8E7A4
:1003C000237E43F002032376BDE8F0870906000090
:1003D0002103000038B50D46044610B1081E18BFB1
:1003E00001203B220549064B9847064B29462046EB
:1003F0009847054B23600020206138BDA0630100B1
:1004000015060000390D00006D03000038B50546E3
:10041000003818BF01200849084B53229847084B61
:1004200028469847044620B92846064B9847204658
:1004300038BD6FF01000FBE7A06301001506000057
:10044000890E0000750E00002DE9F3410D460446AB
:1004500010B1081E18BF01201E49DFF890807A22D3
:10046000C047237E04F1140743F001032376294695
:10047000194B38469847064660B1237E154903F06C
:10048000FE03002023767F22C0476FF0110002B0E8
:10049000BDE8F0812269114B6A60294638469847C9
:1004A000237E03F0FE032376237E13F002030ED097
:1004B0000B4B01A89847237E03F0FD0323762046CB
:1004C000084B984701A8084B98473046DFE7184685
:1004D000DDE700BFA0630100C505000021030000A7
:1004E000010F0000A50E00000F0F00001506000010
:1004F000014B1860014B18479400002013030000C3
:10050000054B10B51C68054B9847054B0146204626
:10051000BDE81040184700BF94000020F102000021
:1005200019030000054B10B51C68054B9847054B97
:1005300001462046BDE81040184700BF9400002047
:10054000FF020000190300000A4A13889BB210B58D
:1005500043F4A0631380084B9847084B9847084B17
:100560009847084B9847BDE81040074B40F6FF708E
:10057000184700BF00400041ED0900001B060000C5
:10058000590600001D060000E50800000B4A93789C
:1005900082B0DBB20193019B990705D5084B1B681C
:1005A00013B1506802B01847019BDB0704D5044B18
:1005B0005B680BB1014AF4E702B0704700000241EA
:1005C00098000020006800B970478842FAD10120E5
:1005D0007047000038B5074B0446984780F001008B
:1005E0000D46054B05493922C0B2984723682B6058
:1005F000256038BDC505000015060000B763010081
:1006000003680B600160704703680BB11A680260F1
:100610001846704700B900BE704770470C4B0D4A32
:100620005A63DA6B12F0060FFBD14FF402629A6341
:10063000022283F83020064AD36B9807FCD4044B7F
:100640001A6CD10702D41A6C9207F9D5704700BF13
:10065000001000404D0E0100014B01225A717047FD
:1006600000080040C3690B42FCD170470268034B8D
:1006700022F0020202600321184700BF6506000055
:1006800070B50C4D06460FCD88B06C460FC495E88A
:100690000F0084E80F006A46002352F8041BB142A1
:1006A00002D1D8B208B070BD0133082BF5D10020BB
:1006B000F8E700BFF063010008B5034B98478000DE
:1006C0002E3000F0FE0008BD810600004209012323
:1006D00000F01F0003FA00F0014B43F822007047BE
:1006E00000E100E04309012200F01F0002FA00F0DF
:1006F0002033044A42F82300BFF34F8FBFF36F8FBC
:10070000704700BF00E100E04309012200F01F0034
:1007100002FA00F06033024A42F82300704700BF3B
:1007200000E100E038B51B4B04469847022805D08D
:1007300019491A4B40F26B2200209847E369184D83
:1007400013F0010F0ED103212046A84723689B0711
:1007500003D5144B98470221A847052323600321A2
:100760002046A84720460121A8470F4B23600321BC
:10077000A8474FF4403363601F21A8470B4BA36089
:100780004FF61143A3810023A373184684F8303039
:1007900038BD00BF81060000D563010015060000CA
:1007A000650600006D0600000400104002007000A5
:1007B0002DE9F3410546003818BF0120144B0C46C3
:1007C000CB2214499847144B204698470646D0B987
:1007D000124BAC619C4208BF114BDFF8548008BF3C
:1007E0001D6020460F4B104F104D984700210446C6
:1007F0006318D8B20190C0470198B84701310198F9
:10080000A8470429F4D1304602B0BDE8F08100BF0A
:1008100015060000D56301002507000000200141F6
:10082000A8000020B906000009070000CD0600005E
:10083000E50600008069036843F0020303600321BA
:10084000004B184765060000836999627047836909
:1008500001229A757047836902229A7570470000D9
:10086000194B186810B58469237EDA0708D5A37D73
:10087000DB0705D5012323750368BDE81040184741
:10088000237E990706D5A37D9A0703D502232375F6
:100890008368F2E7237E5B070CD5638B03F0370395
:1008A00013B1FF23638310BDA16A4368BDE8104004
:1008B000C9B21847237EDB09F5D080232376C368AD
:1008C0009847638B9BB2EDE7A8000020004B1847C8
:1008D00061080000004B184761080000004B1847F2
:1008E00061080000C30707D5044B054A1A6243F6A6
:1008F000FD7259681142FCD1704700BF001C0040D6
:1009000007010100FEE7000018491948814210B5AF
:100910000AD0184BDA1C121A22F00302C41EA3429A
:1009200038BF0022144B9847144B1548DA1C121A92
:10093000C11E22F00302994288BF0022114B002100
:100940009847114A114B22F07F029A60D3F8882011
:1009500042F47002C3F88820BFF34F8FBFF36F8F4C
:100960000B4B98470B4B9847FEE700BF2847020008
:100970000000002074000020F962010000C800207F
:1009800078000020496301000000000000ED00E055
:10099000916201009909000008B5024B024C98478A
:1009A000A047FDE7AD090000E509000010B5074BC1
:1009B0009847074B9847074B9847074B9847074B73
:1009C0009847BDE81040064B184700BF4905000096
:1009D000C5120000251200005D1100004D1200003C
:1009E00071130000004B18471D140000064B42F223
:1009F0008E329A8200229A75DA75DA6902F47C5294
:100A0000DA6101221A7470470014004000238362E7
:100A1000C3690BB108381847704700238362436AE3
:100A20000BB108381847704770B50446054BA0F164
:100A300008052C309847236A1BB12846BDE8704052
:100A4000184770BD790C000070B50E461546044677
:100A500018B1D9B1101E18BF01200F4B0F4940F239
:100A60003B129847B4F84420B4F84C309A420FD166
:100A70000023A4F844300123236304F10800084B49
:100A8000A664A4F84C509847284670BD0846E4E791
:100A90006FF01B00F9E700BF150600003964010084
:100AA0004F080000838FB0F844209A4210B50446E6
:100AB0000AD0026C591C8187D15C044B9847044BC7
:100AC0002046BDE810401847024BFAE749080000ED
:100AD0004F080000570800002DE9F7430E4617465F
:100AE000044618B1E9B1101E18BF01201049114B7E
:100AF000DFF850904FF4AC72984734340E4B01A895
:100B000098470E4B204698470D4B804601A89847C2
:100B10000025A84501D0BD4205D1284603B0BDE857
:100B2000F0830846E2E771192046C8470135F0E72F
:100B30003964010015060000010F0000BD0C000023
:100B40000F0F0000390C0000F8B50D4616461F4681
:100B5000044620B109B312B3181E18BF0120124970
:100B6000124B3A229847124B3A46314604F1340070
:100B70009847B0B90F4B294604F10800984758B977
:100B80000D4B63600D4B23600D4BA3600D4BE36079
:100B90000D4B23610D4B6361F8BD0846DFE710463E
:100BA000DDE76FF00C00F7E739640100150600007F
:100BB000FD0B0000B1070000D90A0000490A00003F
:100BC000A50A0000290A00000D0A00001B0A000007
:100BD00010B50446003818BF01200549054B6122B5
:100BE000984704F10800044B9847002010BD00BF4F
:100BF00039640100150600003508000070B50E4686
:100C00001446054618B189B1101E18BF01200849C5
:100C1000084B28229847631E13EA040003BFC5E966
:100C20000130E8602E606FF00C0070BD0846EEE702
:100C3000566401001506000038B50D46044610B193
:100C4000081E18BF01200A4B0A4940229847D4E9E0
:100C500002329A4209D0626813402268D35C2B703A
:100C6000A3680133A360002038BD6FF00900FBE7E3
:100C7000150600005664010038B50446003818BF58
:100C800001200D460B4B0C4951229847E3686268DE
:100C900013402268D554D4E90121E368591A9142DE
:100CA00088BF9A1A03F1010388BFA260E3600020A5
:100CB00038BD00BF150600005664010010B504469B
:100CC000003818BF01200449044B67229847D4E933
:100CD0000230C01A10BD00BF5664010015060000A6
:100CE00003690B42FCD1704770B5104D06460FCD1D
:100CF00088B06C460FC495E80F0084E80F006A4680
:100D0000002052F8041BB14202D130B908B070BDC6
:100D100001300828F5D10020F8E700200449054BF0
:100D20004FF49E7298474FF0FF30EFE79064010058
:100D30007A640100150600002DE9F843454B814611
:100D400008460C469847444B4449C9F80C408D224C
:100D50008046012098472369414A13F0010F11D1C1
:100D600003212046904723689B0706D5236823F07C
:100D7000020323609047022190470123236003214F
:100D800020469047374F142505FB08750121204662
:100D900090476E6A26600321904795F82A30E373E6
:100DA00006F00C062B8DE380082E4FF00103237311
:100DB0003AD1EB6AE361C021904700232362904758
:100DC00001236372284B9C4204BF284BC3F8009058
:100DD000142303FB0873B3F92230002B0DDB5A09EF
:100DE000012103F01F0301FA03F32032204941F8E7
:100DF0002230BFF34F8FBFF36F8F142000FB0877B3
:100E0000B7F92230002B0CDB03F01F015B099B00BC
:100E100003F1604303F5614301228A40C3F8802156
:100E20001A600020BDE8F8832EB9AB8DA383C021E2
:100E30009047E683C3E7042EC2D195F82C30237780
:100E4000C021904700236377904795F82B30E376D5
:100E50002021B4E7E90C0000150600007A640100C7
:100E6000E10C00009064010000380040AC0000205C
:100E700000E100E0C068036843F00203036003215F
:100E8000004B1847E10C000008B5C068034B032174
:100E900098470068C0F3400008BD00BFE10C0000A7
:100EA0000020704710B50A4BC0689847094B0A49A3
:100EB000044640F20F1201209847084B142000FB13
:100EC0000430BDE8104090F82200054B184700BFE1
:100ED000E90C0000150600007A640100906401002E
:100EE000D5020000054B1868C3689A7AD20703D56B
:100EF00001229A7203681847704700BFAC000020B7
:100F0000EFF31083036072B6BFF35F8F7047BFF3D8
:100F10005F8F036883F31088704700000122430944
:100F2000914200F01F0002FA00F010D002291FD0F9
:100F300029BBDB0103F1824303F50043586082B211
:100F400042F08042000C9A6240F040400EE0DB012B
:100F500082B203F1824303F5004342F0804242F43F
:100F6000003258609A62084A42EA1040986270471C
:100F7000DB0103F1824303F500439860DFE7034997
:100F8000034B462200201847000002C0C464010041
:100F90001506000030B54B1CC5B2184B00F01F04FD
:100FA0004FEA50104FEAC010034407D1234493F88E
:100FB000402002F0FE0283F8402030BD181903EBF8
:100FC000540390F8402002F0FE0242F0010280F843
:100FD000402093F8302015F0010FC9B219BF02F07C
:100FE0000F0242EA011101F00F0102F0F00214BFFA
:100FF000C9B2114383F83010DFE700BF0080004121
:1010000001294FEA501300F01F000FD002291DD014
:1010100069BB00EBC31000F1824000F5004090F87E
:10102000403003F0FB0380F840307047DB0103F1F0
:10103000824303F5004381401844596090F84020F2
:1010400042F0040280F8402099617047DB0103F10F
:10105000824303F500430122824018445A6090F80D
:10106000401041F0040180F840105A617047024975
:10107000024B892200201847C464010015060000B5
:10108000530010B5540104F4703403F47C7323430B
:1010900002F00704520302F0E0522343134303EA31
:1010A000010221EA03018261416110BD38B5054C9E
:1010B000054B40256561984780236361A361A56165
:1010C00038BD00BF00800041811000002DE9F041D3
:1010D000074F884616461D460024A54201DCBDE8A0
:1010E000F08136F814204146B8470134F5E700BFD7
:1010F000AD1000002DE9F84F4701154BDFF858A05F
:10110000884616465FFA87FB002528FA05F2D207C3
:1011100019D5EC19E4B22046717898470BEB050914
:101120000C4B31782046984771684846D04704F008
:101130001F016409E40104F18244012204F5004422
:101140008A40034B62610135202DDED1BDE8F88F66
:101150001D0F000001100000950F00002DE9F7435E
:101160004FF000096A46294BCDF8009002254FF058
:10117000FF342749DFF8A8808DF801500120019441
:10118000984729460620234F234EC047494606204C
:10119000B84721460620B04729460420C0474946A3
:1011A0000420B84721460420B04729460320C04701
:1011B00049460320B84721460320B0472946052069
:1011C000C04749460520B84721460520B047294673
:1011D0000720C04749460720B84721460720B047A7
:1011E00001216820C04729466820B8472146682069
:1011F000B0470A4B40229A6110229A6108229A61F4
:1012000080229A6103B0BDE8F08300BFF5100000B2
:10121000F7C3031C01100000950F0000008000417F
:101220001D0F00007047000010B4064CD4E90023E5
:10123000501C43F10001C4E90001034B5DF8044B6D
:1012400001201847B000002079DA000070B512487C
:10125000124B134C9847134A536943F4804353612C
:10126000114B4022C3F8A420104B984704F11C05F1
:1012700002460F490F4B28469847012323612376E6
:101280000D4A0E4B626104F1080128469847284632
:101290000B4BBDE87040184710E000E0F10400007F
:1012A000B000002000080040001C0040A10E00001B
:1012B00000380040D5030000291200004904000056
:1012C0000D040000214B37B54022C3F8DC20432237
:1012D000C3F88C201E4A1F4993691F4D43F40073C5
:1012E00093611E4A002302F110040093204610234C
:1012F000A8471B4B93F8D82002F0FE0242F00102EF
:1013000083F8D82093F8BC2002F0F00242F00302E8
:1013100083F8BC2093F8D92002F0FE0242F00102CB
:1013200083F8D92093F8BC2002F00F0242F030027B
:1013300083F8BC2020460B4B98470B490B4B0C22E3
:10134000204603B0BDE83040184700BF001C0040F5
:101350000008004000200141490B0000E800002087
:1013600000800041D10B000000000020A502000019
:1013700030B51A4B1A4C1B4D8DB098471A4B9847F5
:1013800000221A4920464FF47F53A84701A8184B62
:101390009847184B049301A8174B02949847174B92
:1013A00000209847164B002104469847154B1649D4
:1013B00005469847002211462846144DA847144B6D
:1013C000002120469847232204465A21A847114964
:1013D000114B204698470DB030BD00BFDD1C00000A
:1013E00048010020E1D700009D1400006C0100209E
:1013F000A1D700004116000001D800002518000008
:101400005D47010009450100EC640100552800001A
:101410007D590100E064010081560100004B18472E
:1014200045FA0000094908B540234B61084B0246C4
:10143000187818B92020486101211970054B064918
:1014400006489847014B40229A6108BD0080004140
:101450000C000020AD100000F7C3031C8080004189
:10146000094908B540234B61084B0246187818B16A
:101470002020886100211970054B064906489847CD
:10148000014B40229A6108BD008000410C00002001
:10149000AD100000F7C3031C808000412DE9F84324
:1014A00000BF5F4F5F4E1024BC613220B0477C61AB
:1014B00000BF3220B047BC613220B04700BF4FF0C0
:1014C00040080A20C7F81480B0470520C7F81880E4
:1014D000554D564CDFF86091B0470120A8471420C5
:1014E000B0470120A8471420B0470120A847142086
:1014F000B047E220C7F81480A8472F20A047032058
:10150000A0475420A047E020A8470120A047484B0F
:1015100064209847E020A8470320A0470120B04757
:101520000120A8470120B047E620A8470120A04796
:10153000CC20A047CC20A047B020A8472820A04717
:101540003C4E8020A047B047C8470138C0F3072071
:10155000A047B047C8470138C0B2A047DFF8DC90C9
:10156000B047C8470138C0F30720A047B047C84775
:101570000138C0B2A0470020A047F020A8470320B0
:10158000A0473A20A8475520A047B420A8470220EA
:10159000A0470D20A0470020A0472B20A0472820CF
:1015A000A0470020A0470020A0470020A047B62069
:1015B000A8470120A0471D20A0470020A0470C20DD
:1015C000A0470920A0470020A0470020A0472A20CC
:1015D000A8470020A0470020A0470120A047DF2007
:1015E000A0472B20A8470020A0470020A0470120AB
:1015F000A0470F20A0472920A847BE20A8470620C3
:10160000A047FF20A0470120A047FF20A0470020BF
:10161000A0470120A047C7F81880BDE8F88300BFA5
:101620000080004125050000251400006114000021
:101630000105000041D900004DD9000071D900001A
:101640002DE9F04FB1F904302DED028B002B08EE9F
:10165000100A81B00D469046C0F28180B1F9063083
:10166000002B7CDB404FDFF818A1B847D047B5F915
:101670000030834273DAB8473C4CA047B5F90260AA
:10168000B042A3466BDDB5F90040B847D047B5F985
:101690000430984224EAE47426EAE67652DCB8473D
:1016A000D04700F1FF3AB847D847B5F9063098421D
:1016B0004ADCB847D847471EDFF8C890DFF8C8B003
:1016C0002A20C847C4F30720D847E0B2D847CAF356
:1016D0000720D8475FFA8AF0D8472B20C847C6F3BF
:1016E0000720D847F0B2D847C7F30720D847F8B249
:1016F000D8472C20C847AB881D4A2D881178013364
:101700005D1BADB21B4B19B12021996100211170F5
:1017100040225A61C4F1010353441748DFF86CA01A
:10172000DFF86CB09CB26D00BE420FDD114B402261
:101730009A6118EE100A114B01B0BDEC028BBDE8A6
:10174000F04F18479A46AEE71F46B5E74246234694
:1017500051460136D847A844074836B2E4E701B0FD
:10176000BDEC028BBDE8F08F41D9000071D90000BB
:101770000C0000200080004180800041FDD9000065
:101780004DD900002514000061140000F7C3031CAC
:10179000CD100000003818BF01207047F0B51B4B7A
:1017A000C3B0074616469847E528044629D802AD37
:1017B0000246174B3946284698472B1920222A55AE
:1017C00028225A7030229A70124C7822DA70181D32
:1017D0001C2226FA02F101F00F012144043AC97CCF
:1017E00000F8011B111DF4D129221A7300225A732B
:1017F000094B0095BC220949094C0320A04743B07E
:10180000F0BD054B0097BF22F5E700BF7D630100E7
:1018100079EC00005DEB010081EB010053EA01006F
:1018200031E9000037B5044670B9084B98470446C3
:1018300050B9074B00930749074B084D2E22022051
:10184000A847204603B030BDE46BFAE741D9000059
:10185000C4EB010094EB010034ED010031E900001C
:1018600037B5044670B9084B9847044650B9074B42
:1018700000930749074B084D4B220220A8472046FA
:1018800003B030BD246CFAE741D90000FDEB010044
:1018900094EB010048ED010031E9000037B5044642
:1018A00070B9084B9847044650B9074B0093074955
:1018B000074B084D5C220220A847204603B030BDEC
:1018C000646CFAE741D9000036EC010094EB0100AA
:1018D0005EED010031E9000070B5094D002428B922
:1018E00064B12046074BBDE87040184790F834308B
:1018F00013F0200F18BF0446A847F0E770BD00BFE3
:10190000D5200000C52700002DE9F347067D16F01D
:1019100001060546884617465CD1C468DFF8C8A0B2
:101920004FF00109002C4CD12B7DDB0601D4002E99
:1019300050D1B9F1000F4DD02846C0470446002EC3
:101940003AD1002846D006464FF000092068D0471B
:1019500002460028E6D1EB68A3423BD01F4E7BB184
:1019600018680192C36917219847EB68019A1868B3
:101970000E21B04701282DD1EB681868184B984705
:101980002068EC60C369002216219847EB680022AA
:1019900018680D21B04701281CD1EB681868114B5D
:1019A0009847EB6818680E4B98472B6993B1284607
:1019B00002B0BDE8F04718474FF00009002CC5D130
:1019C000B2E721462846B847002E08BF2646B04257
:1019D0000446F3D102B0BDE8F08700BF291F000024
:1019E00039270000D9180000D12500000148024B1A
:1019F00018211847488600204DE60000014A024998
:101A0000024B1847FDE60000F1E60000091900004E
:101A1000014A0249024B18471DE70000F7E60000A3
:101A20000919000038B5037DC3F3001543F0100316
:101A3000037504461B0754BF034B044B9847237D93
:101A400065F30413237538BDFD190000111A000059
:101A50002DE9F3410D460446002836D0254EB04707
:101A6000B046254E30BBAB6B73B1244B284698472C
:101A700050B1A86B224B234E9847234B0093234928
:101A8000234B7F220120B047224BAC63204698476E
:101A9000214B064698470746F0B91D4B1B4900935A
:101AA00085220320174CA0471C481D4932463B465F
:101AB0008847FEE70368AB420AD11A4B00931349EB
:101AC000134B104C75220120A04702B0BDE8F081F5
:101AD00001462046B047C5E7002EF6D035602046C7
:101AE000C0478642F1D1064B204602B0BDE8F04126
:101AF000184700BFF1E60000FDE60000D9410000F4
:101B0000251A000031E900004CEE0100D1ED010082
:101B10008EEE0100A9E600009517000002EE01001C
:101B20009D17000010EE0100F8B5846B0646002CEE
:101B300033D0E368002B30D01B681C4D83421BD18F
:101B4000237DDA0744BF6FF3000323752046A847BF
:101B5000E368834222D1164B20469847E3689842B7
:101B60001CD100680022C36917219847E3681B68ED
:101B7000B34204BF0023E3602046A8470D4F05464B
:101B80005DB12B68B342294620460BD10A4B9847DA
:101B90000A4B284698470023B363F8BD084B2046FC
:101BA0009847E3E7B8470546EAE700BFF1E60000DB
:101BB000F7E60000FDE60000B5E700002DEB0000B1
:101BC000251A000010B1C06800B10068704710B15C
:101BD000007DC0F340007047F8B50C4D0C4E044634
:101BE0000020A847002700B9F8BD90F8503043F016
:101BF000020380F850307368984208BF376014B110
:101C0000C36B9C4200D1C763A847ECE75DDA0000D4
:101C1000EC800020014B0020184700BFD91B0000BA
:101C2000014B5868704700BFEC80002090B190F8DD
:101C3000503043F0020380F85030084B5A6882421B
:101C400004BF00221A6011B1C36B8B4205D100237F
:101C5000C3637047024B084618477047EC8000206A
:101C6000D91B0000014B1868704700BFEC800020B2
:101C70002DE9F047051D124BDFF8489028460E4627
:101C8000174698471FFA86F804461FFA87FA0CB9D8
:101C9000BDE8F087238A43442382638A53446382E6
:101CA000A38A4344A382E38A5344E38220463A460C
:101CB0003146FFF7DDFF21462846C8470446E6E7E0
:101CC000F1E60000FDE60000013900F1080311F81B
:101CD000012F00F8012B9842F9D17047F0B5204E42
:101CE000204D337885B043B11F4B00931F49204BE3
:101CF00078220220A84705B0F0BD1E4B1E4C1F4F96
:101D000098471F4B98471F4B98471F4B98471F4BAF
:101D100098471F481021A0471E4B009302224FF006
:101D20001F01CDE901334FF60000B8471A4B984721
:101D30001A4B98471A484FF4B871A04760211948C8
:101D4000A047194B9847194B9847194B01209847C2
:101D5000184B00930120064B04493070A222C9E7BA
:101D6000F480002031E90000CEEE01009FEE01007A
:101D7000A6F001005DEA00004DE600005D250100CF
:101D800079F8000021E4000075DC0000ED19000086
:101D900060860020100000202D030100F54E000099
:101DA0000C86002018860020151C000019D10000A8
:101DB000F1C60000E6EE010073B50E4B04460E4678
:101DC0009847054668B90C4B0C49009340F2945271
:101DD00003200B4EB0470B480B4922462B46884741
:101DE000FEE794F8343066F3C71384F8343002B059
:101DF00070BD00BF95170000FBF001009FEE0100D1
:101E000031E9000003EF01009D17000073B50E4B90
:101E100004460E469847054668B90C4B0C4900939A
:101E20004FF4B46203200B4EB0470B480B492246D7
:101E30002B468847FEE794F8343066F3000384F8B5
:101E4000343002B070BD00BF9517000012F10100E0
:101E50009FEE010031E9000003EF01009D17000033
:101E60002DE9F043804687B016461F460C4691B1D7
:101E7000244B08469847054668B9234B23490093ED
:101E80004FF4DB620320224EB0472248224922460B
:101E90002B468847FEE7214D039400238DF8103030
:101EA0006B68059303AB6B601D4BD5F80890AF6072
:101EB000984718B183680BB131469847B8F1000FC5
:101EC00002D031462046C0476B68C5F808909B6831
:101ED0006B609DF8103083B98CB194F834305A0699
:101EE0000DD5206858B10F4B3A4631469847431EEE
:101EF0005842584107B0BDE8F0830020FAE70120BE
:101F0000F8E700BF95170000D7F101009FEE010030
:101F100031E9000003EF01009D170000F48000206C
:101F2000211C0000291F00007FB50E4603920446C5
:101F3000D8B10F4A9047039B054668B90D4B0E492F
:101F4000009340F2C46203200C4EB0470C480D4988
:101F500022462B468847FEE7A06921460A4C3246B6
:101F6000A44604B0BDE870406047012004B070BDD5
:101F700095170000EAF101009FEE010031E9000031
:101F800003EF01009D170000611E000073B50B4BAD
:101F900004460E469847054668B9094B094900931F
:101FA00040F21B720320084EB047084808492246F9
:101FB0002B468847FEE7E66102B070BD951700002A
:101FC000F8F101009FEE010031E9000003EF01008C
:101FD0009D17000010B1C36903B118470120704775
:101FE00073B50B4B04460E469847054668B9094B36
:101FF0000949009340F237720320084EB047084861
:10200000084922462B468847FEE7266202B070BD8B
:10201000951700000DF201009FEE010031E900006C
:1020200003EF01009D1700007FB50E4B039104469E
:1020300098470399054668B90B4B0C49009340F249
:10204000497203200A4EB0470A480B4922462B46E4
:102050008847FEE7606A094B984700B1606204B0A8
:1020600070BD00BF9517000022F201009FEE010035
:1020700031E9000003EF01009D1700005DEE000054
:1020800073B50E4B04469847054668B90C4B0D498D
:10209000009340F2597203200B4EB0470B480C4995
:1020A00022462B468847FEE7E369002206212046A8
:1020B000628602B0BDE87040184700BF9517000067
:1020C0003BF201009FEE010031E9000003EF010047
:1020D0009D17000073B50B4B04469847054668B939
:1020E000094B0A49009340F29F720320084EB04703
:1020F0000848094922462B468847FEE7206802B077
:1021000070BD00BF9517000057F201009FEE01005F
:1021100031E9000003EF01009D17000073B50E4B7D
:1021200004469847054648B10C4E2046B047254620
:1021300004460028F9D1284602B070BD084B094971
:10214000009340F26B720320074EB04707480849DE
:1021500022462B468847FEE795170000D520000051
:1021600069F201009FEE010031E9000003EF010078
:102170009D1700002DE9F7431E4B0546984704467E
:1021800068B91D4B1D49009340F27F7203201C4E1D
:10219000B0471C481C492A4623468847FEE72B685F
:1021A0001BB12846194B984705461948194E1A4F36
:1021B000DFF85C80B047044664B9184B00930F49C0
:1021C0000D4B0F4D4FF4F2620220A847204603B09A
:1021D000BDE8F08304F130094846B04720B92146F4
:1021E0004046B8470446E7E78542EFD001464846F7
:1021F000B847F3E7951700007BF201009FEE01005E
:1022000031E9000003EF01009D1700001D210000CF
:102210000C860020F1E60000FDE6000010EF010052
:1022200073B5104B04460D469847064668B90E4BE9
:102230000E49009340F2AD7203200D4DA8470D48A2
:102240000D49224633468847FEE7201D25B90B4B32
:1022500002B0BDE870401847094B294602B0BDE8FE
:1022600070401847951700008BF201009FEE0100A7
:1022700031E9000003EF01009D170000F1E60000C6
:10228000FDE6000073B50E4B04460E469847054622
:1022900068B90C4B0C49009340F6010203200B4E29
:1022A000B0470B480B4922462B468847FEE70A4BAE
:1022B00004F11001304602B0BDE87040184700BF7D
:1022C00095170000FCF201009FEE010031E90000CB
:1022D00003EF01009D170000C91C000073B5104BEF
:1022E00004469847054668B90E4B0F49009340F6DF
:1022F000220203200D4EB0470D480E4922462B46C0
:102300008847FEE70C4B2046984728B1238A008A6D
:10231000181A00B202B070BDB4F91000FAE700BF9D
:10232000951700000EF301009FEE010031E9000057
:1023300003EF01009D170000D520000073B5104B7E
:1023400004469847054668B90E4B0F49009340F67E
:10235000360203200D4EB0470D480E4922462B464B
:102360008847FEE70C4B2046984728B1638A408A8D
:10237000181A00B202B070BDB4F91200FAE700BF3B
:10238000951700001BF301009FEE010031E90000EA
:1023900003EF01009D170000D520000073B50D4B21
:1023A00004469847054668B90B4B0C49009340F624
:1023B0004A0203200A4EB0470A480B4922462B46E0
:1023C0008847FEE7A38A208A0133181A00B202B0B8
:1023D00070BD00BF9517000028F301009FEE0100BB
:1023E00031E9000003EF01009D17000073B50D4BAC
:1023F00004469847054668B90B4B0C49009340F6D4
:10240000560203200A4EB0470A480B4922462B4683
:102410008847FEE7E38A608A0133181A00B202B0E7
:1024200070BD00BF9517000039F301009FEE010059
:1024300031E9000003EF01009D17000013B511B949
:10244000283002B010BD8DF800100024044B019418
:102450006A460821984701280CBF01982046F0E7FA
:10246000D51F00002DE9F84F0746984619481A4B2A
:10247000DFF86090DFF87CB00D46164698470446BA
:102480000CB9BDE8F88F4445FBD0144B21464846B3
:10249000984782462068B8421AD1A179A94201D052
:1024A000FF2D15D1A288B24201D0FF2E10D1D847FE
:1024B0000B4A9047A1880B4A90470B4A00212046BF
:1024C00090470A4A484621469047094A2046904785
:1024D0005446D5E760860020F7E600001DE70000BF
:1024E000B55C00000D580000F5DC0000B5E7000009
:1024F0002DEB00003D24000037B50E4B04460D4681
:10250000984750B90C4B00930C490D4B0D4C40F2C1
:1025100092420220A04703B030BD0B4B98472046A3
:102520000A4C0023FF222946A44603B0BDE83040F0
:10253000604700BF3D24000058EF01009FEE0100FE
:10254000F5F3010031E90000C55C000065240000DE
:102550002DE9F041164B04681648164E164F984761
:10256000002590B945B9A179144B20689847144BC0
:102570009847A188134B98470E48134B214698471C
:102580002046124BBDE8F0411847A0420CD002682B
:1025900023689A4208D1436823F07F42636823F09E
:1025A0007F439A4208BF012501463046B847D8E725
:1025B000F1E6000060860020FDE600003D240000FA
:1025C000B55C00000D580000B5E700002DEB0000E1
:1025D00073B50C4B04469847054668B90A4B0B493E
:1025E000009340F641220320094EB04709480A49AA
:1025F00022462B468847FEE794F83400C0F30010CB
:1026000002B070BD9517000043F401009FEE010079
:1026100031E9000003EF01009D1700002DE9F041B2
:10262000354B86B0044688469847054668B9334B13
:10263000334900934FF4F0720320324EB0473248D2
:10264000324922462B468847FEE7314F2046B8479D
:10265000002841D12F4B204698472F4B05469847DD
:102660002E4B0646984785422CD1B4F932502C4B5C
:1026700004F1100102A89847BDF80820ABB2D21AA5
:10268000ADF80820BDF80A20264DD21AADF80A2070
:10269000BDF80C201A44ADF80C20BDF80E204146C0
:1026A000134404A802AAADF80E30A847A0B1DFF881
:1026B00084802046C047044688B91B4B04A9304695
:1026C000984709E0194B304698478542CDD0184BC2
:1026D000304698478542C8D006B0BDE8F08104A9CD
:1026E00004F110020846A8470028F5D02046B84754
:1026F0000028F1D12046DDE79517000055F40100D0
:102700009FEE010031E9000003EF01009D1700007A
:10271000D12500001D2100007521000025180000B2
:10272000C91C0000D1DE0000F94E00006118000055
:102730009D180000D52000007FB51A4B054698472C
:10274000044668B9184B1949009340F20D22032042
:10275000174EB047174818492A4623468847FEE7D0
:10276000B5F93240154B05F1100102A89847BDF8A4
:102770000820A3B2D21AADF80820BDF80A20D21A58
:10278000ADF80A20BDF80C201A44ADF80C20BDF8B5
:102790000E201344ADF80E3002A9094B2846984785
:1027A00004B070BD951700006CF401009FEE0100AD
:1027B00031E9000003EF01009D170000C91C000073
:1027C0001D260000F7B5194B05469847044668B921
:1027D000174B1849009340F262220320164EB0476F
:1027E000164817492A4623468847FEE7154B2846D0
:1027F0009847071D144B044638469847854213D026
:10280000124E2046B0472A46394638460123104F1B
:10281000B847E3692A4601212046984720463346B7
:1028200003B0BDE8F040184703B0F0BD95170000B5
:102830007EF401009FEE010031E9000003EF01008A
:102840009D170000D5200000F1E6000039270000A8
:1028500035E800002DE9F0432E4B87B0044688464A
:1028600017469847054668B92B4B2C49009340F210
:10287000962203202A4EB0472A482B4922462B464F
:102880008847FEE726685EB9284B00932349224B10
:10289000234C4FF427720220A04707B0BDE8F08315
:1028A000218A338A628A5B1A03EB0801738A9B1AB6
:1028B000DA1997B21FFA81F812B258EA07030DB27B
:1028C0000392EAD02046DFF87090C84704A920465A
:1028D000174B9847238A039A43442382638A3B44D5
:1028E0006382A38A9844E38AA4F814801F4429468B
:1028F0002046104BE7829847E36904AA022120464C
:102900009847F36922460121304698472046C84738
:10291000C3E700BF95170000ACF401009FEE010073
:1029200031E9000003EF01009D1700008EEF010068
:1029300085220000711C00003927000073B50F4B81
:1029400004460E469847054668B90D4B0D4900935D
:102950004FF4337203200C4EB0470C480C4922460A
:102960002B468847FEE70B4B204698470A4B02460A
:102970003146204602B0BDE8704018479517000068
:10298000BBF401009FEE010031E9000003EF0100FC
:102990009D1700003D2300005528000073B50F4B24
:1029A00004460E469847054668B90D4B0D490093FD
:1029B0004FF4367203200C4EB0470C480C492246A7
:1029C0002B468847FEE70B4B204698470A4B0146AB
:1029D0003246204602B0BDE8704018479517000007
:1029E000C8F401009FEE010031E9000003EF01008F
:1029F0009D170000DD220000552800002DE9FF474B
:102A0000DFF8D890BDF9308004460D4617461E46C3
:102A1000C847824668B92A4B2A49009340F26D3272
:102A20000320294DA847294829492246534688476B
:102A3000FEE71DB9274B2046984705462846C8475C
:102A4000814668B91E4B1F49009340F27132032042
:102A50001D4CA0471D481E492A464B468847FEE7A5
:102A60003A4604F1100103AB05F11000DFF8709055
:102A7000C847184B20469847BDF80E20BDF80C10EB
:102A8000B0F91230008A42443144091AD21A09B20C
:102A900012B2114BADF80C102046ADF80E2098473D
:102AA00094F8493084F848706FF34103A4F8446007
:102AB000A4F84680256484F8493004B0BDE8F08766
:102AC000D5F401009FEE010031E9000003EF0100A1
:102AD0009D170000D5200000552800009517000024
:102AE00079E100002DE9F04F87B0CDE903235C4D7B
:102AF000BDF94030059380460E46A847AB460446D4
:102B000068B9584B5849009340F295320320574D0D
:102B1000A84757485749424623468847FEE7564B41
:102B2000DFF8689140469847544B04464046984722
:102B3000534B82464046984705464046C84707469D
:102B40001EB950494046884706463046D8474C4B48
:102B5000834668B9434B4449009340F2A1320320B5
:102B6000424CA0474248434932465B468847FEE70D
:102B7000039A05EBD57507EBD77745F34F0547F378
:102B80004F07142A26D8DFE802F00B591B5F5D4E71
:102B9000675B63591B5F5D4E67595B5D5F636700F1
:102BA0003046984700EBD070C5EB600004B2304669
:102BB000C84700EBD070C7EB60000FFA80FA09E05D
:102BC0003046984700EBD070C5EB60007F4204B2FE
:102BD0000FFA87FA2B4B40469847049B318A059A97
:102BE0001944738A0C441344018A408A03EB0A0295
:102BF000611A121A244B12B209B240469847039B3D
:102C000088F84830049BA8F84430059BA8F8463063
:102C100098F84930C8F8406043F0020388F849301A
:102C200007B0BDE8F08F3046984700EBD070C5EB99
:102C3000600004B23046C847C01BBEE76842C5E723
:102C40006842B3E76842F4E730469847401BBDE767
:102C500030469847401BA9E730469847401BE8E7B5
:102C600095170000E2F401009FEE010031E9000039
:102C700003EF01009D170000DD2200003D2300004E
:102C80009D230000D520000055280000ED23000002
:102C900073B5124B04469847054668B9104B114965
:102CA000009340F22A4203200F4EB0470F481049CC
:102CB00022462B468847FEE794F84950B4F946006F
:102CC000216C94F84820B4F9443000902046AC07B9
:102CD0004CBF084C084CA04702B070BD95170000CF
:102CE000F5F401009FEE010031E9000003EF01005F
:102CF0009D170000E52A0000FD290000F8B500211D
:102D00000B4D0C4F0646A847044604B9F8BD2046B3
:102D1000B847E36900220421204698472046B84777
:102D20002046FFF7EBFF21463046A8470446ECE774
:102D3000212200003927000073B5464B05460C469A
:102D40009847064668B9444B4449009340F21D52E7
:102D50000320434CA047434843492A46334688470B
:102D6000FEE77F2C414E57D86F2C1AD85C2C48D8E0
:102D70003F2C3DD8072C4AD8012C42D92846B047D1
:102D8000EB690022042128469847182C55D8142CAA
:102D900055D92868002852D0C369002201219847DC
:102DA0004DE0A4F170030F2B2BD801A252F823F0B1
:102DB0007D2D00007D2D0000032E00007D2D0000E4
:102DC0007D2D00007D2D0000032E0000032E00004D
:102DD000032E0000032E0000032E0000032E00002F
:102DE0007D2D0000032E00007D2D00007D2D0000B4
:102DF000A4F1400293B201229A401D4B1340002BD4
:102E0000BCD12846334602B0BDE870401847A4F153
:102E10001003082BF5D8B1E748F281039C4208D88B
:102E200048F27F039C42A9D8902CA7D0FF2CE8D170
:102E3000A4E748F28E039C42F9E7FF2CA9D028466C
:102E4000B047FF2C01D0230402D50A4B2846DAE70D
:102E500002B070BD9517000004F501009FEE01005F
:102E600031E9000003EF01009D1700003927000041
:102E700003100F10FD2C000010B5044B04469847BA
:102E80002046034BBDE81040FF211847F9240000FD
:102E9000392D0000F8B51E4C06460D460027F9B244
:102EA0002846A0470246F8B101794FF0000C5FFABE
:102EB0008CF3994215D9507900F00600062823D1E9
:102EC0000133DBB2994216D9106850F823309E4284
:102ED00003D00CF1010C002EE9D10E4BFF21284646
:102EE00098470137402FDAD10B4F00212846B847C9
:102EF000044610B9F8BD0023E9E721463046FFF744
:102F0000C9FF21462846F2E70029DDD10B46DEE75E
:102F10003D240000392D0000212200002DE9F84F4A
:102F20000F4EDFF84090DFF840A007460020B04782
:102F300004460CB9BDE8F88F04F130084046C84794
:102F4000DFF828B005461DB92046B0470446F0E733
:102F500029463846D04729464046D8470546F2E735
:102F600009DA0000F1E60000952E0000FDE6000001
:102F70002DE9F0413A4B04460D46817900689847A7
:102F8000384B9847A18801F00F03082B16D84DB98C
:102F9000B4F90820344B9847A1882068334BBDE82A
:102FA000F0411847FF2DB4F90C20F3D0B4F90830E4
:102FB000D21A554303EB25252AB2EBE70B2B36D863
:102FC000002D03DC22892A4B9847E5E7FE2D01DD21
:102FD000A289F8E72389A689227AC5F1FF0CC3F3F9
:102FE00045130CFB03F3C6F3451615FB0636237B8E
:102FF00002F01F020CFB02F203F01F0348F28107EC
:1030000015FB03237E437B43C6F3C556C3F3C4536A
:1030100043EA4613667A627BF608D2080CFB06FC8C
:1030200015FB02C27A43D20D43EAC222CBE70D2B35
:103030000FD8002D03DC227A0E4B9847ACE7FE2D0B
:10304000227BF9DC237AD21A554303EB2525EAB219
:10305000F2E77F2DD4BFA268E268074B98479BE751
:103060003D240000B55C000075580000392D0000BB
:1030700045590000155A0000E95A000073B50B4B82
:1030800005469847044668B9094B0A49009340F63B
:10309000B1220320084EB047084809492A46234672
:1030A0008847FEE7002002B070BD00BF9517000002
:1030B000C5F501009FEE010031E9000003EF0100BA
:1030C0009D1700002DE9FF470D460646002877D1E1
:1030D000894B9847044640B9884B00938849894BEF
:1030E000CF220220884DA84716E0884B3030984701
:1030F000874B04469847074660B9824B8049009346
:10310000D4220320804DA8478248834922463B466B
:103110008847FEE724B90024204604B0BDE8F087C4
:103120004C217E4B2046984794F83530A66166F3D3
:10313000051384F835307A4BE3617A4B23622661BC
:10314000794B304698470138A082784B30469847F3
:103150000138E082764B4C21201D9847B4F8483066
:1031600023F4FF7323F00103A4F84830A38E23F463
:103170007F6323F00F0343F4E063002243F0010375
:1031800004F12800A386C4E910226A4B2263A263DB
:10319000A2876262039098470398002D40F0D88080
:1031A000654B002E00F09C80022120469847F36971
:1031B0002246012130469847604B2046984792E0CE
:1031C000534FB847044660B94E4B4D490093ED222A
:1031D00003204D4DA8475A484F4932462346884759
:1031E000FEE74A4B301D98470446B847074660B98A
:1031F000444B43490093F0220320434DA8474548E0
:10320000454922463B468847FEE7002C83D0434B86
:10321000DFF838914C212046984794F835302660E5
:103220006FF3051384F835303D4BE3613D4B23626A
:103230004FF00008B6F912306382C4F81880404697
:10324000778AC8474FF0320A00FB0AF0EF282BDDDF
:103250004046C847502300FB0A30A02390FBF3F000
:1032600080B23844E082374B204698470128074611
:103270001CD1B6F91480A4F814800020C8474FF080
:10328000640A00FB0AF0EF281FFA88F808DD002026
:10329000C847502300FB0A37A02397FBF3F7BFB2C0
:1032A000A8EB0707278255E70120DAE7B6F9107087
:1032B00027820020C8474FF0640800FB08F0EF2881
:1032C000BFB20BDD0020C847502300FB0830A0230D
:1032D00090FBF3F080B23844A0823BE70120FAE78C
:1032E000012120469847184B00930549054B40F2B1
:1032F00087120120F6E600BF41D90000F4EF01007B
:103300009FEE0100D9F5010031E9000061E60000FF
:103310009517000002EE01009D17000061F000000B
:10332000194B0000814500004DD9000071D9000003
:103330004DE6000039550000450301003927000023
:1033400003EF01007D30000044F0010095D900003A
:10335000544B05F128019847534B04F1100005F137
:1033600010019847B5F93230638695F8303084F80B
:10337000303095F8313084F8313095F8483084F8A1
:103380004830B5F94430A4F84430B5F94630A4F8D3
:1033900046302B6C95F84920236494F8493062F349
:1033A000000384F84930AB69A36195F8343094F890
:1033B0003420DB0963F3C71284F8342095F83420F5
:1033C00094F8343062F3000384F8343095F83430E4
:1033D00094F83420C3F3400363F3410284F83420AB
:1033E00095F8353094F83520C3F3420363F3430274
:1033F00084F8352095F8343094F83420C3F38003F2
:1034000063F3820284F8342095F83430D2B2C3F3E7
:10341000C00363F3C30284F8342095F83430D2B289
:10342000C3F3001363F3041284F8342095F83430A6
:10343000D2B2C3F3401363F3451284F8342095F8F5
:103440003430D2B2C3F3801363F3861284F834208D
:1034500095F83C3084F83C3095F8352094F83530B8
:1034600062F3000384F83530A86B10B10F4B21468E
:1034700098470F4B2846984778B1002E3FF433AF5A
:103480000C4B284698470C4B0390284698470399C5
:103490000A4B02462046984789E6002E7FF487AE05
:1034A00021E700BF295D0000C91C0000511A00007F
:1034B000D5200000DD2200003D230000552800003B
:1034C0002DE9FF41334B04460D4617469847064603
:1034D00068B9314B3149009340F2E5220320304D69
:1034E000A84730483049224633468847FEE72F4BED
:1034F00020469847854204D12D4B20469847874265
:103500003AD020462B4EB04702A92B4B2046984775
:10351000628A2A4B013F1744E782204698470128D8
:10352000ADB20BBFA38A238AC5F1010505F1FF35B2
:103530000ABFED18ED182582E36918BFA58202AA1B
:103540000221204698471E4B2046984718B1C36970
:10355000224601219847271D1A4BDFF87080384614
:10356000984705465DB92046B04794F84930DB07D7
:1035700002D5154B2046984704B0BDE8F081EB69B1
:1035800002AA03212846984729463846C0470546DF
:10359000E8E700BF95170000F9F501009FEE010074
:1035A00031E9000003EF01009D1700009D2300009A
:1035B000ED23000039270000852200007D30000047
:1035C000D5200000F1E60000912C0000FDE600008F
:1035D00073B50F4B04460E469847054668B90D4B28
:1035E0000D49009340F2273203200C4EB0470C489F
:1035F0000C4922462B468847FEE70B4B204698474E
:103600000A4B01463246204602B0BDE870401847DA
:10361000951700001AF601009FEE010031E9000045
:1036200003EF01009D1700009D230000C13400003E
:1036300073B50E4B04460E469847054668B90C4BC9
:103640000C49009340F6D72203200B4EB0470B489D
:103650000B4922462B468847FEE794F83C301E4231
:1036600014BF0120002002B070BD00BF95170000FC
:103670003FF601009FEE010031E9000003EF010079
:103680009D1700007FB5134B04460D46984706462C
:1036900068B9114B1149009340F6DE220320104D0A
:1036A000A84710481049224633468847FEE73F2D79
:1036B00003D894F83D0004B070BD00238DF80D30A0
:1036C00003AA0A4B8DF80C500921204698479DF813
:1036D0000D00F0E79517000053F601009FEE010082
:1036E00031E9000003EF01009D170000D51F000025
:1036F0002DE9F74FDFF894A0DFF894B005460E46A9
:1037000017464FEA122814466DB924F4FE44222CC1
:10371000A3B230D028D8032B2FD0072B14BF002002
:103720004FF4807013E0174B3146284698473146D6
:1037300081462846D04707EB002084B20DF10602EF
:1037400021464846D847012804D1BDF9060003B0F8
:10375000BDE8F08F18F0800FD7D01EB928460A4B6D
:10376000984705460026CFE7312B08D0C02B14BF61
:1037700000201020EBE7FF20E9E70620E7E70F2015
:10378000E5E700BF3D240000D5200000853600009D
:10379000895E00002DE9F74FDFF874A0DFF874B000
:1037A00005460E4617464FEA122814464DB924F432
:1037B000FE44293C012C96BF124B0020B3F80206B0
:1037C00012E0114B3146284698473146814628463B
:1037D000D04707EB002084B201AA21464846D847CB
:1037E000012804D1BDF8040003B0BDE8F08F18F043
:1037F000800FDCD01EB92846044B984705460026AA
:10380000D4E700BFA6F001003D240000D520000051
:1038100085360000115F00002DE9F74FDFF880A02A
:10382000DFF880B005460E4617464FEA12281446C8
:1038300075B924F4FE446D2CA0B22AD048F2AD0331
:10384000984226D02C3818BF4FF0FF30C0B213E09A
:10385000114B314628469847314681462846D04785
:1038600007EB002084B20DF1070221464846D847F5
:10387000012804D19DF8070003B0BDE8F08F18F0CF
:10388000800FD6D01EB92846044B9847054600261F
:10389000CEE70020F0E700BF3D240000D520000067
:1038A00085360000995F00002DE9F74FDFF884A00E
:1038B000DFF884B005460E4617464FEA1228144634
:1038C0006DB924F4FE44BE2CA3B227D048F28E0278
:1038D000934201D07E2B23D1124B984711E0124B1B
:1038E000314628469847314681462846D04707EB5F
:1038F000002084B201AA21464846D847012803D1B6
:10390000019803B0BDE8F08F18F0800FD9D01EB930
:103910002846064B984705460026D1E70448F0E7BD
:103920000020EEE7390301003D240000D52000000F
:10393000683F0200853600002160000070B5046811
:10394000A5882068A17905F00F03082B2A460CD81A
:103950000D4B984720810023A380A17920680B4E4E
:1039600023462A46B047A58070BD0B2B02D8084BD2
:103970009847EFE70D2B03D8064B98472072EAE7EC
:10398000054B9847A060E6E7F1360000652400008B
:103990009537000019380000A93800002DE9F04FD4
:1039A00090F83D308B429FB00446884600F042823A
:1039B000954B9847054668B9944B9549009340F25A
:1039C00037620320934EB0479348944922462B46D2
:1039D0008847FEE794F83D300293002384F83D8049
:1039E00003939DF80C608E4B314620469847059016
:1039F00040B1477917F008070BD0039B0133402BE8
:103A00000393EED1874BFF2120461FB0BDE8F04F56
:103A10001847854DB02231462046A847B12209906B
:103A200031462046A847814B0890BE2231462046A9
:103A30009847B222069031462046A847B322ADF8F7
:103A40002C0031462046A847B422ADF82E0031465E
:103A50002046A847B522ADF8300031462046A84799
:103A6000B622ADF8320031462046A847B722ADF85D
:103A7000340031462046A8470497ADF83600049A32
:103A80000BAB33F81270002F00F0B680684B05982E
:103A90009847634B314620469847664B0546984702
:103AA00007F00F03082B824600F2DC806B79DFF809
:103AB00078B143F004036B71029B84F83D303A46C1
:103AC00031462046D8473A46079084F83D80314633
:103AD0002046D8476A79079B6FF38202834281466A
:103AE0006A7100F08980029B84F83D303A46314685
:103AF0002046D847504B84F83D80024683463946DD
:103B000050469847012F22D147F6FF739B4501D0BD
:103B100099451CD1DFF848A12046D04700EBD07072
:103B200040F34F052046D04747F6FF7200EBD070B8
:103B3000934540F34F032AD19D421EDA05F1010B54
:103B400091450FFA8BFB02D101350FFA85F93B4BFA
:103B50003B4898472C4B054698478246E0B9394B7D
:103B60002B49009340F6B26203202A4CA047364806
:103B70002A492A4653468847FEE703F1010B91453F
:103B80000FFA8BFBE3D101330FFA83F9DFE791459D
:103B9000DDD19D42F7DAD7E7002D2DD0A5F808B08A
:103BA000A5F80C90294B2C60AF80AE710EA89847F9
:103BB000274B0F93274B1093274B11930022FF2382
:103BC000CDE91423099B1693089B069A0E955B4238
:103BD0001793069BD11D013B12AA13F8010F02F89F
:103BE000010B9942F9D19DF86E306FF300038DF807
:103BF0006E300EA8194B9847049B0133062B049393
:103C00007FF43DAFF9E600BF95170000AAF601006A
:103C10009FEE010031E9000003EF01009D17000055
:103C20003D240000392D0000F1360000A9380000C5
:103C3000DD5D0000B55C00007558000061E6000025
:103C400060860020BBF6010002EE0100BDDC000032
:103C5000712F00003D3900005125000065DD000096
:103C60009D2300000B2B4BD86B79DFF800B243F09B
:103C700004036B71029B84F83D303A46314620467E
:103C8000D8473A46814684F83D8031462046D84799
:103C90006A79ADF81C006FF382026A711FFA89F924
:103CA00082B29145A8D0029B84F83D303A46314615
:103CB0002046D84739460246604B84F83D8081460D
:103CC000504698475E4B5F4898475F4B054698477C
:103CD000824668B95D4B5E49009340F6C662032098
:103CE0005C4CA0475C485D492A4653468847FEE73E
:103CF000002D81D0BDF81C30A5F80890AB8151E7AC
:103D00000D2B49D86B79DFF868B143F004036B7170
:103D1000029B84F83D303A4631462046D8473A4621
:103D2000079084F83D8031462046D8476A79079B42
:103D30006FF38202834281466A713FF45DAF029B5A
:103D400084F83D303A4631462046D8473946024647
:103D5000434B84F83D80834650469847384B39485A
:103D60009847394B05469847824668B9374B3849DA
:103D7000009340F6DB620320364CA04736483749B3
:103D80002A4653468847FEE7002D3FF435AF85F8B5
:103D900008B085F80C9005E7029B84F83D306B79FC
:103DA000DFF8D0B043F004036B713A463146204649
:103DB000D8473A460A90314684F83D802046D84795
:103DC0000E906B796FF3820381466B710422254B51
:103DD0000EA90AA8984700283FF40EAF029B84F86A
:103DE0003D303A4631462046D847394602461E4BBA
:103DF0000A90834684F83D8050469847104B1148FE
:103E00009847114B05469847824668B90F4B1049B1
:103E1000009340F6EF6203200E4CA0470E480F4976
:103E20002A4653468847FEE7002D3FF4E5AEC5E934
:103E300002B9B7E61FB0BDE8F08F00BF45590000DA
:103E400061E600006086002095170000BBF60100C7
:103E50009FEE010031E9000002EE01009D17000015
:103E6000155A0000D9620100E95A00009537000098
:103E700019380000A938000073B5114B04460D46EF
:103E80009847064668B90F4B0F49009340F27E628F
:103E900003200E4DA8470E480E4922463346884758
:103EA000FEE794F83D3043EA050135EA030305D007
:103EB000094B204602B0BDE87040184702B070BD03
:103EC00095170000C8F601009FEE010031E90000DF
:103ED00003EF01009D1700009D39000073B5114BE1
:103EE00004460D469847064668B90F4B0F490093A4
:103EF00040F28F6203200E4DA8470E480E4922461D
:103F000033468847FEE794F83D301D4223EA050119
:103F100005D00A4B204602B0BDE87040184702B0F9
:103F200070BD00BF95170000D9F601009FEE01009B
:103F300031E9000003EF01009D1700009D390000EA
:103F400073B50B4B04469847054668B9094B0A49B7
:103F5000009340F6F5220320084EB047084809496F
:103F600022462B468847FEE7E06902B070BD00BFDD
:103F700095170000ECF601009FEE010031E900000A
:103F800003EF01009D17000073B50B4B04469847E3
:103F9000054668B9094B0A49009340F61E320320D2
:103FA000084EB0470848094922462B468847FEE795
:103FB000606A02B070BD00BF951700002AF70100CB
:103FC0009FEE010031E9000003EF01009D170000A2
:103FD00073B50B4B04469847054668B9094B0A4927
:103FE000009340F66F320320084EB0470848094955
:103FF00022462B468847FEE7A06B02B070BD00BF8B
:10400000951700004EF701009FEE010031E9000016
:1040100003EF01009D1700002DE9F047394B0446DE
:10402000002215219847384B20469847074610B183
:10403000364B20469847364B364DDFF8F49000213A
:1040400020469847FF2200231146204604F1040829
:10405000A847314B4046984705463DBB2F4B5E680D
:10406000012366BBDFF8CC80DFF8CC90DFF8CCA072
:104070003046C047054645BB2A462946E369284DD8
:1040800020469847274B20469847002837D1264B93
:104090002046984721463030A847606A234D00B13A
:1040A000A84720462B46BDE8F0471847294640461A
:1040B000C84706462846FFF7AFFF3546CDE73268CA
:1040C000944208BF3371B668CBE76B6BA34202D052
:1040D000AB6BA34202D121462846C847EB6BA342F3
:1040E000AB6D08BFEE63BB4205D1D047844202D11D
:1040F00021462846C8472846C0470546BBE7214613
:104100000430C9E7291F0000D13F0000291B00002F
:10411000F5DC000065240000F1E60000F4800020DA
:10412000B5E70000D5200000752100002DEB000050
:10413000FDE600005DDA00002D1C0000651C00009B
:10414000F7B51B4B04469847054668B9194B1A4901
:10415000009340F293120320184EB04718481949B3
:1041600022462B468847FEE7174B20469847174BB9
:10417000204698470646B8B9154B2046984705464D
:1041800078B1C76B3B1B5F425F41124B204698479B
:1041900026B1F36900220121304698470FB1002370
:1041A000EB63002003B0F0BD00273D46EDE700BF04
:1041B000951700005FF701009FEE010031E9000054
:1041C00003EF01009D17000039270000D5200000F3
:1041D000752100001940000073B50E4B0446984746
:1041E000054668B90C4B0D4900934FF43862032023
:1041F0000B4EB0470B480C4922462B468847FEE73A
:10420000A06B20B1094B9847231A5842584102B07D
:1042100070BD00BF951700008BF701009FEE0100F5
:1042200031E9000003EF01009D170000C51B0000ED
:1042300007B5028A90F83030D21AADF80020828A91
:104240001344ADF80430428A90F83130D21AADF8F8
:104250000220C28A1344ADF806300022024B6846A1
:10426000984703B05DF804FB69DF000010B5002338
:1042700050F82340DAB21CB10133072BF8D11A46AB
:1042800040F82210012010BD2DE9F0471446B74F29
:10429000DFF8E482012205460E46B84748F20C02D8
:1042A000208031462846C047052881460AD8002389
:1042B0002373237584F8283084F8363084F844302A
:1042C000BDE8F087237B43B32C2231462846C04704
:1042D0000528207321D929223146DFF894A22846E7
:1042E000D0472322608031462846B847C0B2A0712B
:1042F00070B12A2231462846D0472122A08031467B
:104300002846B8472222208131462846B847608196
:10431000202231462846B8476073237DEBB1302216
:1043200031462846B8472082B8B13C22314628465B
:10433000C047052820750BD9312231462846B84799
:10434000C0B260828A4B3922314628469847E081C4
:10435000322231462846B8476075237FE3B14022B8
:1043600031462846B8472083B0B14C223146284612
:10437000C047052820770AD9412231462846B84748
:104380007B4B60834922314628469847E08242228F
:1043900031462846B847607794F83630002B3BD03A
:1043A000DFF8D8A16E2231462846D047E0620028C7
:1043B00032D06C2231462846C047052884F83600A2
:1043C0002AD96D2231462846C047612284F8370039
:1043D00031462846B84794F83830003818BF0120D5
:1043E00060F3000384F83830E06A624B9847022893
:1043F00040F0AF805E4B692231462846984748F22C
:104400008E02A08631462846D0472063602231467E
:104410002846B84784F8390094F82830052B28D965
:10442000502231462846B847208410B35C223146DA
:104430002846C047052884F828001AD95122314659
:104440002846B8475222608431462846B84753224E
:10445000A08431462846B847454BE084592231466E
:10446000284698475422E08331462846B84784F8C6
:10447000290094F84430052B40D9DFF800A17F22B1
:1044800031462846D047E063002837D07C223146A9
:104490002846C047052884F844002FD973223146A6
:1044A0002846B8477422A4F8480031462846B84741
:1044B0002F4BA4F84A0079223146284698477E229D
:1044C000A4F8460031462846D04770222064314681
:1044D0002846B8477122A4F84C0031462846B84710
:1044E0007522A4F84E0031462846B847722284F857
:1044F000500031462846B84784F85100B9F1F90F09
:104500003FF6DEAE237B1FFA89F013FB00F3C3F303
:1045100007232373237D13FB00F3C3F307232375C2
:1045200094F8283013FB00F3C3F3072384F82830F2
:1045300094F8363013FB00F3C3F3072384F83630C6
:1045400094F8443013FB00F0C0F3072084F84400D3
:10455000B6E694F83730052B7FF658AF044B692246
:10456000314628469847A08650E700BFF136000044
:10457000953700001178000019380000A9380000B4
:104580002DE9F04F022A99B004460F46154659D13D
:10459000DFF814920021C8470646002850D1014692
:1045A00001222046C8470422824631462046C84799
:1045B0000522834631462046C847774B804604F1A2
:1045C000100103A89847BDF80C30BDF80E201FFA63
:1045D0008BF01B1AADF80C30BDF810301844ADF854
:1045E0001000BDF812001FFA88F3D21A0344ADF888
:1045F0000E20ADF812305246684B03A93846984752
:10460000D0B1674F2C2231462046B847F92813D93C
:10461000314620222046C84710F0FF010CD132223B
:104620002046C84710F0FF0106D148F20C02204690
:10463000B847F92888BF0125284619B0BDE8F08F92
:104640000325F9E7002A56D1564B574E03A8984741
:10465000332229462046B047B04608B18DF8205095
:10466000524B03AA002120469847042200212046ED
:10467000C0470522064600212046C04704F1100924
:10468000454B8246494601A89847BDF80800BDF849
:104690000420B3B2D21A0344ADF80830BDF8063096
:1046A000ADF804201FFA8AF01B1AADF80630BDF8E9
:1046B0000A301844ADF80A0003AA394601A83C4B59
:1046C0009847022200212046C0470028B4D0394B29
:1046D000394F1C2098470122064600212046C0473A
:1046E0004946024600233046B847344B04F518715A
:1046F00030469847A0E7012A01D000259CE72A4DC3
:1047000002220021A847A84628B12D4B04F51870B5
:1047100098472C4B9847332200212046C047002859
:10472000EBD0002503A81F4B9847204B8DF818505D
:1047300003AA294620468DF842508DF834509847F8
:10474000294604222046C04705220646294620461F
:10475000C04704F1100180460F4B01A89847BDF8EF
:104760000800BDF80420B3B2D21A0344ADF80830F3
:10477000BDF80630ADF804201FFA88F01B1AADF81A
:104780000630BDF80A301844ADF80A00084B03AAF9
:10479000394601A898474FE7C91C0000D9E000003E
:1047A00019380000B59B0000F13600008942000076
:1047B000019C0000FDEE0000259900001997000003
:1047C000D5970000B1EB00002DE9F0411446284FC9
:1047D00048F28C0205460E46B8470528207245D996
:1047E00048F20C0231462846B847F9289FBF237A81
:1047F00013FB00F0C0F307202072237A052B35D974
:1048000048F289023146DFF874801A4F2846C047C3
:1048100048F28002208031462846B84748F281029B
:10482000A08131462846B84748F28202608131466D
:104830002846B84748F28302207631462846B847D2
:104840000D4B607648F28E02314628469847E28941
:1048500060604FF6FF739A4208D0228A9A4205D0D0
:1048600048F28A0231462846C0472080BDE8F081E0
:1048700019380000F1360000A93800009537000013
:10488000F8B51446234F48F2AC0205460E46B84729
:10489000052820703CD948F20C0231462846B8471A
:1048A000F9289FBF237813FB00F0C0F30720207086
:1048B0002378052B2CD9002363804FF48073238148
:1048C000AB8A2A8A01339B1AC3F3C03202FA83F3FC
:1048D0005B10A380EB8A6A8A01339B1AC3F3C03250
:1048E00002FA83F35B10E38048F2AD0231462846BA
:1048F000B847094BA07248F2A902314628469847AA
:10490000064BA08148F2A002314628469847A07382
:10491000F8BD00BF1938000095370000F1360000DF
:104920002DE9F0475022774F8AB004460E46B8472B
:104930000546002840F0B7800025DFF8D0917F229F
:1049400031462046C8478046002800F081806E4BE3
:104950007C22314620469847052879D97022314675
:104960002046B8477022059031462046B8477E223F
:10497000824631462046C8474FF0000947F61841A5
:10498000CDE9011902464146059BDFF88481CDF847
:1049900000A006A8C047BDF81830ADF82090013B34
:1049A000ADF82430BDF81A30ADF82290013B7522E5
:1049B00031462046ADF82630B8477322824631464C
:1049C0002046B8477422814631462046B8475FFAF0
:1049D0008AF2804607AB08A904F11000DFF834A181
:1049E000D047BDF81C30BDF82010B4F91020BDF838
:1049F0001E004B4411FA83F109B2521AAA42B8BF01
:104A00002A46BDF822504044114615FA80F5B4F903
:104A100012202DB2551B0AB29542B8BF1546BDF8FB
:104A2000242012FA83F3B4F914201BB29B1A2DB27E
:104A3000AB42B8BF2B46BDF8265015FA80F5B4F945
:104A400016002DB22D1A1BB2AB42B8BF2B461DB2B9
:104A5000402231462046B847804678B12A4B4C2246
:104A6000314620469847052808D94122314620463C
:104A7000B84740448542B8BF05462DB231460422AE
:104A80002046B8470522804631462046B847404573
:104A9000B8BF404600B20028C4BF2D182DB228462A
:104AA0000AB0BDE8F087184B5C2231462046984793
:104AB00005287FF641AF532231462046B84705EB23
:104AC000D57500EB6505512231462046B847522284
:104AD000804631462046B8470028B8BF4042B8F16A
:104AE000000FB8BFC8F100080135ADB280B21FFA9F
:104AF00088F840452CBF2D1845442DB225EAE575B0
:104B00001BE700BFF136000019380000A93800008B
:104B1000FD01010079E10000082910B5044608D123
:104B200013781BB928345460012411E0002353602A
:104B3000FAE7072905D1BDE810402749274B104661
:104B40001847012906D1264B984780F00100C4B2CE
:104B5000204610BD062909D1224B00219847B4F9FF
:104B600032309842B8BF18466086DDE7032907D186
:104B700090F8494014F00104D6D01B4B9847E7E762
:104B8000042902D1194B9847CEE70B2903D1184BC2
:104B900010219847C8E7A1F10D02012A02D810217F
:104BA000144BF6E716290ED1134B9847134B984731
:104BB0000F4B10B106212046EBE702212046984713
:104BC00004212046ECE7172901D10621F9E7002945
:104BD000AAD10B4BDDE700BF9FF001006D42000042
:104BE0003136000021490000912C00008120000096
:104BF000793E0000DD3E0000D13F0000CF1B0000E9
:104C0000F924000038B5174D174B28689847174B03
:104C100004462868984758B9286801234268A36168
:104C2000116AC90709D400230AE0C3690BB1984788
:104C30002868A369002BF8D1EEE7126A9207F2D533
:104C4000E361C3681BB1A26804F1100198472268B0
:104C500032B1636823B1A1688A4218BF1346A360CA
:104C600038BD00BF0081002025DA000029DA0000ED
:104C70002DE9F84300220C46174B103107469847A0
:104C800010B90020BDE8F88394F83430DB06F8D47E
:104C9000236A9BB1022239462046984703280646DC
:104CA000EFD004F104080D4BDFF8349040469847EC
:104CB00005462DB9012EE4D12046E3E70226F0E7B0
:104CC00029463846FFF7D4FF0028DBD12946404665
:104CD000C8470546EDE700BFD9E00000F1E6000057
:104CE000FDE600002DE9F04390F8349019F010092A
:104CF0008BB0044688463CD1B0F93250314E324F29
:104D000004A9B047BDF81020ABB2D21AADF81020FC
:104D1000BDF81220D21AADF81220BDF814201A44A2
:104D2000ADF81420BDF816204146134402A804AA89
:104D3000ADF81630B847E0B1236A1BB14A4602A964
:104D40002046984704A92046B04704AA4146684631
:104D5000B84740B104F104081C4BDFF8749040469A
:104D60009847054645B9236A1BB1012202A920468E
:104D700098470BB0BDE8F08308A92846B0476B8E72
:104D8000BDF82020D21AADF82020BDF82220D21A7A
:104D9000ADF82220BDF824201A44ADF82420BDF837
:104DA00026206946134406A808AAADF82630B8475D
:104DB00018B106A92846FFF795FF29464046C8477F
:104DC0000546CFE785220000D1DE0000F7E60000AF
:104DD0001DE700002DE9F0470E46044628B9154BA3
:104DE0001868154B9847044658B131462046134F72
:104DF000DFF84C80DFF84C90B8472046C0470546A6
:104E00000DB9BDE8F08705F1040A21465046C847B0
:104E1000044650B92B6A1BB10122314628469847F7
:104E20002846C0472C460546EAE731462046B847A3
:104E3000EBE700BF0081002025180000E54C0000D2
:104E4000D52000001DE7000073B51A4C1A4B06462A
:104E500020689847194B05462068984720B305F10C
:104E600010023146164B174D68469847164B20687E
:104E70009847164B0146684698476946A847144B21
:104E8000206898476946A847124B206898476946AA
:104E9000A8472068104B984708B9104B984702B0B4
:104EA00070BDC3690BB198472068AB69002BF8D17E
:104EB000D5E700BF0081002025DA000029DA0000D4
:104EC000D1DE0000D54D000025180000714C000017
:104ED000611800009D18000039DA0000054C000040
:104EE000013900F1080311F8012F00F8012B984255
:104EF000F9D17047704700002DE9FF410D46044687
:104F000018B92F4B9847044630B145B9B4F8683109
:104F100065F30903A4F8683104B0BDE8F08100230B
:104F2000ADF80030ADF802302046264B98470138E6
:104F3000254BADF80400204698470138ADF806002F
:104F4000224B6A46294602A898470028E4D02369E4
:104F500013B102A92046984704F14805DFF878808C
:104F600000262F46B4F86831B2B2C3F3090090426C
:104F70001CD81F289BBF0930C0F309006FF3090339
:104F800002A991BF04EBC000A4F868316946384615
:104F90000F4A9047B4F86831E06A5A1C62F309037B
:104FA000A4F8683103210B4B9847B5E72946002246
:104FB00002A8C047013608350028D3D0ACE700BFAF
:104FC00041D900004DD9000071D90000D1DE0000A8
:104FD000E14E0000C9FB0000D9E00000014B186859
:104FE000704700BF008100202DE9F04F2DED028BAE
:104FF000834B844C8BB005469847EB6823600021B7
:10500000814B08EE900A284698472368D96B0029FF
:1050100040F08B80B3F8682161F30902A3F868219E
:105020000BB0BDEC028BBDE8F08F334493F84851D0
:10503000002D3CD001362368B3F86821C2F3090182
:105040008E42F2D300206060002971D16D4F386824
:10505000B0F86831C3F3090303B36C4B98470028D9
:1050600040F0A58120686A4D4FF480714830A84710
:105070002068202100F5A470A8472368B3F86821B0
:105080006FF30902A3F8682118EE900A614B984764
:10509000014620688369002B40F0E1815E4B984710
:1050A0005E4B0BB0BDEC028BBDE8F04F18474FEAEA
:1050B000C609DFF888A109F148092068B0F868310D
:1050C000C3F309039D42B5D2431993F8483153BB4A
:1050D000AE4228D04FEAC50B0BF1480B00EB0B0199
:1050E0004844B847F8B121684D4B01EB0B0208A8C2
:1050F0004944984708A8D047804620684844D0478C
:10510000039020685844D047039B184480450AD236
:10511000D4F800B0434B0BEB090008A9AB44984707
:1051200001238BF848310135C7E73F4F002682E75E
:105130004F1E03F5A472791C5CD100275B68DFF871
:10514000C48093F820206FF3000283F8202093F8A6
:1051500020206FF3410283F820204FF0000BD8F895
:105160000090B9F86831C3F309039B45BFF66EAFF1
:1051700009EB0B0393F84831002B40F0CA80D9F8B3
:105180000430BB4502BF93F8202042F0010283F8AF
:10519000202093F820204FEACB056FF3410283F8DB
:1051A000202005F1480304934B4408EE103A48468A
:1051B000164B98471D4B002842D020689847002680
:1051C00005461B4B0682206898470138194BA88278
:1051D0006E8220689847236801385A68E88292F8FE
:1051E000203043F0020382F8203018EE100A124BF0
:1051F000984781E0D15D0029A0D0013F9BE700BF27
:105200008DDA000000810020C9FB000039DA0000BF
:1052100061F00000A1DA000025EC000085D7000055
:1052200025DF0000E14E00009DE0000025DA0000CF
:105230004DD9000071D90000494E0000B5DE0000D4
:105240004D4420689847B5F84C90B5F84830B5F90A
:105250004E20039209F10109A9EB0309B5F84A3080
:1052600002F1010AAAEB030A06467E4B2068984722
:10527000039A7C4B82420FFA89F90FFA8AFA4BDBC8
:1052800020689847013803B2F268B2FBF9F9D8F800
:1052900000201269CA45A8BFCA46002A43D000228E
:1052A000ADF82020ADF82420ADF822200FFA8AF9BD
:1052B000D8F80000CDF80C9009F1FF390FFA89F900
:1052C0000269ADF8269008A905939047BDF926100C
:1052D000BDF82220059B01318A1A12B292451EDACE
:1052E000B9F1000FE4DC604B00936049604B614D05
:1052F0004FF4CF720220A847D8F80000836943B169
:10530000049B18445C4B9847D8F804301844C8F8FC
:1053100004000BF1010B22E7B5F94E30B4E7039A14
:10532000002AE0DD8A461FFA8AF1481EB5F94A20B4
:1053300005904FF0000902EB0A00013898420CDD9D
:105340004B45D9D0B5F9480021683082B5F94C00F9
:10535000B0827282F3824A6841E7B5F94800308230
:10536000B5F94C00B08290B203900598728210FAA1
:1053700082F90FFA89F99945A8BF99464B45A6F8D5
:10538000169008D1D8F80020506890F8202042F0FC
:10539000020280F82020394A18EE100ACDE90631C1
:1053A0009047039A0799069B0A4412B2C3E73868EC
:1053B0004369002B7FF456AE314B9847314B05467D
:1053C0009847AB69002BFCD1D5F80090D5F808B010
:1053D0002D4B3868D94508BFD5F80490984700256B
:1053E000804643003A68B2F86811A8B2C1F30901D7
:1053F00081427FF637AE511991F8481109B1013554
:10540000F0E702EBC502B2F94800B2F94A60B2F81F
:105410004C20013208FB0601121A05F1090012B2F4
:10542000C0000BEB410A4FEA420C09EB410103902B
:105430003868039A1044B0F90600B042DFDB0693E7
:105440006246124B5046CDE9041C9847069B0499CE
:10545000DDF814C0013636B29A441944E8E76268B0
:1054600098471BE671D90000CDF701009DF70100B8
:105470001DF8010031E90000B5DE0000494E0000D2
:1054800025DA0000054C00004DD9000079EC000041
:10549000437903F00603062B08BF0131037908BFE7
:1054A000C9B28B4286BF036853F8210000207047C1
:1054B000F0B578B34FF0FF32CFB24FEA112C002392
:1054C0001646C1F30624C15CFF2901D1104609E04C
:1054D0008F4211D1C5186D788CEA050E1EF07F0F32
:1054E00001D11846F0BD05F07F0535EA040E03D161
:1054F000B542C4BF2EB21AB201F00F01082902D87A
:1055000002330233DFE70B29FAD90D2994BF0133A7
:105510000433F6E74FF0FF30E4E70139024411F8B5
:10552000013F00F8013B9042F9D17047014B042143
:10553000184700BF61F00000014B0821184700BF69
:1055400061F00000F7B5037904460E464BB10068E0
:10555000002250F82210B1423CD00132D1B28B422D
:10556000F7D803B0F0BD013B9900214B9847214B80
:1055700005469847074668B91F4B204900934FF4EA
:10558000827203201E4CA0471E481F492A463B46F4
:105590008847FEE74DB1002321791A46D8B28842E8
:1055A0000DD3013921712560DBE7184B00931349B6
:1055B000114B134C4FF483720220A047D1E72068AF
:1055C00050F82300B0421EBF45F822000132D2B28B
:1055D0000133E3E7012BC6D10D4B9847002323602D
:1055E000A38823F4FF7323F00103A380B9E700BF6E
:1055F0005DEE00009517000033F901002AF8010064
:1056000031E9000002EE01009D1700005BF8010087
:105610002DEB00002DE9F3410F46054638B3294B29
:1056200098472979A1B9284B04209847274B04466D
:105630009847064690B9264B26490093D02203206E
:10564000254DA84725482649224633468847FEE788
:1056500001312868234B89009847E7E754B9224B6A
:1056600000931C491A4B1C4CD2220220A04702B0C6
:10567000BDE8F0816B792E79C3F34008DB0748BFA2
:1056800008F10108A6EB0802D2B24645C2F10100BA
:1056900006F180414FEA800001F1FF3138BF04205C
:1056A00000EB810100EB86004FEA82020F4B38BF0E
:1056B0000022214420440136984744F828702E7176
:1056C0002C60D4E74555000075EA000095170000EE
:1056D0004FF901002AF8010031E9000002EE010053
:1056E0009D1700005DEE000096F8010015630100B3
:1056F0004379DB0773B5054605D51A4B002102B087
:10570000BDE870401847184B04209847174B0446D3
:105710009847064668B9164B1649009340F2354241
:105720000320154DA847154815492246334688479A
:10573000FEE75CB9134B00930E490D4B0E4D40F242
:1057400037420220A847204602B070BD0E4B2046CB
:1057500098470E4B2146284698476B7943F0010342
:105760006B71F0E79154000075EA00009517000096
:1057700068F901002AF8010031E9000002EE010099
:105780009D170000C6F801002D55000015560000B9
:1057900010B5034B0446006898470023236010BDF2
:1057A0002DEB0000006828B10023C25CFF2A02D163
:1057B000023398B2704702F00F02082A02D802336F
:1057C0000233F2E70B2AFAD90D2A94BF01330433CE
:1057D000F6E7000037B505460C4679B10B686BB1AA
:1057E0000846074B9847074B019098472860019A55
:1057F0002168054B03B0BDE83040184703B030BD09
:10580000A557000075EA000079EC0000F8B50F46D6
:10581000044630B30668144B30469847051E20DB1B
:105820002E44737883EA17235B061AD10F4B204668
:1058300007F00F0198470B290CD90E2934BF032319
:105840000623C11AA942206806D8094B9847206050
:105850000120F8BD0423F4E74219D25C425501351A
:10586000F0E70020F5E700BFB1540000A5570000A5
:105870005DEE000070B50668284B86B005463046E0
:10588000ADF80E10ADF80C200C46984700280DDB43
:1058900033185B7883EA14235B0607D10230204B70
:1058A000022203A93044984706B070BDFF23ADF82B
:1058B000163028461B4B9847041E08BF02240434A8
:1058C000A4B2194B214630469847184B2860984798
:1058D000064668B9164B174900934FF4C37203206C
:1058E000154CA0472A681548154933468847FEE7F6
:1058F00028680B4EA31F0DF10E0118440222B04779
:105900002868231F03A918440222B0472868023CD4
:1059100002220DF116012044B047C5E7B154000042
:105920001B550000A55700005DEE00009517000014
:105930007EF901002AF8010031E9000002EE0100C1
:105940009D17000070B50668284B86B005463046A6
:10595000ADF80C20ADF80E100C46984700280DDB72
:1059600033185B7883EA14235B0607D10230204B9F
:10597000022203A93044984706B070BDFF23ADF85A
:10598000163028461B4B9847041E08BF02240434D7
:10599000A4B2194B214630469847184B28609847C7
:1059A000064668B9164B1749009340F2B51203201A
:1059B000154CA0472A681548154933468847FEE725
:1059C00028680B4EA31F0DF10E0118440222B047A8
:1059D0002868231F03A918440222B0472868023C04
:1059E00002220DF116012044B047C5E7B154000072
:1059F0001B550000A55700005DEE00009517000044
:105A000090F901002AF8010031E9000002EE0100DE
:105A10009D17000070B50668294B86B005463046D4
:105A2000ADF80E108DF80D200C46984700280EDBBF
:105A300033185B7883EA14235B0608D10230214BCC
:105A400001220DF10D013044984706B070BDFF23CF
:105A5000ADF8163028461C4B9847041E08BF022498
:105A60000334A4B2194B214630469847184B28609E
:105A70009847064668B9174B174900934FF4F272DE
:105A80000320164CA0472A68154816493346884714
:105A9000FEE728680B4E631F0DF10E011844022229
:105AA000B0472868E31E0DF10D0118440122B047EC
:105AB0002868023C02220DF116012044B047C4E7D9
:105AC000B15400001B550000A55700005DEE00001A
:105AD00095170000A4F901002AF8010031E900003F
:105AE00002EE01009D17000070B50668284B86B0D5
:105AF000054630460292ADF80E100C469847002835
:105B00000DDB33185B7883EA14235B0607D1023080
:105B1000204B042202A93044984706B070BDFF23F1
:105B2000ADF8163028461C4B9847041E08BF0224C7
:105B30000634A4B2194B214630469847184B2860CA
:105B40009847064668B9174B1749009340F213224D
:105B50000320164CA0472A68154816493346884743
:105B6000FEE728680B4EA4F108030DF10E0118445E
:105B70000222B0472868A31F02A918440422B04794
:105B80002868023C02220DF116012044B047C4E708
:105B9000B15400001B550000A55700005DEE000049
:105BA00095170000B6F901002AF8010031E900005C
:105BB00002EE01009D1700002DE9F0410E46174648
:105BC0000546C0B1D0F80080B8F1000F13D00B4BE0
:105BD00040469847041E0EDBA11C094B38460222A2
:105BE00041449847286804446378C3F3060303EAF2
:105BF0001620BDE8F0814FF0FF30FAE7B154000005
:105C00001B5500002DE9F0410E4617460546C0B170
:105C1000D0F80080B8F1000F13D00B4B40469847E6
:105C2000041E0EDBA11C094B384601224144984753
:105C3000286804446378C3F3060303EA1620BDE82A
:105C4000F0814FF0FF30FAE7B15400001B5500001F
:105C50002DE9F0410E4617460546C0B1D0F8008048
:105C6000B8F1000F13D00B4B40469847041E0EDBD3
:105C7000A11C094B38460422414498472868044433
:105C80006378C3F3060303EA1620BDE8F0814FF002
:105C9000FF30FAE7B15400001B550000427912F0C2
:105CA000010305D0036892074CBF58681868704715
:105CB00018467047437913F002031ABF0368186847
:105CC0001846704738B5044628B34379DA0708D533
:105CD000114B9847054620B1104B9847104B28466A
:105CE000984763799B0709D50E4B20469847054690
:105CF00020B10A4B98470A4B28469847237913B19D
:105D00002068074B984700232360A38823F4FF6390
:105D100023F00703A38038BD9D5C0000915700006D
:105D20002DEB0000B55C000070B50C46264B054617
:105D300098472368B3B163792079244E13F0010F9B
:105D400003F00202224B17D16AB101388000984754
:105D5000286022792168013A92000431B047237902
:105D6000013B2B7170BD8000984728602279216823
:105D70009200B0472379F4E7C2B102388000984717
:105D8000286022792168023A92000831B0472379CD
:105D9000023B2B710F4E2846B04705462046B047C0
:105DA0000D4B01462846BDE8704018470138800079
:105DB0009847286022792168013A92000431B0475F
:105DC0002379013BE5E700BFC55C000079EC0000EA
:105DD00075EA0000F1560000D557000043799A0794
:105DE00073B5054604D51D4B02B0BDE87040184799
:105DF0001B4B042098471B4B04469847064668B93E
:105E0000194B1A49009340F2CD220320184DA847A0
:105E100018481949224633468847FEE75CB9174BB4
:105E200000931249104B124D40F2CF220220A84796
:105E3000204602B070BD124B204698472146114BB8
:105E4000284698476B7943F002036B71DB0742BF2A
:105E50002B68D3E90021C3E90012E9E7B55C000033
:105E600075EA000095170000C8F901002AF8010042
:105E700031E9000002EE01009D170000F3F8010077
:105E80002D550000155600002DE9F74F0F4690469E
:105E9000054618B3006808B300261B4BDFF86CB04A
:105EA000ADF806604FEA112A4FF0FF342A790FFA55
:105EB00086F9914503DBE043C0F3C0300EE0F1B258
:105EC000284698470DF106023946D84782450E4BC1
:105ED00007D1BDF80630A8F80030012003B0BDE8B6
:105EE000F08F6A79910706D5002804DBB9F1000F1D
:105EF00001D15207EDD58442BEBFBDF80620A8F8F7
:105F0000002004460136D1E791540000B95B00003F
:105F10002DE9F74F0F469046054610B3006800B3D1
:105F200000261B4BDFF86CB0ADF804604FEA112A75
:105F30004FF0FF342A790FFA86F9914503DBE043ED
:105F4000C0F3C0300DE0F1B22846984701AA3946A7
:105F5000D84782450E4B07D1BDF80430A8F8003071
:105F6000012003B0BDE8F08F6A79910706D50028BB
:105F700004DBB9F1000F01D15207EDD58442BEBF59
:105F8000BDF80420A8F8002004460136D2E700BF7F
:105F900091540000B95B00002DE9F74F0F46904681
:105FA000054618B3006808B300261B4BDFF86CB039
:105FB0008DF807604FEA112A4FF0FF342A790FFA63
:105FC00086F9914503DBE043C0F3C0300EE0F1B247
:105FD000284698470DF107023946D84782450E4BAF
:105FE00007D19DF8073088F80030012003B0BDE8E4
:105FF000F08F6A79910706D5002804DBB9F1000F0C
:1060000001D15207EDD58442BEBF9DF8072088F824
:10601000002004460136D1E791540000055C0000E1
:106020002DE9F74F0F4690460546F8B10068E8B1F4
:10603000194BDFF868B04FEA112A00264FF0FF3401
:106040002A790FFA86F9914503DBE043C0F3C030AB
:106050000CE0F1B22846984701AA3946D847824554
:106060000D4B06D1019BC8F80030012003B0BDE8FC
:10607000F08F6A79910706D5002804DBB9F1000F8B
:1060800001D15207EED58442BEBF019AC8F8002064
:1060900004460136D4E700BF91540000515C000073
:1060A000F0B5C2F1FF03C1F34514C0F345155C43DD
:1060B00048F2810605FB02447443C4F3C55501F060
:1060C0001F0400F01F075C43C1F3C42107FB024417
:1060D000C0F3C420594300FB021374437343C4F359
:1060E000C45444EA4514DB0D44EAC320F0BD00006B
:1060F0000B46052AF0B403F01F07C3F34515C3F39D
:10610000C42402D80846F0BC7047C0F3C42323441B
:10611000C0F345142C441F2B00F01F053D4428BF3D
:106120001F233F2C28BF3F241F2D28BF1F25FF2AD8
:1061300003F01F0304F03F0405F01F0508D14FF0E2
:10614000000065F3040064F34A1063F3CF20DAE73C
:1061500065F3040064F34A1063F3CF20F0BC014BF5
:10616000184700BFA16000000B46052AF0B403F0F9
:106170001F06C3F34515C3F3C42402D80846F0BC78
:106180007047C0F3C423E31AC0F345142C1B00F07E
:106190001F05751B23EAE37324EAE47425EAE57519
:1061A000FF2A03F01F0304F03F0405F01F0508D188
:1061B0004FF0000065F3040064F34A1063F3CF204E
:1061C000DDE765F3040064F34A1063F3CF20F0BC0D
:1061D000004B1847A16000002DE9F04F8DB0054637
:1061E00006939DF85C309DF858709DF860B005935B
:1061F000042B8A46144640F2A580002F00F0A280AE
:10620000A44B9847A44B06469847A44BD0F8089057
:106210008046524629460AA89847002800F09280F6
:10622000BDF82810B8F81000BDF82C20B8F812C03E
:10623000BDF82A500B1A101AADF82C00BDF82E002C
:10624000A5EB0C05A0EB0C0C0698ADF82EC01BB20C
:106250002DB20793ADF82830ADF82A50002840D170
:10626000706900285BD1BBF1000F40F01D82894BA3
:106270009847B8F81460B8F81030BDF92820BDF878
:106280002E100136F61ABDF82C3001339B1A1BB2C2
:106290000793BDF92A30013136B2C91A09B206FB9B
:1062A0000322012FA5B28246089109EB420840F073
:1062B0002F81059BFA2B40F2A480436A002B00F04B
:1062C0009C80774B0AA89847F02840F29680DAF82D
:1062D0002450ADF800400AAB324649465046A84724
:1062E00030E0307AC307BBD40698069B02F1010A5E
:1062F000AAEB010A0FFA8AFA0138C3F1010E0EEB7C
:10630000000CE245ACDD10F801CFBCF1800F4FF07E
:10631000FF3C98BF4FF0000C80F800C0EFE75D4BEA
:106320009847B8F81420B8F81030BDF92A50013257
:10633000D21A012F064612B221D1AA46BDF92E303B
:106340009A4502DD0DB0BDE8F08FBDF928700FFA57
:106350008AF8BDF92C309F4202DD0AF1010AEDE70F
:10636000059B0293ADF80440CDF800803BB27569FF
:10637000069249463046A8470137069AE9E7BDF834
:106380002C80BDF92830069908F10108C91AA8EB3C
:10639000030806910FFA88F8BDF92E309D42D1DC32
:1063A000BDF928A00FFA85FBBDF92C309A45069B54
:1063B00003DD434406930135EEE713F80A300599EF
:1063C000ADF8044013FB01F31B0A0293CDF800B0B3
:1063D0000FFA8AF37769079249463046B8470AF1BF
:1063E000010A079AE0E74046079A2946B847B044B1
:1063F0000134089BA342F6DCA4E72A4F7600002470
:10640000F7E7036A0BB3264B0AA89847F0281CD974
:10641000254B079A5A4513DCBDF92A50224F7600C6
:10642000BDF92E309D428DDC059B00934146DAF884
:106430002040079B3A465046A047B0440135EFE75D
:1064400023F8025B0BF1010BE3E74FF00007059A1D
:10645000164B204639469847C4F3C42BC4F3451A5B
:1064600004F01F040BFB02FB0AFB02FA5443730007
:10647000D24300F01F05C0F3451C0593C0F3C420B0
:106480004FF0000ED2B2089B73457FF75BAF4346D7
:10649000002635E0DD4F000025DA0000D1DE0000E7
:1064A000B5DE000051E3000008810020A16000007B
:1064B00019881FFA87F9894513D058781D78C008C4
:1064C000C1F3451C05F01F0500FB02B00CFB02AC3C
:1064D00005FB02450F46C0F30420CCF3052CC5F3A1
:1064E0000425197865F30401197019886CF34A11B1
:1064F0001980C1F3072160F3C701597001360233D7
:106500000799B142D4DC059B0EF1010E9844BAE71D
:10651000710009910599FA2910D839F812C0DFF8ED
:10652000989260465A46BDF92E108B423FF70AAF4B
:10653000069944464E1EC1F1010AA9E0079B9E4FF1
:10654000043B0593089B5B457FF7FCAEDDF818A084
:10655000C146002409E01AF8012B1AB1FF2A1FD105
:10656000A9F80050013409F10209079BA3425646DD
:1065700002DD1AF0030FEED108EB4409059BA3429C
:1065800015DA08EB4409013E079BA34253DC099B43
:106590009844DDE90632134406930BF1010BD1E771
:1065A000B9F800102846B847A9F80000DAE73368C0
:1065B0004BB101330CD1A9F80050A9F80250A9F849
:1065C0000450A9F806500436043409F10809D5E747
:1065D00032781AB1FF2A19D1A9F8005072781AB18D
:1065E000FF2A1AD1A9F80250B2781AB1FF2A1BD19A
:1065F000A9F80450F278002AE5D0FF2AE1D0B9F8D2
:1066000006102846B847A9F80600DCE7B9F80010DC
:106610002846B847A9F80000E0E7B9F80210284674
:10662000B847A9F80200DFE7B9F804102846B847D0
:10663000A9F80400DEE716F8012F1AB1FF2A05D1E8
:10664000A9F80050013409F102099DE7B9F80010DA
:106650002846B847A9F80000F4E716F8011FB1B1C1
:10666000594510D0FF29059A02D011FB02F2120AF7
:10667000218808932846C84796F800B0B4F800C0AF
:10668000089B80B202E021886145F1D1208002346C
:10669000079F0AEB06018F42DFDC099988440699BF
:1066A0003944069101333EE7BBF1010FB8F9100000
:1066B000B8F914600CD0BBF1020F2FD03F4B009300
:1066C0003F49404B404C4FF404720220A04739E64A
:1066D000DFF8F8B00136361A36B206FB05F0012FA6
:1066E00009EB400A4FEA460629D14FF00008059A07
:1066F000314B414620469847BDF92A70BDF92E30EE
:106700009F423FF71FAEBDF928500AEB4509BDF97E
:106710002C309D4205DDB2440137EFE7DFF8B0B021
:10672000D8E7B9F800101FFA88F38B4203D0059A16
:1067300020468846D84729F8020B0135E7E7C1F122
:1067400001089044DDE9063239F810100FFA88F894
:106750009F1A08464FF0000CBDF92E309D423FF7BE
:10676000F1ADBDF928900AEB4903BDF92C20914504
:1067700003DDB24447440135EEE717F80920BAB10A
:10678000624503D1B3F800E08E4510D0F92A94BFDA
:106790000599059A06939CBF12FB01F2120A19880B
:1067A0002046D847069B17F809C0198880B2188080
:1067B00009F101090233D8E7A16000001DFA0100C8
:1067C000E7F9010042FA010031E90000F160000040
:1067D000696100002DE9F04F8FB08B469DF864A0F1
:1067E0000593BAF1040F9DF860309DF86890089207
:1067F0000A9340F2D980002B00F0D6800A46B74BAE
:1068000001460CA89847002800F0CE80B44B98476A
:10681000B44B0646984704468368BDF832E0BDF89D
:1068200036100793638ABDF83050008ABDF83420D3
:10683000AEEB0308CB1AA5EB000CADF83630059B88
:106840000FFA8CFC0FFA88F8101AADF830C0ADF8CA
:106850003280ADF83400002B5CD17369002B72D10B
:10686000C5F1010515442AB2A68ABBF80470B4F933
:106870001030BBF90000B4F912400692BBF90220B7
:1068800001360137F61A3F1A141B36B23FB2A8EB95
:10689000040406FB08F57C43B9F1000F40F0F881D1
:1068A000CEF10102C31A0A4412B26544ACEB030CE8
:1068B000089B09926444079A03EB4404884B02EB5B
:1068C00045059847730007937B0008930A9B012BAB
:1068D000804640F0ED80036A002B00F0BA80824BC6
:1068E0000CA89847F02840F2B480BDF93270BDF989
:1068F00036309F4258DCCDF800A0069BD8F82060C7
:10690000224629464046B047079B1D44089B013755
:106910001C44ECE7337ADB079FD4059F0598531C92
:106920005B1BC7F101071BB201380697069F07449E
:10693000BB4292DD10F8017F802F4FF0FF3798BFE8
:1069400000270770F2E7664B9847BBF80450B4F98C
:1069500010C0A28ABBF900E0BBF90280B4F9124072
:10696000BDF93260BDF930100135A8EB0404A5EB88
:106970000E052DB2A6EB04080746ACEB0E040898F2
:1069800005FB084400EB44040A980132A2EB0C0218
:1069900001284FEA450012B2C1F10003069025D14B
:1069A000BDF936309E4202DD0FB0BDE8F08FBDF973
:1069B00030800FFA86F9BDF93430984503DD069B27
:1069C00001361C44ECE7CDF808A034F81830ADF8D7
:1069D0000430CDF800900FFA88F307997D6905928D
:1069E0003846A84708F10108059AE4E7BDF8348065
:1069F00008F10108A8EB0108059919440FFA88F875
:106A00008B46BDF936309E42CEDC33B2BDF93090B4
:106A10000593BDF93430994504DD069BC3441C44FD
:106A20000136EEE71BF809300799089213FB0AF3C9
:106A30001B0A029334F81930ADF80430059B00931B
:106A40007D690FFA89F33846A84709F10109089AC8
:106A5000DFE7BAF1FA0F27D9069BDFF890805F00D5
:106A60000026099BB3429FDD214628463A46C0478F
:106A7000079B1D44089B01361C44F2E735F81610AD
:106A800034F816005246C04725F816000136069B1A
:106A9000B342F3DC079B1D44089B01371C44099B50
:106AA000BB4281DD0026F2E7DFF844800027F6E7ED
:106AB000BAF1FA0F40F2EA80069BDFF83480043B1B
:106AC000CDE90A93DDE9093293427FF76DAFDDF836
:106AD00014A0A946A34600261AE000BFD1DE00009C
:106AE000DD4F000025DA0000B5DE000079EC000083
:106AF000A16000001AF8012B2AB1FF2A2AD1BBF8A5
:106B00000030A9F80030013609F102090BF1020B3F
:106B1000069BB342574602DD1AF0030FEAD105EB9C
:106B2000460904EB460A0B9BB3421BDC05EB460906
:106B300004EB460A013F069BB3426BDC079B1D44F6
:106B4000DDE9053213440593089B1C440A9B01337D
:106B50000A93B7E7B9F80010BBF80000C047A9F8DE
:106B60000000D0E73B688BB1013316D1BAF8003092
:106B7000A9F80030BAF80230A9F80230BAF80430A7
:106B8000A9F80430BAF80630A9F8063004370436FC
:106B900009F108090AF1080AC5E73A782AB1FF2A7B
:106BA00020D1BAF80030A9F800307A782AB1FF2A4B
:106BB00020D1BAF80230A9F80230BA782AB1FF2AF7
:106BC00020D1BAF80430A9F80430FA78002ADDD0D0
:106BD000FF2AD7D0B9F80610BAF80600C047A9F8BE
:106BE0000600D3E7B9F80010BAF80000C047A9F8CA
:106BF0000000DAE7B9F80210BAF80200C047A9F8B5
:106C00000200DAE7B9F80410BAF80400C047A9F89E
:106C10000400DAE717F8012F2AB1FF2A09D1BAF8E0
:106C20000030A9F80030013609F102090AF1020A20
:106C300081E7B9F80010BAF80000C047A9F80000D1
:106C4000F1E7059B9A5D6AB1F92A98BF1AFB02F237
:106C500035F8161034F8160094BF120A5246B84799
:106C600025F816000136069BB342EADC079B1D445B
:106C7000DDE9053213440593089B09F101091C4421
:106C8000099B4B457FF790AE0026ECE7384FF7E7BE
:106C9000B9F1010F0CD0B9F1020F2BD0354B009395
:106CA0003549364B364C40F253320220A0477BE642
:106CB000DFF8D0B0079A02EB4505089A02EB4404CE
:106CC0000A9A012A4FEA46064FEA470720D11B1AC3
:106CD00004EB4304BDF9363098453FF765AEBDF986
:106CE0003090BDF93430994507DD35443C4408F116
:106CF0000108EFE7DFF890B0DCE735F8191034F859
:106D000019005246D84725F8190009F10109E8E7AA
:106D1000059BA3EB0C030593A4EB4C04BDF93630A3
:106D200098453FF741AEBDF93090BDF934309945F3
:106D300008DDDDE905321344354405933C4408F190
:106D40000108EBE7059B13F809206AB1F92A98BFFF
:106D50001AFB02F235F8191034F8190094BF120A20
:106D60005246D84725F8190009F10109DDE700BFAF
:106D7000A16000001DFA0100E7F901004FFA0100CF
:106D800031E90000F16000006961000030B5A1B098
:106D9000044603920BA80C4A029190470B4A0299B1
:106DA0001288ADF82E2020460BAA094DA84704A84A
:106DB000084A9047002200922046039B0299064C05
:106DC00004AAA04721B030BDB59B0000E0FA010045
:106DD000019C00005578000085780000013900F121
:106DE000080311F8012F00F8012B9842F9D17047E0
:106DF0002DE9F04F2DED028BB9B01C469DF81031F6
:106E00000C939DF81431079382469D4B22A8894626
:106E1000154698479B4B98479B4B9847BDF8883041
:106E2000068A04909B1B408AADF88830BDF88E30EE
:106E3000BDF88A10BDF88C201B1A091A921BADF8F8
:106E40008E30924BADF88A10ADF88C2098470B909D
:106E5000F8B96388EBB92389B3F5807F19D10C9B0E
:106E6000BBB9079B002B40F09B80A37A002B40F01E
:106E70009980A27B02922278019201220092844C96
:106E80002A4651464846A04739B0BDEC028BBDE8C2
:106E9000F08F079B002B14BF032302230593049B51
:106EA000BAF80480B3F91210BAF90020B3F910301F
:106EB000BAF90270BDF98A00BDF9886008F10108CD
:106EC000A8EB02087F1AD21AC71BB21A0FFA88F869
:106ED00008FB0722059F02FB07520892BDF88C2091
:106EE000013213FA86F3961BB2B29BB2013AADF8A7
:106EF00090301344ADF89430BDF88E30013311FA60
:106F000080F1181A03B21793638809B236B211964A
:106F1000ADF89210ADF89610002B40F064822389F2
:106F2000B3F5807218BF012215920B9A002A40F027
:106F30005C82B3F5807F40F058820C9B002B40F0C0
:106F40005482A37A002B40F05082079B002B00F064
:106F50004C82504D22A8A847B0F5F07F24D822A833
:106F6000A84707464C4E7800B04708EE100A38464E
:106F7000B047059B119A13FB08FA22EAE2724FF020
:106F80000008064643460492179A42454EDD18EE25
:106F9000102A06EB030C02EB430E0021089A14E0C2
:106FA00003237BE7022379E74FF4F077DAE7907861
:106FB0000CF8010B30B192F801B0107800EB0B2007
:106FC0002EF8110005980131024411988842EEDC38
:106FD000049ABDF888101344089A52440892BDF8E8
:106FE0008C200132521A03FA82F2BA4207D2BDF85B
:106FF00096200132ADF8962008F10108C4E7A37B82
:107000000293237801930223009318EE102A33464B
:107010001F4D24A94846A847BDF8963001331BB23E
:10702000ADF89230ADF896300023E5E7BDF9963023
:10703000BDF992209A420FD0013BADF89630A37B68
:107040000293237801930223009318EE102A104C28
:10705000334624A94846A0473046104CA04718EEB6
:10706000100AA04710E74FF4F0730A93C7E1052216
:10707000DDE110931693199312E24FF0020B23E215
:10708000DD6D0000DD4F000025DA0000FD970000F7
:10709000D5670000B5DE0000FDEE0000B1EB00009A
:1070A000049BBDF98820B3F910301344BAF90020CD
:1070B0009B1A1C9307EB080308EE903A069318EE10
:1070C000103A03EB48031D93089B0D930023099A84
:1070D0000E931B9B13441BB21E93119B0E9A93425B
:1070E00043DC1F9B98440B9B33B30498BDF88A2064
:1070F000408ABDF88C30BDF888109D4D0244099837
:1071000002440498008A01335B1A01441BB218EE52
:10711000900A12B209B2A847002840F02481BDF8B5
:107120008C10BDF888300131C91A18EE900A914BC5
:1071300009B298474FF0020B089B1A9A1344089320
:10714000BDF88C30BDF8882001339B1A0A9A08FAE2
:1071500083F3934280F01681BDF896300133ADF889
:107160009630099B01330993C9E1159B002B00F070
:10717000D8800E9A1C9BBDF9A05013441BB21E9AD6
:107180005B1BBDF9A250551BBDF8A620B2F5807F50
:10719000DDE92F6019D1DDE931C101FB03F20CFB00
:1071A00015224D430CFB035306EBE21600EBE313F1
:1071B000BDF99C200F93B2EB262F4FEA262318939C
:1071C0001CDC069A00231370B2E0BDF8CE20BDF996
:1071D000A41053436A4311B91E441318E8E7DDE9CC
:1071E00031C103FB01F502FB1C5506EBE53602FB42
:1071F00001F503FB0C5500EBE533D9E73312002B07
:10720000DFDB0F9B0F991B121293BDF99E30B3EB7E
:10721000212FD6DD129B002BD3DB9DF8CC5015F02F
:107220000401139167D0301202FB030215F0020F24
:1072300026994FEA420351D111F812208DF8AC2063
:10724000C81842788DF8AD20022213929DF8CC2008
:10725000D20704D5BDF8AC20B2F5FC6FB1D09DF8D3
:10726000AB209AB10F9AADF8D2203693189A139B9F
:10727000ADF8D4208DF8DC30129A3F4BADF8D060D9
:1072800026A8ADF8D620984700289AD0069A9DF8EF
:10729000AE301370BDF8AC30A27AD2B11699149802
:1072A000149DC3F3451202FB0012109803F01F0156
:1072B000D20801FB0501C1F3042102F4FC620A4378
:1072C0001999DB0A03FB0513C3F3072342EAC3231F
:1072D0009BB21D9A0E9922F8113029E01344CA1866
:1072E000C95C8DF8AC1051788DF8AD1092788DF89E
:1072F000AE200322A9E7BDF96010BDF94820BDF812
:10730000A8301E4D2CA8CDE92012A8471C4BADF883
:10731000AC00DDE920122CA89847139B8DF8AE0035
:1073200094E7079B7BB10D9B069A9B7813706BB912
:107330000E9B059A01330E930D9B13440D93069BF0
:1073400001330693C9E6069AFF2313700D9B5A7802
:107350001B7803EB02230C9A9BB2002A9CD0B3F556
:10736000FC6F99D12DE7022808BF4FF0020BE3E62E
:107370006997000061F000002DC20000C5BD00004B
:10738000BDBE0000A37B029323786B4DCDE900B313
:1073900018EE102A3B4624A94846A847BDF8963067
:1073A00001331BB2ADF89230ADF89630079BA3B90C
:1073B0000C9B93B9638883B92389B3F5807F14BF8D
:1073C0004FF0020B4FF0010B0B9B4BB10A995B4B3B
:1073D000384698474FF00008C3E64FF0020BF3E73A
:1073E000DDF82C80BDE601231593554E22A8B04749
:1073F000B0F5F07F3FF637AE22A8B0470A900A9B5F
:10740000504E5800B04708EE100A0A98B0474E4B4D
:107410000746482126A89847159B63B3079B002B76
:107420007FF425AE0C9B002B0CBF04220622638840
:10743000ADF8A4302389ADF8A630BAF80630BAF812
:107440000210269501335B1AADF89E30A388ADF883
:10745000A030E388ADF8A230A389ADF8A830E37B73
:10746000ADF89C80C3F300038DF8AB3026A8374BF2
:107470008DF8AA209847A37ADA43D2B21492002B4F
:107480003FF4F7AD627BD2085A431992A289C2F346
:1074900045125A431692227B02F01F025343109367
:1074A000079B002B7FF4E9AD0C9B002B7FF4E5AD2F
:1074B0006388002B7FF4E1AD2389B3F5807F14BF8F
:1074C0004FF0020B4FF0010B0B9B1BB10A991B4BAA
:1074D00038469847049BBDF98A20B3F9123013440B
:1074E000BAF902209B1A1B93059B13FB08F31A930E
:1074F000002309939846119B23EAE3731F93179B7C
:10750000099A93423FF7CCADBDF99630BDF9922070
:107510009A420ED0013BADF89630A37B02932378BC
:10752000054CCDE900B318EE102A3B4624A9484685
:10753000A047384691E500BFD5670000BDF00000C8
:10754000B5DE0000FDEE000061F00000A9BF000004
:1075500010B5084B0446102198470023A381FF2350
:1075600023704FF480732381E37B43F00103E373C3
:1075700010BD00BF61F000000438C0B20A289DBFF2
:10758000024BC01880780020704700BFE0FA01006D
:10759000032805D0063804288CBF0020012070473E
:1075A000012070470E2809D8012303FA00F047F69E
:1075B000A473184214BF01200020704700207047B8
:1075C0002DE9F04F2DED028B04468DB088461F4605
:1075D00010464AB9794B0093794B4D2279497A4D3F
:1075E0000220A847794A14E01B78052B6AD9B9898B
:1075F000774B98470546002800F0BF8083698BB120
:10760000744B0093F722744B6E496F4E0220B047C3
:10761000AA69724B414620460DB0BDEC028BBDE815
:10762000F04F1847037B6E4ADFF8DCB103F01F030D
:1076300018469047039018466A4B98472B69049068
:10764000002B44D0684B08A8214698477B8838898E
:1076500013B9B0F5807F26D0E28861882688013290
:10766000521AA1880131891B3E1DCDE900061BB2CB
:1076700012B209B25D4E08A8B0472288BDF820308A
:10768000BDF822101344ADF8203063881944ADF8DA
:107690002210BDF824100A44ADF82420BDF826209D
:1076A0001344ADF8263008AA41460AA8D84748B185
:1076B000049B0193039B009320462A694C4C3B4654
:1076C0000AA9A0470DB0BDEC028BBDE8F08F2246A1
:1076D000414606A8D8470028F4D0BDF81C60BDF884
:1076E00018300136F61A36B2424B06EB4600984780
:1076F0003D4B06A9814608A898473F4B012108A8A1
:107700009847BDF91830B4F90020BDF91AA0B4F9B2
:107710000210CDF814B09B1A1BB2AAEB010108EEBF
:10772000103A0291BDF91E309A4503DD334B4846AD
:107730009847C7E7059B08AA41460AA8984700282A
:1077400038D0BDF90820DFF8C4B0CDF8009018EEAD
:10775000101A33462846D847012813D02846284B0C
:10776000194D9847274B009302201B4B15494FF4A6
:107770009A72A847214B48469847164B00935822C7
:107780000F4B2BE7049B0193039B0093DFF860B042
:107790003B464A460AA908A8D847BDF8223001331B
:1077A000ADF82230BDF826300133ADF82630029B0B
:1077B000013302930AF1010AB4E700BF8FFA010016
:1077C000EDFA01005BFA010031E90000A7FA0100BF
:1077D000EDC40000AFFA0100F9FA01008D6D000060
:1077E00091750000A5750000DD6D0000A5C00000CA
:1077F000F16D0000FDEE0000ABDE0000B1EB00001B
:1078000091D00000C0FA0100D1DE000071D000006C
:1078100050B10378A3F120025F2A07D913F0800F3B
:107820000CBF0020022070470320704701207047E2
:10783000A0F13003DBB2092B0AD9602884BF2038BD
:10784000C0B2A0F14103052B9ABF3738C3B2002361
:107850001846704710B5094B04461C219847FF2372
:107860002372074B63604FF6FF73E38123824FF46B
:10787000F81323600023A37510BD00BF61F0000062
:10788000100000202DE9F04F2DED048BD1B08A4679
:107890000A9300232193137A5E9C0590052B93464F
:1078A00040F2DB800A9B1B78002B00F0D6805368E7
:1078B0000A4608EE103A01469C4B31A8984700282A
:1078C00000F0CB809BF817309F0700F1CB80059B21
:1078D000059A9B88128801339B1A1BB218EE102A56
:1078E000B2F90870059ABBF91410B2F900200B9296
:1078F000059ABBF90A50B2F90260BBF91220259231
:10790000721890B212B23D440692002C00F0BC8076
:10791000002940F0BD80002E80F2B880A268921B42
:10792000002AB8BF5242C5F50071B2EB410FC4BF87
:107930004FF0FF3222602268002AC0F2A980049230
:107940006268024412B206921BB2049E0A98BBF906
:107950000C2009EE103A9BF817300093304419EED2
:10796000103A18EE101A724EB047049BC3180793D2
:10797000069ABAF902109BF817303A448A420A9ADA
:10798000C0F2898004995E0702EB010040F1AD80EE
:10799000079A0093511ABBF90C30664C18EE102A66
:1079A00089B2A047059B059A9B88128801339B1AD0
:1079B0001BB2181A0B9B00EBD07003EB600003B2F4
:1079C0000B939BF808302093BBF80E301193BBF853
:1079D00010301293DDE91132934288BFCDE91123B3
:1079E0009BF8183099071CD0534B35A89847BBF823
:1079F0000030ADF8D430DBF80430B3F908300A2297
:107A0000053393FBF2F3ADF8D6309BF808309BF8C2
:107A100019208DF8DC309DF8DD3062F301038DF81C
:107A2000DD30464B3BA89847BBF80230ADF8EE304E
:107A3000209B0B9CFA2B88BFFF230993ABB22293A8
:107A4000BDF818301E9300231D93049A0A9B13441B
:107A50001C930A9B9B5C002B60D151B0BDEC048B46
:107A6000BDE8F08F029347F618430193BBF90A3043
:107A70000093DBF80420BBF90C300A99304D3BA889
:107A8000A847BDF9EC3029E704945DE704915BE772
:107A90000022049258E70799009302EB010819EEBF
:107AA000103ABBF90C2018EE101A4046B047079B5D
:107AB0001844069B2B441BB2069374B113F5806FD8
:107AC0000BDB2368002B08DA079B2360059B069AD3
:107AD000B3F90230D21AC4E90123079B049398F842
:107AE0000030002BB9D0079042E71C077FF569AF43
:107AF000079A04990093511ABBF90C300D4C18EEFB
:107B0000102A89B2A047059B059A9B8812880133E9
:107B10009B1A1BB2181A0B9B184450E7259B1C4458
:107B200023B20C93002330930893BFE0D1DE000012
:107B3000250001007DFF0000FD850000B59B0000D1
:107B4000FD010100119A4FF6FF739A4224D0129A58
:107B50009A4221D0049AA14B0A981B681144984775
:107B600086B29F4C1C98236830A998471C9A2368BA
:107B7000054630980021104498479BF8173013F0C1
:107B80000103024600F02281232D0FD1089929B963
:107B9000BDF8C0201D92C7E70026E2E7089B012B35
:107BA00045D0022B40F012810023BDE7089B012B3A
:107BB00040F00C81202D79D1309B1D9A9B1A072B08
:107BC00032D11C9B1D999A1858589388ADF8E4300F
:107BD000844A3890C0F30745C0F30764C0F3072612
:107BE000C0B290470146F0B2904700EB0111E8B2F5
:107BF00090470546E0B2904700EB05149DF8E4007D
:107C0000904705469DF8E500904700EB0510C0F34E
:107C1000C400C4F3850440EA4414C1F3C40144EA37
:107C2000C123219302237FE7BBF80030F9E700234B
:107C3000BBF8004008936C4B18EE100A2946984791
:107C4000119A1F904FF6FF739A4220D0129A9A42CF
:107C50001DD0119BB3421AD8B24218D90C9BADF873
:107C6000E030069BADF8E230BBF80C300C9A013BDB
:107C700013440344ADF8E430229B069A013B1344BD
:107C8000ADF8E6303BAA594B514638A89847209B9F
:107C9000042B00F28A841F9B43B1BBF80C400C9B61
:107CA00023441C461F9B23441BB20C93079B049A3E
:107CB00030999B1A8B423FF645AF9BF818309D07D1
:107CC0001FD50B9BADF8CC30DBF80430BDF9D620C6
:107CD000B3F90830464C02EBD27203EBD371531068
:107CE0001E9A03EB610313441BB20C9AADF8CE301D
:107CF000ADF8E020ADF8E230524635AB38A933A8F4
:107D0000A0479BF81830DC071ED50B9BADF8CC3094
:107D1000BDF9D630DBF80420354C1189528903EBCC
:107D2000D3735B1001330B449B1A1E9A13441BB28E
:107D30000C9AADF8CE30ADF8E020ADF8E230524606
:107D400035AB38A933A8A0470A9B079A294C9E183F
:107D50009BF81730009318EE101A19EE103ABBF981
:107D60000C203046A047079BC518059BB3F900407F
:107D70009BF817300146580740F1018418EE102A8D
:107D800000933046BBF90C301B4EB047059B059A5B
:107D90009B88128801339B1A1BB2181A00EBD07013
:107DA00004EB600424B2229A069B13441BB2069390
:107DB0001E9B13449BB21E93079B069A0493BAF929
:107DC00006309342FFF649AE07953EE6BBF8004009
:107DD000219B0899022908BF1C462CE7640000205B
:107DE0005800002031780000B9D10000019C00004B
:107DF00019860000250001007DFF0000BDF8E42089
:107E0000BDF8E23052EA03013FF445AFBDF9E61098
:107E10000C9801440B440D91BAF900108B42FFF607
:107E20003AAFBAF904300D9999423FF734AF18EEE2
:107E3000103A18EE101AB3F90830B1F90A105B1AAB
:107E400006990B44BDF9E8109B1A5B1A1A44169365
:107E5000BAF902309A42FFF61EAFBAF90630169A06
:107E60009A423FF718AF18EE100AA94B29469847D7
:107E7000074628B9A74B009340F2B712A64BA9E3D7
:107E800018EE102A127BBDF93460BDF958809DF8B8
:107E9000EA30920700F0FE8104F01F022B92C4F337
:107EA00045122A92032BC4F3C422299200F0E180E8
:107EB000013B072B00F2D780DFE813F00800E00059
:107EC000D500DB00D500D500D500D0008023149369
:107ED000924B01241593BDF8E230179304FB03F194
:107EE000BAF90030179DBDF8E420B342C6BF9B1B12
:107EF00003EB430300231393BAF904300320B5FBCB
:107F0000F0F030449842C5BF9B1B0133179B03EB35
:107F100043031993BAF902304345CCBFA3EB0803DE
:107F200000230E93BAF9063002EB08009842C2BF54
:107F3000A3EB080301332493139B0E98D8BF24921C
:107F4000634300FB013307EBE30103F007030F93E7
:107F5000179B734F1A915343B3F5F07FA8BF4FF4AB
:107F6000F07318461893B847189B05465800B84751
:107F70006C4B08EE900A98476B4B9847B0F81490FA
:107F8000B0F910C0139B8768032209F1010993FB24
:107F9000F2F1B0F912300D98A9EB0C090FFA89F93A
:107FA000A8EB030309FB0363A3EB0C0C0E9B09FB7B
:107FB00003139C4407EB4C031093BDF8343011FAC3
:107FC00080F1013BADF8CC10199991FBF2F21A4403
:107FD000ADF8D020169B0E9A13441BB2ADF8CE30EC
:107FE000ADF8D230514B9847139A199B26909B1AA3
:107FF0002393179B1344199A9B1A6343239A27933D
:108000006FF0020392FBF3F399444FEA490328937C
:10801000C4F108034FF000082D930E9B249A93425D
:1080200031DBBDF9D230BDF9CE209A420FD0013BF1
:10803000ADF8D2301B9B0293099B0193022300935E
:1080400018EE902A3A4C2B4633A95046A0472846B2
:10805000384CA04718EE900AA0471CE6FF23149363
:108060000824354B36E7354B009340F27A22344BE7
:10807000B0E2F02314930424324B2BE7C023149373
:108080000224314B26E7149B0F9A23FA02FE139B1E
:108090000D9346460022199B0D998B425ADC269B74
:1080A000BBB1BDF8D030BDF9CC10BDF9D220274FFF
:1080B0000133A8445B1A1BB24046B84748B9BDF823
:1080C000D010BDF8CC300131C91A09B2204B40465E
:1080D0009847239B189AF3189A4240F3C480BDF83E
:1080E000D2300133ADF8D2300F9B279A13441A9A3D
:1080F00002EBE30203F007031A920F93109A289BF6
:108100001A440E9B109201330E93B04685E700BFD0
:10811000A9D1000065FB0100EAFC0100E8FC0100B8
:10812000FDEE0000DD4F000025DA0000FD970000A5
:10813000D5670000B1EB0000D4FB010092FB010009
:10814000F9FC0100D4FC0100E4FC01006997000087
:1081500061F000000F9BE31816931A9B16991B7889
:10816000C1F1080103EA0E03CB4013F0FF0306D070
:108170000999FF2961D1082C01D01599CB5C02F532
:10818000A07169440132032A01F8843C49D1109B53
:108190009DF8BC005B7829999DF8BE909DF8BD7054
:1081A000C0F1FF0210FB01FCDB0802FB03CC109BBB
:1081B0002B991B78C9F1FF0203F01F0319FB01F192
:1081C00002FB03110B0A1793109B1B88C3F3451383
:1081D0001A46C7F1FF032C932A9B114640EA090077
:1081E0002C9A384317FB03F302FB01331CBF4FF0FB
:1081F000FF32AA55179A08BFA8551B0A02F01F01A3
:1082000003F03F0318EE902A4FEA1C2C41EA431377
:1082100043EACC2322F81630109B02330136109328
:1082200000220F9B2D998B4215DA169B0F932EFA85
:1082300004FE0D9B01330D932DE7082C17BF1599F4
:108240000999CB5C09990BBF4B4313FB01F3C3F3B3
:1082500007231B0A93E71A9BDDF850E001331A93BA
:1082600000230F93E5E71B9B0293099B01930223D5
:10827000A84E009318EE902A2B4633A95046B047DB
:10828000BDF8D23001331BB2ADF8CE30ADF8D230EC
:10829000002629E7032B09EE904A00F0BA80013B43
:1082A000072B00F2B080DFE803F004BAAEB4AEAE44
:1082B000AEA780221392984A012502230E92099AB2
:1082C000F92A12D8954A099892F80011814240F093
:1082D000AC80D2F80421AA4240F0A7808F4B099AC3
:1082E00083F80021C3F804510E93BAF90030BDF8A9
:1082F000E290BDF8E420B342CCBF9B1B00230F9358
:10830000BAF9043009EB06009842C4BF9B1B013345
:10831000BAF90260C8BF1093BAF90630D8BFCDF8D9
:10832000409002EB08004645CCBFA6EB08060026AD
:108330009842C2BFA3EB0803013317930F9BD8BF2A
:10834000179205FB09F103FB05F406FB014407EB5B
:10835000D403149302FB09F3B3F5F07FA8BF4FF4E5
:10836000F073159318466E4B98470D9A0F99BDF808
:10837000343011FA82F2ADF8CC20109A013B13444C
:10838000ADF8D030169B33441BB2ADF8CE30ADF80B
:10839000D230644B08EE900A9847C5F108030D935C
:1083A0000F9B19909944109BA9EB030905FB09F356
:1083B00004F007041A934FF00009179B9E4245DB17
:1083C000BDF9D230BDF9CE209A4210D0013BADF8B4
:1083D000D2301B9B0293FF260223CDE9003619EE13
:1083E000902A18EE903A504C33A95046A04718EE08
:1083F000900A4E4B98474EE4FF22139208254C4AB0
:108400004FF480735AE74B4B009340F2E5124A4B0E
:10841000E0E0F02213920425484A10234EE7C022E0
:1084200013920225464A042348E70E993B480B4421
:1084300011F8012BFF2A17BF099C099A12FB04F2BD
:10844000120A994200F8012BF2D147E7139B0F98CB
:10845000CDF88C9023FA04F118EE903A03EB09085A
:108460004246109B834239DC0F9A10999B1A16934F
:108470008A42C8BF002318939944199BB3B1BDF831
:10848000D030BDF9CC10BDF9D2202E4F01335B1A8C
:108490001BB24046B84748B9BDF8D010BDF8CC3043
:1084A0000131C91A09B2284B40469847189B169AC1
:1084B00013449846239B9844159B434546D9BDF8E1
:1084C000D2300133ADF8D2301A9B1C44149B03EB1D
:1084D000D403149304F0070401366EE7149B0D9F38
:1084E0001B78A7EB040C0B4023FA0CF313F0FF03EB
:1084F0001CBF0E9FFB5C13700D9BA3429DBF149B82
:108500001399013364198EBFE9401493002401309C
:108510000132A6E7D5670000E8FC0100C88400200E
:10852000FDEE0000FD970000D9610000B1EB0000F6
:10853000D4FB0100B8FB01000BFD0100D4FC0100DD
:10854000E4FC01006997000061F000001B9B0293AE
:10855000FF270223CDE9003719EE902A18EE903A52
:108560001F4F33A95046B847BDF8D23001331BB274
:10857000ADF8CE30ADF8D2304FF00009A4E71A07BD
:108580007FF511AC18EE102A00933046BBF90C3081
:10859000144EB047059B059A9B88128801339B1A9D
:1085A0001BB2181A0444FFF7FDBB9BF819301B934C
:1085B00018EE100A0C4E00232A4638A9B0470028AE
:1085C0007FF41CAC1F2D7FF666AB084B0093084B65
:1085D00040F2A1120749084C0220A047FFF75BBBFD
:1085E000D96100007DFF0000ADD1000040FB01001B
:1085F000EAFC01000AFB010031E9000010B5054B5F
:1086000004460A219847FF23237200232380012375
:10861000638010BD61F000002DE9F04F2DED048B5B
:108620009B46B3F90230C7B0CDE9050108EE902AA8
:10863000002B00F0E3809BF80820052A40F2DE8042
:10864000059AB0F90040B1F90000B2F90210069A9B
:108650008442B2F9022002D1914200F0CF8003EBB4
:10866000D373C3F34F038442D4BFC3EB0405C3EBFE
:108670000005ADF828508442ACBF1D191D18914269
:10868000D4BFC3EB0100C3EB02009142ACBF5B1847
:108690009B180AA9ADF82A0018EE902AA94CADF84B
:1086A0002C500846ADF82E30A047002800F0A680D8
:1086B000059BB3F90290069BB3F90280C14540F0D7
:1086C0005781A14B9BF808409847A04B9847BBF9AE
:1086D0000260BBF90650731E03F0010680465F106E
:1086E00006EB630625B1BBF90450003D18BF012518
:1086F000974B9847002840F0868085F00102069B42
:108700000599B3F90030B1F900108B421846A8BFA3
:1087100008468B42B8BF0B46013BADF89C30059B29
:10872000ADF898005B889E1B3B44ADF89A60ADF8AD
:108730009E30002A69D09BF8093003F00303CDE98D
:10874000014301230093BBF80020824C002326A99B
:108750000AA8A0479BF8093013F00C0F4ED07E4BAF
:1087600031A89847BBF80030ADF8C63047F6FF7324
:10877000ADF8C4309BF808308DF8D030BBF902302A
:108780005C10DB4303F001059BF809305A0718D54C
:10879000059B1A88A3B2D11AADF89810059949889B
:1087A0001A44C81A0B44521B5B1BADF89A00ADF873
:1087B0009C20ADF89E3018EE901A684B31AA26A87E
:1087C00098479BF809301B0718D5069B1A88A3B257
:1087D000D11AADF89810069949881A44C81A0B4462
:1087E000521B5B1BADF89A00ADF89C20ADF89E3093
:1087F00018EE901A594B31AA26A8984747B0BDECFD
:10880000048BBDE8F08F002279E726AA4D4B0AA918
:108810001046984700289DD0B8F81240BDF99A003C
:10882000B8F81010B8F91060BDF89870BDF99CC088
:10883000BDF998E0ADF8C4E0031BADF89A30BDF87F
:108840009C30ADF8C8C07A1A591AADF89C10BDF822
:108850009E10ADF8C600091B5C1C12B2E41BADF8FB
:108860009820ADF89E1024B2ADF8CA00DDB11644D0
:10887000BBF90430BBF906201A4496FBF2F302FB65
:10888000136633B20793364BDFF8C8A020469847EB
:10889000BDF99A900746BDF99E30994505DD3846E9
:1088A000304B984756E70795EDE72F4B2F4E214663
:1088B00038469847BDF89830B8F81220B8F810102C
:1088C0004A44194412B2234609B23846B047024618
:1088D00095B188B10023079918460AE0BBF9042036
:1088E0008A4225DB13445B1A1BB2013301321BB2EF
:1088F00011B29C42F2DC02229BF8093003F0030320
:1089000002939BF8083031A9CDE900230AA83B4621
:10891000BBF80020D047BDF8C6300133ADF8C630F3
:10892000BDF8CA300133ADF8CA3009F10109B2E728
:10893000BBF906C062449142BABFF8540A4600220D
:10894000D3E700BFD1DE0000DD4F000025DA0000D4
:10895000FD970000D9610000B59B0000019C00005C
:10896000FDEE0000B1EB0000BDF0000069970000D3
:10897000059BB3F90070069BB3F90060B74240F065
:10898000DB80664B9BF808609847654B9847BBF9BE
:108990000280BBF9065008F1FF3303F001080746D7
:1089A0004FEA630908EB630825B1BBF90450003DA9
:1089B00018BF01255B4B984720BB85F00102059B42
:1089C00005991B88B1F90210A3EB08084B44ADF8D8
:1089D0009C30069BADF89880B3F902308B42184664
:1089E000A8BF08468B42B8BF0B46013BADF89A00C2
:1089F000ADF89E3042B19BF8093003F00303CDE996
:108A000001639EE60022DAE726AA0AA91046A047DB
:108A100000283FF49FAE3A8ABDF898C07E8ABDF91F
:108A20009A10BDF99840BDF99C00ADF8C800ACEBB8
:108A30000203ADF898308B1BADF89A30BDF89C302E
:108A4000ADF8C4409A1AADF89C20BDF89E20ADF850
:108A5000C610921B5E1CA6EB0C0633B2184608EE3D
:108A6000103AADF89E20304BADF8CA1098478046BA
:108A7000C5B1BDF99830B7F91040BBF904201C44CA
:108A8000BBF90630134494FBF3F203FB124424B207
:108A9000BDF99A90DFF89CA0BDF99E30994503DDA1
:108AA0004046FDE62C46F3E718EE101A1F4B204E09
:108AB00040469847BDF898307A8A398A4A44194422
:108AC00012B218EE103A09B24046B0476DB150B13B
:108AD000BBF90420BBF906301344A242B8BF002002
:108AE0009C42A8BF0024013424B2002302939BF8C7
:108AF0000830BBF80020CDE9000331A943460AA89D
:108B0000D047BDF8C6300133ADF8C630BDF8CA3025
:108B10000133ADF8CA3009F10109BDE7DD4F0000AE
:108B200025DA0000FD970000FDEE0000BDF000001A
:108B300069970000D9610000C14505DB4B46C1467D
:108B400098463B4637461E46F31B0993A8EB09039C
:108B50000893F31B83EAE372A2EBE372089B07928C
:108B600083EAE37AAAEBE37A52451346D8BF079B20
:108B7000BBF90250CABF4FEA4A135B01B3FBF2F3E1
:108B8000B34AD8BFB3FBFAF3D15C3F2315FB0135E1
:108B9000C5F3CF13BE42D4BFC3EB0602C3EB07023B
:108BA000ADF83020BE42ACBF9A19DA19ADF83420C6
:108BB0000CA9C845D4BFC3EB0802C3EB0902C845E2
:108BC000ACBF43444B44ADF83220ADF836300AAA6E
:108BD000A04B0846EC11984700283FF4BBAD079B1B
:108BE00004F0010404EB25245345A4B2C5F30F257A
:108BF00040F3ED8014FA89F31BB208EE103AF31B30
:108C0000A9EB050A14FA88F4A8EB0505002B4FF030
:108C1000000324B20FFA8AFA2DB2019340F3C68002
:108C2000009533465246394610A88B4DA84701237C
:108C3000CDE9004318EE102A334639461BA8A84751
:108C4000DFF840A2002110A8D047002109EE100A49
:108C50001BA8D0479BF8095015F0100509EE900AA3
:108C600040F0CF800322BDF820400192F21BBDF8F6
:108C70002430079319FA82F23B1B12B23946009254
:108C8000754F1BB24A4626A8B84702220192079A9E
:108C9000424412B2331B1BB200923146424631A805
:108CA000B847294626A8D0472946099031A8D04779
:108CB00082466A4B6A4E98476A4B9847BDF8301017
:108CC000028A8B1AADF830300546BDF83230408A42
:108CD0001B1AADF83230BDF834309A1AADF8342092
:108CE0005C1CBDF83620641A121A23B20CA8ADF829
:108CF00036200793B047B0F5F07F80F087800CA84E
:108D0000B0470746584B384698472B8ABDF8302065
:108D10001A4412B20892ADF83820BDF8342013443A
:108D2000ADF83C306A8ABDF8323013441BB2ADF85E
:108D30003A30ADF83E3039464C4B06469847BDF9BF
:108D40003280B5F912304FF000099844BDF9363041
:108D5000B5F91220134498455BDDBDF93E30BDF9ED
:108D60003A209A4213D0013BADF83E309BF80930CF
:108D7000BBF800203E4C03F0030302939BF808303D
:108D80000193022300930AA933460EA8A047394B4A
:108D9000394C3046984719EE100AA04719EE900A50
:108DA000A0470998A0475046A047D3E418EE102AE0
:108DB000009433463946284C10A8A0470123CDE93A
:108DC00000535246334639461BA8A04738E714FAE9
:108DD00086F3002214FA87F421B2CDE900821BB297
:108DE0004A461D4C10A8A0471FFA86FABAB2511B7A
:108DF000AAEB05030122CDE900821BB24A4609B263
:108E0000E2E74FF0FF3ACDF824A052E74FF4F077B5
:108E100078E706EB090308EE103A0899079B174C10
:108E200018EE100A0FFA88F2A04720B90799144BE0
:108E300018EE100A9847079B99444B449F4223D948
:108E4000BDF83E300133ADF83E3008F101087DE752
:108E500026FD0100D1DE000019980000DD4F000062
:108E6000B5DE000025DA0000FDEE0000BDF00000D8
:108E7000D9610000B1EB0000AD97000069970000D8
:108E800061F00000199700009BF80930BBF8002042
:108E90000D4C03F0030302939BF808300193022367
:108EA00000930AA933460EA8A047BDF83E3001330F
:108EB0001BB2ADF83A30ADF83E303946034B304680
:108EC00098474FF00009C0E7D9610000BDF00000ED
:108ED000F9290AD8052907D910FB01F048F28101C8
:108EE0004843C0F3C7507047002070472DE9F8434E
:108EF000089D6E8A95F82870891B0446A88A0EB2D0
:108F0000296A121A12B207F0010099BB2D7C05F0F4
:108F1000020780B13FB105F00305022D05D10132F2
:108F2000ACBF00200120BDE8F883032D01D1002A49
:108F3000F9DC0020F7E7002F40F06C8105F003001A
:108F400001280AD1002EEEDCDE42F2D4002E00F31E
:108F5000638171428B42ECDD98E00028F4D1F11876
:108F600000F15881002EE4DC70429842C0F29980F2
:108F70000220D8E707F0020C002800F09680EF6985
:108F800006FB07F1002F4FEAA1215FFA8CF005DD07
:108F90008A4205DA003818BF0120C4E78A42F9DCAA
:108FA000F1187943002F4FEAA12105DD8A4206DD41
:108FB000B0FA80F04009B6E78A42F9DB0132A969CC
:108FC00012024A4392124FEA222C12F0FF021FBFF4
:108FD000696AC2F1FF074F433F1214BFC7F1FF0791
:108FE000FF27ACEB0606002A52D0002E0FDBB3425F
:108FF0000DDDC2F1FF02C7F1FF015143C1F347216B
:1090000008B9C943C9B2A05D944A9047A055721CE3
:10901000DFF84882696A95F828008F4200F0020064
:1090200016DC934227DD002A25DBA96979438912E2
:109030007943EF69C1F34721002FBCBFC943C9B2CF
:1090400008B1C943C9B2A05C844FB847A05412E02C
:10905000002A0ADB934208DDA7EB6101C9B208B11F
:10906000C943C9B2A05CC047A054696A01329342A7
:10907000A7EB0107CEDC95F8281089070AD5B34283
:10908000FFF657AF002EFFF673AF3146204609E0DA
:109090003246BDE7501C3FF54CAF8342FFF668AF48
:1090A000191A20446E4B984762E7A96901FB02F741
:1090B00000294FEAA727CCBF07F1010EBE4676452F
:1090C0005FFA8CF03FF766AF06EB030C67453FF79E
:1090D0006FAF4FEA022E013212024A4301FB0EFE2D
:1090E0004FEAA248B8EBAE4FCEF3872CC6EBAE47A3
:1090F00000F09780002953DA07F1FF39BCF1000F27
:1091000000F08C80EE6976420CFB06F6002F4FEAE9
:10911000A6260CDBBB420ADD06FB0CF1C1F347219E
:1091200008B1C943C9B2E05D4C4A9047E055B9F176
:10913000000F17DB4B4515DDAA6914F80900C6F1CD
:10914000FF065142714395F8282089127143C1F3FB
:109150004721960758BFC943404A58BFC9B29047F4
:1091600004F8090095F82820950714D54B45FFF61B
:10917000FFAEB9F1000F7FF7FBAE494686E7013736
:109180009F42A8BF1F46002F3FF4D3AE7FF7F0AE3B
:10919000D91BE01986E7781C83423BDB00287DE77A
:1091A000EA69CCF1FF014A43002F4FEAA2220BDB10
:1091B000BB4209DD5143C1F3472108B9C943C9B2D4
:1091C000E05D264EB047E0557E1C15D4B34213DD5A
:1091D000C2F1FF00AA6902FB00F1891295F828206C
:1091E0004143C1F34721900748BFC943A05D1B4AD3
:1091F00048BFC9B29047A05595F82820920707D5D7
:10920000BB42FFF696AE002FFFF6B2AE39463DE701
:109210000237B5E7012086E6002B9CE64F464FF06B
:10922000FF0C002F0DDBBB420BDDC2F38721614435
:10923000C1F3470108B1C943C9B2E05D074A90478D
:10924000E05595F82820920799D5A8EB06018B42A6
:109250007FF76FAE0029FFF68BAE17E7D18E0000C7
:1092600061F00000013900F1080311F8012F00F846
:10927000012B9842F9D170472DE9F04F8BB006468B
:10928000DDF8508098F81290B8F910A08B461D4672
:1092900008F10801924B08A809F001091746984700
:1092A000BDF92220B9F1000F3AD1BA4201DD002008
:1092B00039E0BDF92630BB42F9DBBDF9201001EBE6
:1092C0000A039B45A1EB0B0407DBBDF9243005EB3A
:1092D0000B00A3EB0A03984209DD02EB0A039F424D
:1092E000BDF926003EDBA0EB0A039F423ADCB9F150
:1092F000000F25D1A542DADB002C03DB794B214698
:1093000030469847BDF92400A0EB0B01481C00280B
:10931000CDDDA8420FDA291A3044724B98470DE090
:10932000BA4203DD01200BB0BDE8F08FBDF9263055
:10933000BB42C2DAF6E70CB9A842F3D00220F2E74A
:1093400024EAE474AC42F9DCBDF92410A1EB0B0172
:10935000091B01316318AB42C8BF291B0029EDDB93
:109360003019DAE7BDF8243001335B1A1BB292B230
:109370000293BF1AB8F9103001303FB2801A5B4334
:10938000BA4500B2019300F3AA81A0EB0A039F4201
:10939000D4DBC01BD8F81430BAF5807FAAEB0000EC
:1093A000D4BF4FF400624FF40042984200F101072D
:1093B00070D0019B039200FB103005A94A4B9847DF
:1093C000039A6FE0B8F81A30ADF81230B8F81830D8
:1093D000ADF81030019B039207F1FF3B0BFB1B30F4
:1093E00005A9414B9847BDF81630A8F81A30BDF8CA
:1093F0001430C8F814B0BDF81410A8F81830BDF82F
:109400001030039A01398B4207D1BDF8161021B9EB
:10941000FF21ADF81430ADF81610BDF814109942C4
:1094200066D1BDF81220BDF816100A44C2F34702F7
:10943000B9F1000F01D0D243D2B2AAEB0303013B32
:10944000E71807D4AF4205DAF05DDFF8A0801146D7
:10945000C047F0550299CB1A581E041906D4AC42E5
:1094600004DA305D214B114698473055B9F1000FB1
:1094700028D1AF423FF71BAF002F03DB194B394612
:109480003046984701343FF512AFAC423FF756AF34
:10949000291B65E7B8F81A30ADF81630B8F818305F
:1094A000ADF81430019B039207FB173004A90E4B53
:1094B0009847BDF81230A8F81A30C8F81470BDF8F3
:1094C000103098E7781C20EAE070AC42D4BF211A33
:1094D000291AA842BFF632AF0029FFF62FAF1BE7CB
:1094E0006592000061F00000DDE90000D18E00000F
:1094F0000133AAEB030A029B04EB0A08A3EB0A0A56
:109500000AF1FF3A5444B9F1000F10D008F10100FC
:1095100020EAE070A542ACBF211A291AA84206DA57
:10952000002904DB794B029230449847029ABDF837
:1095300010B0019B029206A90BFB1B30744B98479D
:10954000BDF81A10724B029A0BF1010A39B9BDF835
:1095500018100139ADF81810FF21ADF81A10BDF838
:109560001810B94230DB019807A90AFB1A00984786
:10957000BDF81E20BDF81230C2F1FF01C3F1FF0398
:109580004B43C3F34723B9F1000F01D1DB43DBB2F7
:10959000B8F1000F08DB454506DD16F808005D4F01
:1095A0001946B84706F80800002C06DBA54204DD82
:1095B000305D1946574B9847305508F1FF38013454
:1095C000ADF81A200BF1020ABDF81430BDF818B03E
:1095D0000293BDF81A10BDF81C20BDF81E304FEAEA
:1095E0000B1B0020029F574540D228B1ADF81A103E
:1095F000ADF81C20ADF81E30BDF81A1009B3BDF847
:1096000016304B43C3F34723B9F1000F01D0DB43BE
:10961000DBB2B8F1000F08DB454506DD16F808009F
:109620003C4A1946904706F80800002C06DBA54284
:1096300004DD305D1946374B9847305508F1FF3847
:109640000134B9F1000F7FF479AE08F101018D42C8
:10965000FFF62DAE002902DB2C4B30469847002C3C
:10966000FFF625AEA5427FF769AE11E7C1F30F13F0
:1096700003EB0B02019B02FB02F00AFB1A33C0EB67
:109680000323500093FBF0F31344C3F30F121B01A9
:1096900003F0F0031944C1F34701B9F1000F01D001
:1096A000C943C9B2B8F1000F09DB454507DD16F81B
:1096B0000800184F0391B847039906F80800002CDA
:1096C00005DBA54203DD305D124FB847305508F188
:1096D000FF3801340AF1010A1946012082E7D8F85F
:1096E0001430BAF5807FAAEB0707D4BF4FF40062AD
:1096F0004FF40042BB423FF465AE019B039207FB6F
:10970000173004A9024B9847039A63E661F0000002
:10971000DDE90000D18E000073B50E4C002354F833
:109720003360DAB204EBC30576B10133102BF6D106
:10973000094B00930220094B09490A4C5722A047C4
:109740004FF0FF3002B070BD44F83300696010B2D2
:10975000F8E700BFF48600207CFD0100A2FD0100B7
:1097600047FD010031E900002DE9F3470E4E0746A1
:10977000884691469A460025346834B9002D14BFB6
:109780000220012002B0BDE8F0870094246853460F
:109790004A4641463846A0470028F3D0022808BF71
:1097A00001250836E8E700BFF4860020431C18BFF7
:1097B000074B4FF000021DBF53F8301043F8302024
:1097C00003EBC003114618BF5A600846704700BF3C
:1097D000F48600200022084B30B5114614465D681F
:1097E0000132854204BF1968C3E90044102A03F11D
:1097F0000803F4D1084630BDF48600200023054A52
:10980000184652F8331009B10130C0B20133102BA1
:10981000F7D17047F48600202DE9F041BDF918809A
:1098200015460E461F462C213C4B0446984745459D
:1098300005DD2B464546984633463E461F46237C6B
:109840009DF81C20658162F301032374A8EB0502D7
:10985000BB1B83EAE37082EAE271A0EBE370A1EB49
:10986000E271884294F82810A582D4BF002001201C
:1098700060F300012A4D84F828100020C907C4E9CC
:1098800006002681A781A4F80E80668225602071DB
:1098900024D533B14FF4801191FBF3F15143891278
:1098A000E16132B14FF4801191FBF2F253439B120C
:1098B000A361E369227C236212F00302216A94F817
:1098C00028301DD16FF3410384F8283000294FEA76
:1098D000A103B8BF5B426362BDE8F08132B14FF4CF
:1098E000801191FBF2F159438912A16133B14FF418
:1098F000801191FBF3F35A439212E261A369D9E715
:10990000012A02D143F00203DEE7022A02D1002934
:10991000F8DCD7E70029D5DCF4E700BF61F00000F0
:10992000ED8E0000F8B50446C8888D881F464B8828
:109930000130C01A0B880135ED1A00B22DB2A842D1
:10994000A8BF2846B2EB600F4FEA6003164604F149
:109950000800C8BF1EB2084B9847A37C268267F355
:109960000003A374054B2360022323714FF00042D0
:109970000023C4E90523F8BD659200007992000038
:10998000B0F9083070B503FB01F4B2EB242F4FEAB5
:10999000242501DC408870BDB0F90A4001FB04F6C3
:1099A000B2EB262F01DB8088F5E7E41A521B01FB9E
:1099B00004F312B2C2EB02221B1292FBF3F3828871
:1099C000C2F345144288DBB2C3F1FF05C2F345126E
:1099D0006A4348F2810103FB04224A43C2F3C5549F
:1099E000027902F01F06827802F01F026A4303FB2D
:1099F00006224A43C2F3C45242EA44124479C07870
:109A0000C008E408684303FB04004843C00D42EA71
:109A1000C020C0E72DE9F04FCB074FEA610A4FEABB
:109A2000400587B058BF0AF1FF385A4B0446284614
:109A30000E46174654BF0FFA88F8D0469847AB1E1B
:109A400001934FEA4A0302936FF0010308FB0333CB
:109A50000146B9464FF0000B03935C4525DC3B887B
:109A600093FBF6F304FB04F93B803A463B464FF088
:109A7000010CE14544D804FB0AF36FF001004343B5
:109A80000493631E05FB0373029308F10103019322
:109A900008FB055303934FF0000C64453EDC3E4B3E
:109AA000084607B0BDE8F04F1847019B029839F807
:109AB000032000EB090C03987243631E484421F80D
:109AC000132003EB0A0E7445CCBF3CF813E04FF0B3
:109AD000000EA2EB0E0EA3EB0802002AD4BFB9F8C9
:109AE000002030F81320013B7244E8D248462B4B4B
:109AF00004912A469847A94404990BF1010BACE75D
:109B0000588833F802EB70451CBF90FBF6F01FFA43
:109B100080FEA3F800E00CF1010CAAE7049813887A
:109B200000EB020903980027104405909646734302
:109B300090463846002BACBFC3F38F1B4FF0000B91
:109B400021F810B0A0EB0A0BBBF1000FD4BFB8F89E
:109B500000B039F807B0A3EB0B0B019B03449C4208
:109B6000CBBF059B029BDB5B33F81C30013084428A
:109B70005B44A8442F44DDDC002331F81300AEF829
:109B8000000001339C42AE44F7DC0CF1010C0232C0
:109B900083E700BFFDEE0000B1EB000079EC0000B0
:109BA000013900F1080311F8012F00F8012B984248
:109BB000F9D1704710B50F4B5421044698470E4B0E
:109BC0001B8863800022FF23A280E281A4F8462044
:109BD000E2836381237323772375A28684F836306A
:109BE000064A84F8443084F828300F232263226424
:109BF000638210BD61F0000034FE010010000020FF
:109C00002DE9F04F2DED048BADB003460490C088D4
:109C10005D88431C5B1B1BB2002B8846914641F3B9
:109C20008181049B9A881988531C5B1A1BB2002BF4
:109C300041F37881B9F92040002C00F0518599F862
:109C400028300793052B40F24B85D9F82070B9F9DD
:109C50002460B9F92630012F03D116B9002B40F347
:109C60003F85B9F822709BB2A7EB030CB6B21F4434
:109C70003A44F71A3344034498B204EBD4736FEABE
:109C800063065B1092B20133ADF8442012FA83F2FE
:109C900010FA83F3ADF84E30079BADF84C206144C9
:109CA0003D44FB2B89B2ADB228BFFF23ADF8401075
:109CB000ADF8425011FA86F115FA86F5ADF8481064
:109CC000ADF84A500793ADF846007B4B98477B4B65
:109CD00098477B4B0546424612A914A8984700288E
:109CE00000F0FE842E8ABDF85030688ABDF852100C
:109CF000BDF85420734D9B1BADF85030BDF8563065
:109D0000921B091A1B1AADF85210ADF85420049991
:109D1000ADF8563016A86C4B9847BDF85A10BDF8F0
:109D200058B0BDF85C30BDF84470013188B20BF119
:109D3000010BBDF85E10ADF85A005A1E1FFA8BFBDE
:109D4000ADF858B0ADF85C20A3EB0B0B4A1E091A16
:109D50000BB20FFA8BFB9B45A8BF9B46ADF85E206C
:109D6000B9F90020BDF840304FEA6B0B934507F17D
:109D700001075946A7EB0307A8BF1146BDF84630B7
:109D800008EE901ABDF8421001335B1A1BB23FB2C5
:109D90009F42A8BF1F467F109742A8BF174604EBFB
:109DA000070A0AFB0AF04000A847B9F92040464BD1
:109DB000059010A91EA8984704F0010204EBD47383
:109DC000BDF844100992C3F34F0364F00102BDF8DB
:109DD00040001A443A44C943014492B2ADF87C2091
:109DE0000A44ADF87820BDF84620BDF84210013392
:109DF0000132521A9BB2ADF87A3013443E193A46FA
:109E0000ADF87E30314F00231EA925A8B847012C9C
:109E1000304618BF6410A84773000893059B06934B
:109E200033B208EE103A07464FF0000B5E4509DCEE
:109E3000274B38469847012C06FB06F540F09D81DC
:109E4000002352E0234B31463846984725AB009318
:109E5000259D18EE103A0FFA8BF200213846A847DC
:109E600050B9089906981C4B9847069A089B1A44C3
:109E700006920BF1010BD9E73A78069B06989201FE
:109E800092FBF4F223F8022B089A394610189842F4
:109E9000EBD08C4611F8012F9CF800C094450CBF04
:109EA00033F8022C920103F1020318BF92FBF4F283
:109EB00023F8022CEBE700BFDD4F000025DA00009D
:109EC000D1DE0000FDEE0000A19B000025990000FE
:109ED000B1EB0000BDF0000061F00000059A0599AB
:109EE00032F813209209CA540133AB42F6D1BDF8BF
:109EF0004E30BDF84A2001339B1AC3F3C03101FA3A
:109F000083F302EB63039AB21BB20893BDF84C30A3
:109F10000A92BDF8482001339B1AC3F3C03101FAFD
:109F200083F302EB63039AB21BB20993AD4B0B921E
:109F30009847002840F04F81B9F92250002D40F099
:109F40004C81B9F92430002B40F04981B9F92650F1
:109F5000B5FA85F35B090693BDF84C00BDF84830AF
:109F6000A14D0130C01A00B2A04B984718EE902ABC
:109F7000012316A908EE100A25A8A8479C4B00212A
:109F800025A89847BDF94C30ADF864301FFA8AFB1C
:109F90000133A3EB0B03ADF86030BDF94A30ADF8E7
:109FA0006230013B5B4408EE900AADF866304246F1
:109FB000904B18A91AA89847002838D0BDF96E30E0
:109FC000089ABDF86C609342C4BF1346ADF86E307A
:109FD000099ABDF968309342DEBF0B9B0133ADF89F
:109FE0006830BDF968500136761B36B2002E1EDD92
:109FF000BDF86E30BDF96A2001339B1A1BB20C9379
:10A00000BDF96230D21ABDF96030ED1A059B0AFB2A
:10A0100002551D441AA9784B1EA89847BDF87A30FE
:10A02000ADF87E3000270C9B9F42C0F2E980BDF95D
:10A030004C30BDF94E20ADF864300133A3EB0B0377
:10A04000ADF86030531CA3EB0B03ADF86230ADF8F4
:10A050006620684B424618A91AA8984700283AD0AB
:10A06000BDF96A30089ABDF86C609342D8BF0A9B6C
:10A07000099ADCBF0133ADF86A30BDF9683093420C
:10A08000DEBF0B9B0133ADF86830BDF96850013677
:10A09000761B36B2002E1EDDBDF96E10BDF86A309B
:10A0A0004A1CD21A13B20B93BDF96020BDF9663079
:10A0B000AD1A5B1A0AFB0355059B1AA91D441EA87D
:10A0C0004D4B9847BDF87E30ADF87A3000270B9B9A
:10A0D0009F42C0F2C280BDF94C30ADF8643001330C
:10A0E000A3EB0B03ADF86030BDF84A305B44ADF82C
:10A0F0006230BDF84E30A3EB0B03ADF8663042463C
:10A100003C4B18A91AA8984790B3069B4BB1049BE7
:10A11000BDF96820B3F904309342B8BF1346ADF8D7
:10A120006830BDF86C50BDF968300135ED1A2DB2BC
:10A13000002D1DDDBDF86E20BDF86A100132521AE7
:10A1400012B20B92BDF960200AF1FF369B1A0AFB8E
:10A150000636059B1AA91E441EA8274B9847BDF832
:10A160007A30ADF87E3000270B9B9F42C0F2A28070
:10A17000059A4FEA6A060020D7E030B22146059AD8
:10A180001E4F0690B8470999214401290CDD059B13
:10A19000059A1B8806989B010124B3FBF1F31380F9
:10A1A000AC4203D3059AB847002311E0538832F834
:10A1B000026BB3421EBF9E01B6FBF1F6B6B216802B
:10A1C0000134EDE7059A059932F81320CA5401339A
:10A1D000AB42F7D18BE60023BDE60690BCE60695C0
:10A1E000BAE600BFFD97000025990000FDEE0000D3
:10A1F00019970000D1DE0000A19B0000159A000015
:10A2000029464D4B4D4C324618EE100A9847BDF981
:10A210007A20BDF97810334618EE100AA04799F855
:10A22000293002930128079B454C08BF0220CDE945
:10A2300000031EA918EE103AB9F81E204046A047A8
:10A24000BDF87A300133ADF87A30BDF87E30013395
:10A25000ADF87E3055440137E5E62946364B374C9C
:10A26000324618EE100A9847BDF97A20BDF97810E9
:10A27000334618EE100AA04799F8293002930128B6
:10A28000079B2F4C08BF0220CDE900031EA918EE42
:10A29000103AB9F81E204046A047BDF87A30013B7D
:10A2A000ADF87A30BDF87E30013BADF87E305544D4
:10A2B00001370CE7204B18EE100A2A463146984722
:10A2C000069B53B9BDF97A20BDF978101B4C18EEE6
:10A2D000100A2B46A047012800D1022099F8293006
:10A2E000029399F82830164CCDE900031EA918EE08
:10A2F000103AB9F81E204046A047BDF87A30013325
:10A30000ADF87A30BDF87E300133ADF87E300137DC
:10A310002AE711F8017F13F801CD81F800C01F7002
:10A32000EF1ABE42F5DC5244013082450ADD02EBF1
:10A330000A05511E2B46F3E779EC000069970000EF
:10A34000D9610000BDF94830ADF86030013B5B4495
:10A35000ADF86430BDF94A30ADF86230013B5B4482
:10A36000ADF866304246B94B18A91AA8984700289C
:10A3700037D0BDF96E30089ABDF968509342C4BF1A
:10A380001346ADF86E30099ABDF96C309342C4BFE4
:10A390001346ADF86C30BDF86C600136761B36B2F2
:10A3A000002E1EDDBDF86E30BDF96A2001339B1A08
:10A3B0001BB20B93BDF96230D21ABDF96030ED1AB1
:10A3C000059B0AFB02551D441AA9A14B1EA89847DC
:10A3D000BDF87A30ADF87E3000270B9B9F42C0F26B
:10A3E000A685BDF94830BDF94E20ADF86030013B7F
:10A3F0005B44ADF86430531CA3EB0B03ADF8623043
:10A40000ADF86620914B424618A91AA89847002833
:10A4100039D0BDF96A30089ABDF968509342D8BF67
:10A420000A9B099ADCBF0133ADF86A30BDF96C3084
:10A430009342C4BF1346ADF86C30BDF86C60013672
:10A44000761B36B2002E1EDDBDF96E10BDF86A30E7
:10A450004A1CD21A13B20893BDF96020BDF96630C8
:10A46000AD1A5B1A0AFB0355059B1AA91D441EA8C9
:10A47000774B9847BDF87E30ADF87A300027089BBF
:10A480009F42C0F28285BDF94830ADF86030013B93
:10A490005B44ADF86430BDF84A305B44ADF86230DF
:10A4A000BDF84E30A3EB0B03ADF866304246674B68
:10A4B00018A91AA8984790B3069B4BB1049BBDF905
:10A4C0006C20B3F900309342A8BF1346ADF86C304E
:10A4D000BDF86C50BDF968300135ED1A2DB2002D74
:10A4E0001DDDBDF86E20BDF86A100132521A12B29D
:10A4F0000892BDF960200AF1FF369B1A0AFB063666
:10A50000059B1AA91E441EA8514B9847BDF87A30E6
:10A51000ADF87E300027089B9F42C0F26485BDF8ED
:10A5200048305B44ADF86030BDF84C30A3EB0B0312
:10A53000ADF86430BDF94A30ADF86230013B5B44A0
:10A54000ADF866304246414B18A91AA8984780B327
:10A55000069B4BB1049BBDF96E20B3F902309342C8
:10A56000A8BF1346ADF86E30BDF86C50BDF868302A
:10A57000BDF96A600135ED1ABDF86E3001339B1BE1
:10A580001BB20893BDF96230F61A0AF1FF330AFBD9
:10A590000636059B1AA91E441EA82D4B9847BDF8E8
:10A5A0007A30ADF87E302DB20027089B9F42C0F272
:10A5B0006185BDF84830BDF94E20ADF866205B449A
:10A5C000ADF86030BDF84C30A3EB0B03ADF8643050
:10A5D000531CA3EB0B03ADF8623042461B4B18A98A
:10A5E0001AA89847002835D0069B4BB1049BBDF9AB
:10A5F0006A20B3F906309342B8BF1346ADF86A300B
:10A60000BDF86C50BDF86830BDF96660BDF86A10E1
:10A610000135ED1ABDF96E305A1CF31A0AF1FF36F6
:10A620000AFB0366059B521A12B21E441AA9084B74
:10A6300008921EA89847BDF87E30ADF87A302DB24A
:10A640000027089B9F42C0F24E8503E0D1DE000048
:10A65000A19B0000BDF848305B44ADF86030BDF808
:10A660004C30A3EB0B03ADF86430BDF84A305B44CB
:10A67000ADF86230BDF84E30A3EB0B0BADF866B011
:10A68000B94B424618A91AA89847F8B1069BEBB9EE
:10A69000BDF86C60BDF86830BDF86E70DFF80CA3D3
:10A6A000DFF80CB30136F61ABDF86A300137FF1A2D
:10A6B0001AA9AE4B1EA89847BDF87A30069DADF892
:10A6C0007E3036B23FB2BD42C0F24685A84BA94C9F
:10A6D00018EE900A984718EE100AA0470598A04770
:10A6E00099F80C30052B40F2AB80A04B049916A8CA
:10A6F0009847B9F91030012B24DD99F81430F92B63
:10A7000020D9B9F90030EBB1B9F81230BDF85810C2
:10A71000C3F380020A44BDF85A10ADF85820C3F3C1
:10A7200040020A44ADF85A20BDF85C20C3F3C001D2
:10A73000521AADF85C20BDF85E2003F00103D31A75
:10A74000ADF85E3099F80CA08B4BBAF1FB0F28BF27
:10A750004FF0FF0A9847894B9847834B0590424634
:10A7600016A918A8984700286AD0059BBDF8600074
:10A770001A8ABDF86210831AADF86030059B5C8AB6
:10A78000BDF864309A1AADF8642003F1010BBDF8EE
:10A790006620ABEB000B091B121B0FFA8BF3ADF815
:10A7A0006210ADF86620184608EE103A744B9847D0
:10A7B000744B054698470C90BDF830300D93002B34
:10A7C00040F0F68499F80630023B18BF0123BDF82B
:10A7D0005C60BDF85E400893BDF85A20BDF8583063
:10A7E00001360134F61AA41A24B236B2B442B9F9C9
:10A7F0000030A8BF344664109C42A8BF1C46089B8A
:10A80000002B00F0D884002C40F0D58499F8063055
:10A81000002B40F0808599F80D205B4CCDE901A21A
:10A8200001220092B9F8022016A94046A0474FF035
:10A83000FF3309934E4B099898474E4B284698474B
:10A84000D9F82C00D0B199F83630052B16D94F4BDA
:10A8500098470128064600F2B986D9F82C004C4BDF
:10A8600025A99847012800F052864A4B00934A498F
:10A870004A4B4B4C40F294520220A04799F81430B6
:10A880000593052B40F27A81B9F91030002B00F0C6
:10A890007581B9F91230002B00F07081059BFB2BFC
:10A8A00028BFFF230593344B9847344B98470499AE
:10A8B0002D4B8346424614A89847002800F05E813D
:10A8C000BBF81020BDF85000BBF81240BDF8521084
:10A8D000831AADF85030BDF854309A1AADF85420B0
:10A8E00003F1010ABDF85620254BAAEB000A091B0B
:10A8F000121B0FFA8AFAADF85210ADF856205046E6
:10A900009847204B04469847002840F04A87B9F9F9
:10A910001230A3F10F056B426B411F46049B049953
:10A920009B8809880498B9F90020408801335B1A94
:10A9300019B2049BDB8801331B1A1BB28B42A8BFE0
:10A940000B465B109342A8BF1346002B089340F3BD
:10A950002B87089A0499134D00231EA8A847124B71
:10A9600000211EA826E000BFD1DE0000A19B000050
:10A97000AD970000B1EB0000DD4F000025DA0000CC
:10A98000FDEE0000FD970000D96100001178000085
:10A990006DCF0000E8FD0100B3FD010036FE0100AF
:10A9A00031E90000259900001997000001F000002E
:10A9B0006997000098470B9016A80499C24B9847D6
:10A9C000B9F81210BDF82050B9F81030BDF8582071
:10A9D00048075EBF5B195B429BB21344B9F8102075
:10A9E000ADF858300B0758BF5319BDF85C0056BF7F
:10A9F0005B4213469BB2C31A8E07ADF85C3058BF5A
:10AA00005319BDF85A00B14E56BF5B4213469BB274
:10AA10000344ADF85A30CB075CBF53195B42BDF815
:10AA20005E004CBF13469BB2C31AAA1A12B2ADF80D
:10AA30005E3016A9012325A8B047A54B002125A803
:10AA40009847B9F91030089ABBF912C0BDF95260A5
:10AA50009A42ACBF089B03F1FF330793B9F80E305D
:10AA600008EE103A99F815300693049B08EE900A08
:10AA70000CEB0600B3F90010B3F9042000B2002F6C
:10AA800000F0A687049B079FB3F90230ADF8601071
:10AA9000A3EB0C03BDF956C0ADF864203B449C45C4
:10AAA000A8BF9C46CDF824C0ADF86200ADF86600A2
:10AAB000099BB34280F27D86049ABBF91230B2F949
:10AAC0000660079AF61AB21ABDF952609642B8BFEC
:10AAD0001646099AB242A4BF1646013633441BB249
:10AAE000ADF86230ADF86630BDF956309E4240F3A5
:10AAF000DF86049B079A5B88764D013313FA82F355
:10AB0000ADF86230049BDB88013B9B1AADF86630E0
:10AB1000049BB9F81020B3F90030ADF86030013A69
:10AB20001344ADF86430069B02930126059B019304
:10AB300018EE102A002318A940460096A847049B47
:10AB4000B3F90420B9F81030ADF86420F31A1344B7
:10AB5000ADF86030069B0293059B18EE102ACDE9F4
:10AB6000006318A900234046A8475B4D18EE900AE1
:10AB7000A8470B98A847594B20469847D9F83C104E
:10AB8000002967D099F84430052B63D9002447F693
:10AB90001843CDE90134B9F94E300093B9F94C307E
:10ABA000D9F840204E4D18A8A847BDF8603099F854
:10ABB00050200498ADF87840013BADF87C30BDF8EA
:10ABC0006230ADF87A40013BADF87E301EA91AAB79
:10ABD000444DA847B9F84830BDF86820B9F84A1084
:10ABE0001A44BDF8783013FA82F3ADF87830BDF826
:10ABF0006A300B44BDF87A1011FA83F1ADF87A107F
:10AC0000BDF87C1011FA82F2ADF87C20BDF87E20F0
:10AC100012FA83F3ADF87E3025A8334B9847D9F864
:10AC200040302693B9F84C30ADF8A030B9F84E302A
:10AC3000ADF89E30B9F84630ADF8943099F844300C
:10AC400000948DF89C30294CD9F83C3025AA414617
:10AC50001EA8A04799F81C300593052B40F262818D
:10AC6000B9F91830002B00F05D81059B164DFB2BC8
:10AC700028BFFF2305931E4B984704990A9012A8FA
:10AC8000A847B9F81A70BDF84830BDF84AA0069335
:10AC9000DB1BADF84830AAEB0703ADF84A30BDF82E
:10ACA0004E30BDF84C403B449BB23C440793ADF85A
:10ACB0004E30A4B2B9F900300B9312A9B9F918308B
:10ACC000ADF84C4016E000BFA19B000025990000A4
:10ACD00019970000D9610000AD970000B1EB0000AA
:10ACE000FD01010079E10000557800008578000041
:10ACF000FD97000014A80C93A847B9F81860BDF898
:10AD00005030BDF854B0BDF8565008939B1BADF8B9
:10AD10005030BDF852300993B34435449B1B1FFAA1
:10AD20008BFBADB2ADF85230ADF854B0C64BADF8B8
:10AD300056509847C54B9847C54B0490424614A9B6
:10AD400016A89847002800F0ED80069B0899BDF8EA
:10AD50005800C3F10102CAF1010A079BC1F10101C8
:10AD600031443A4457443B4422448B4409991CB231
:10AD700012B2A242C1F101010B9BA8BF22460E44B0
:10AD800052102E449A4236B20FFA8BFBA8BF1A46D5
:10AD90005E450C9BA8BF5E4613444FEA660B9B457D
:10ADA000A8BF9B46049BAB4E198A431AADF8583096
:10ADB000049B5C8ABDF85A301B1BADF85A30BDF8B5
:10ADC0005C30591AADF85C105D1CBDF85E102D1A90
:10ADD000091B2BB208EE103AADF85E10012312A940
:10ADE0001EA8B0479C4C00211EA8A0470FFA8BF26A
:10ADF000002314A908EE900A25A8B047002125A831
:10AE0000A047964B09EE100A18EE100A9847B9F9B8
:10AE10001830BDF95A600A9AB9F81670BDF9541085
:10AE20009B45BCBF03F1FF33079399F81D30069390
:10AE3000049BA8BFCDF81CB0B3F912C00CEB0603FD
:10AE400004461BB2BDF95000002A40F04987BDF905
:10AE50005220079DADF86000A2EB0C0202EB050A40
:10AE6000ADF86410ADF86230ADF86630B24580F2EE
:10AE70003086049BBDF95660B3F91230079AF61A72
:10AE8000B61AB245A8BF0AF1010633441BB2ADF8A9
:10AE90006230ADF86630BDF95E309E4240F39A866E
:10AEA000BDF85230079A6E4D013313FA82F3ADF8B4
:10AEB0006230BDF85630013B9B1AADF86630BDF9E3
:10AEC0005030B9F81820ADF86030013B1344ADF8AC
:10AED0006430069B02930126059B01933A460023AA
:10AEE00018A940460096A847BDF95420B9F8181093
:10AEF000ADF8642093195B1AADF86030069B02939D
:10AF0000059B3A46CDE9006318A900234046A847AF
:10AF1000544D18EE900AA84719EE100AA847524B54
:10AF2000204698472DB0BDEC048BBDE8F08F294634
:10AF30004E4B4F4C324618EE100A9847BDF97A2016
:10AF4000BDF97810334618EE100AA04799F8293059
:10AF500002930128079B424C08BF0220CDE9000361
:10AF60001EA918EE103AB9F81E204046A047BDF8B9
:10AF70007A300133ADF87A30BDF87E300133ADF868
:10AF80007E3055440137FFF728BA2946374B384CF5
:10AF9000324618EE100A9847BDF97A20BDF97810AC
:10AFA000334618EE100AA04799F829300293012879
:10AFB000079B2B4C08BF0220CDE900031EA918EE09
:10AFC000103AB9F81E204046A047BDF87A30013B40
:10AFD000ADF87A30BDF87E30013BADF87E30554497
:10AFE0000137FFF74CBA214B18EE100A2A463146BA
:10AFF0009847069B53B9BDF97A20BDF978101C4CCF
:10B0000018EE100A2B46A047012800D1022099F81B
:10B010002930029399F82830114CCDE900031EA97C
:10B0200018EE103AB9F81E204046A047BDF87A3015
:10B030000133ADF87A30BDF87E300133ADF87E30A3
:10B040000137FFF768BA00BFDD4F000025DA0000C6
:10B05000D1DE00002599000019970000FDEE0000E8
:10B06000D9610000AD970000B1EB000079EC000061
:10B07000699700003378079A02EA0301FF291CBF91
:10B0800012FB03F3C3F3072118EE100AAA4B2A465A
:10B090009847069B53B9BDF97A20BDF97810A74CA3
:10B0A00018EE100A2B46A047012800D1022099F87B
:10B0B00029300293FF23CDE90003A14CB9F81E20EB
:10B0C00018EE103A1EA94046A047BDF87A30013369
:10B0D000ADF87A30BDF87E300133ADF87E3056449D
:10B0E0000137FFF762BA3378079A02EA0301FF29B2
:10B0F0001CBF12FB03F3C3F3072118EE100A8E4B9B
:10B100002A469847069B53B9BDF97A20BDF97810B5
:10B110008A4C18EE100A2B46A047012800D10220C5
:10B1200099F829300293FF23CDE90003844CB9F844
:10B130001E2018EE103A1EA94046A047BDF87A30EE
:10B14000013BADF87A30BDF87E30013BADF87E3082
:10B1500056440137FFF775BA99F82810784C18EE65
:10B16000100A3246D047BDF97A20BDF9781033462F
:10B1700018EE100AD84799F829300293012808BF21
:10B180000220FF23CDE900031EA918EE103AB9F8FA
:10B190001E204046A047BDF87A300133ADF87A3022
:10B1A000BDF87E300133ADF87E300135FFF78BBA44
:10B1B0000023FFF70CBB002C40F3AD800023224698
:10B1C00016A925A85F4FB8475F4B002125A89847CF
:10B1D000099099F80630B9F802B0022B40F0A88027
:10B1E000B9F804205A4500F0A380584B70009847E6
:10B1F00000270690BE42564B00F39180BDF95C20BB
:10B20000BDF95810ADF86C20531C5B1A1BB2A3EBB0
:10B2100044030A93059BBDF962205B8AADF8681070
:10B2200013441BB2ADF86A30ADF86E300792BDF929
:10B230006630079A9A4240F38F8099F806300C9A4C
:10B240001A4312F0FF035DD10A9A322A5ADDBDF883
:10B250005820A6B212FA84F4BDF85C20ADF868401C
:10B26000921BADF86C20BDF95A20ADF86A2032442B
:10B27000ADF86E2099F80D20314CCDE901A20122E4
:10B280000092B9F802201AA94046A047BDF95E1005
:10B29000BDF96E302A4CADF86E108A1B12B29A427C
:10B2A000D8BF0133ADF86A20D8BFADF86A3099F83D
:10B2B0000D30CDE901A301270097B9F80220002342
:10B2C0001AA94046A047BDF85830ADF86830BDF81F
:10B2D0005C30ADF86C30BDF85A303B443344ADF8C7
:10B2E0006A30BDF85E30013B9E1B99F80D30009727
:10B2F000CDE901A3ADF86E60B9F8022000231AA9C8
:10B300004046A047069B002B3FF494AA1846114BD9
:10B310009847FFF78FBA4FF0FF33099359E73AB2D6
:10B32000314648469847069B23F81700013761E7E6
:10B330000023069362E700BF01F000006997000058
:10B34000D96100002599000019970000FDEE00006A
:10B3500081990000B1EB0000059BB3F91270079BC7
:10B360001F44BDF95A30234401339F4209DDBDF922
:10B370005E301B1B013B9F4203DA089B002B40F011
:10B38000958018EE101ABC4BBC4E28469847059B7A
:10B390005A8A079B1A44059B198ABDF860301944E4
:10B3A00012B218EE103A09B22846B047064699F88C
:10B3B0000630012B12D1B9F80220B9F804309A42B4
:10B3C0000CD0BDF85E10BDF85A300131FA1AC91A16
:10B3D00012B2AB4B09B2484698478346089B002BF4
:10B3E00066D00A9B322B63DDBDF95A3023449F425D
:10B3F00004DDBDF95E301B1B9F4259DBBDF958309F
:10B40000ADF87830013B13FA84F3ADF87C30BDF829
:10B410006A30ADF87A30BDF86E30ADF87E3099F80C
:10B420000D30984F0096A2B2CDE901A30B922B46A6
:10B430005A461EA94046B84799F80620012A14D159
:10B440000B99BDF858300B44ADF87830BDF85C303E
:10B450005B1AADF87C3099F80D300092CDE901A36C
:10B460005A4600231EA94046B847BDF95C300B99E7
:10B47000ADF87C305A1C571A059AADF87870B2F9BD
:10B480001020BDF960101B1B0A4401339B1A99F868
:10B490000D200096CDE901A2002BACBFEB182B1CB0
:10B4A0005A461EA9774E4046B04710E001267EE777
:10B4B00099F80630022B18D199F80D30069A0096AB
:10B4C000CDE901A3704E2B461AA94046B047BDF8FE
:10B4D0006A300133ADF86A30BDF86E300133ADF833
:10B4E0006E30079B01330793A1E6012B08D199F831
:10B4F0000D300096CDE901A35A462B461AA9D1E793
:10B500000D9B002BF3D10A9B322BE0DCEFE75F4B66
:10B51000259DBDF896A01AA8984799F836308DF861
:10B52000683099F837308DF87230B9F83430ADF8AA
:10B530007430C5F38A25CAF34A1A1FFA8AF77B1EAC
:10B540001FFA83FB99F83830B9F90020DB0740F186
:10B55000CF8004994E4C002325A8A0474D4B0021D5
:10B5600025A89847049B9C881B880134E41A24B2C0
:10B5700094FBF5F305FB134404EBD47463100593BB
:10B58000049B5A88DB8801339B1A1BB293FBFAF1A8
:10B590000AFB113A0AEBDA7AA2EB6A0A1FFA8AFA74
:10B5A000ADF862A008EE100ADA44DFF80CB1ADF88D
:10B5B00066A0049BBDF96220B3F906309A423ADDD9
:10B5C00018EE100A344B9847FFF758B9022821D1DA
:10B5D000324B334C1EA89847B9F83430ADF8783068
:10B5E00099F836308DF88030002147F61843D9F8A5
:10B5F00030201F92CDE90131BDF982300093D9F896
:10B600002C10BDF9843025A8A047BDF99450BDF990
:10B6100096A092E7234B00932349244B244C40F2FD
:10B62000AE520220A04700230498224C1A464146FD
:10B63000A047FFF723B9049B059A1B881FFA85FAD8
:10B640009B1A9BB20AF1FF32ADF860301344ADF89B
:10B650006430049BBDF96020B3F904309A422DDDBB
:10B66000BDF862303B44ADF86230BDF866303B4413
:10B67000ADF866309DE700BFBDF00000699700009F
:10B6800081990000D9610000D56700005175000064
:10B690002599000019970000AD970000557800002B
:10B6A000FD01010007FE0100B3FD010036FE0100AF
:10B6B00031E90000C175000085780000022ED9F83C
:10B6C0002C200FD1002300934146134618A81EAA30
:10B6D000D847BDF860305344ADF86030BDF86430F1
:10B6E0005344B4E7B24C1AAB414618A8A047F0E760
:10B6F0000499049B89881C885888DB880131091BC0
:10B7000001331B1A09B2491B1BB201EBD171A3EB28
:10B710000A0304EB610103EBD37400EB640089B20C
:10B7200080B2013D0D44ADF8601000EB0B0189B211
:10B73000022EADF86200ADF86450ADF8661007D186
:10B7400003F0010318440B44ADF86200ADF8663015
:10B750000499984B18A898470446C8B90346B9F904
:10B7600000200499944D25A8A8472146934B25A86D
:10B7700098470446022ED9F82C200CD100230093C0
:10B780008F4D134641461EAA18A8A847204619E720
:10B790004FF0FF34EEE7864D1AAB414618A8A84794
:10B7A000F4E70023FFF7B9B84FF0FF330B93FFF72F
:10B7B00003B9844B844F514620469847BDF850301A
:10B7C000BBF81220BBF810103244194412B2534691
:10B7D00009B22046B847BDF86230ADF86A30BDF80E
:10B7E0006630ADF86E30049B0A90B3F90030ADF8C6
:10B7F0006830013B2B44ADF86C30069B0293059BEF
:10B80000019318EE102A009023461AA96F4F404664
:10B81000B847049BB9F91010B3F90230BDF96E2096
:10B820000B449A4215DA049B1B882B44ADF8683010
:10B83000049B9B885B1BADF86C30069B0293059BB9
:10B8400001930123009318EE102A00231AA9404601
:10B85000B847049BBDF95010B3F90430ADF86C3013
:10B860005A1C521BADF86820089A584F9B1ABBF916
:10B87000102001330A449B1A069A0292059A0192FB
:10B880000A9A0092002BACBFE318231C18EE102A72
:10B890001AA94046B847BDF862300133ADF86230AE
:10B8A000BDF866300133ADF866300136FFF700B9F8
:10B8B000444B454F514620469847BDF85030BBF8A1
:10B8C0001220BBF810103244194412B2534609B288
:10B8D0002046B847049B0990B3F90030ADF86830B2
:10B8E000013B2B44ADF86C30BDF86230ADF86A30E6
:10B8F000BDF86630ADF86E30069B0293059B019350
:10B9000018EE102A009023461AA9304F4046B84737
:10B91000049BB9F91010B3F90630BDF96E205B1A1B
:10B920009A4215DD049B1B882B44ADF86830049BBC
:10B930009B885B1BADF86C30069B0293059B0193C3
:10B940000123009318EE102A00231AA94046B84795
:10B95000049BBDF95010B3F90430ADF86C305A1C9B
:10B96000521BADF86820089A184F9B1ABBF910209B
:10B9700001330A449B1A069A0292059A0192099A87
:10B980000092002BACBFE318231C18EE102A1AA952
:10B990004046B847BDF862300133ADF86230BDF8BB
:10B9A00066300133ADF866300136FFF79DB800BF51
:10B9B000C1750000D9E0000025990000199700002A
:10B9C00085780000BDF0000069970000D961000093
:10B9D000B9F91230ADF86010042BADF86420ADF861
:10B9E0006200ADF8660061D1079A8A18ADF864204C
:10B9F0000022022B8DF83E208DF83F205DD10123DF
:10BA00008DF83E309DF83E30002B60D19DF83F30E0
:10BA100083F0010303F00103AE4D8DF84030BDF912
:10BA200056309E423FF7A1A89DF84030ABB99DF833
:10BA30003E30BDF9622033B1049B0799B3F902305F
:10BA40000B449A4209DD9DF83F301BB3049B0799D4
:10BA5000B3F906305B1A9A421CDB9F4B9F4F51464D
:10BA600020469847BDF85030BBF81220BBF81010A4
:10BA70003244194412B2534609B22046B847069BD5
:10BA80000293059B18EE102ACDE9000318A923465E
:10BA90004046A847BDF862300133ADF86230BDF8CA
:10BAA00066300133ADF866300136B8E7082B02BFC7
:10BAB0000799521AADF860209AE7012B04D0032BA6
:10BAC000A0D101238DF83E308DF83F309AE7002356
:10BAD000A0E718EE101A804B804D20469847049B33
:10BAE0005A8A198ABDF858303244194412B218EEF5
:10BAF000103A09B22046A847BDF86230ADF86A3066
:10BB0000BDF86630ADF86E30BDF95030ADF8683034
:10BB1000013B13FA8BF3ADF86C30069B02931FFACE
:10BB20008BF2059B099008920193009023463A46B8
:10BB30001AA9684D4046A847BDF95230B9F9181006
:10BB4000BDF96E200B449A4215DA089ABDF85030C0
:10BB50001344ADF86830BDF854309B1AADF86C3022
:10BB6000069B0293059B0193012300933A46002311
:10BB70001AA94046A847BDF954300899ADF86C3071
:10BB80005A1C521AADF86820049ABDF95810B2F93F
:10BB90001020504DA3EB0B030A4401339B1A069A65
:10BBA0000292059A0192099A0092002BACBFE31809
:10BBB000231C3A461AA94046A847BDF86230013313
:10BBC000ADF86230BDF866300133ADF8663001364D
:10BBD000FFF74CB918EE101A3F4B404D20469847DE
:10BBE000049B5A8A198ABDF858303244194412B25B
:10BBF00018EE103A09B22046A847BDF95030ADF80A
:10BC00006830013B13FA8BF3ADF86C30BDF862304D
:10BC1000ADF86A30BDF86630ADF86E30069B029321
:10BC2000059B08900193009023463A461AA9294D96
:10BC30004046A847BDF95630B9F91810BDF96E2035
:10BC40005B1A9A421FFA8BFA15DDBDF85030534447
:10BC5000ADF86830BDF85430A3EB0A03ADF86C3092
:10BC6000069B0293059B0193012300933A46002310
:10BC70001AA94046A847BDF95430BDF95810ADF88F
:10BC80006C305A1CA2EB0A02ADF86820049A114DE0
:10BC9000B2F91020A3EB0B030A4401339B1A069A56
:10BCA0000292059A0192089A0092002BACBFE31809
:10BCB000231C3A461AA94046A847BDF86230013312
:10BCC000ADF86230BDF866300133ADF8663001364C
:10BCD000FFF7E1B8D9610000BDF0000069970000EE
:10BCE000DFF87090DFF870B0DFF870A0ADF860009A
:10BCF000ADF86410ADF86230ADF86630BDF95E3075
:10BD00009E423FF705A918EE101A2046C847049B2B
:10BD10005A8A198ABDF858303244194412B218EEC2
:10BD2000103A09B22046D847069B0293059B3A4633
:10BD3000CDE9000318A923464046D047BDF862303C
:10BD40000133ADF86230BDF866300133ADF86630CE
:10BD50000136D3E7BDF0000069970000D96100000B
:10BD6000F0B5C2F1FF03C1F34514C0F345155C43C0
:10BD700048F2810605FB02447443C4F3C55501F043
:10BD80001F0400F01F075C43C1F3C42107FB0244FA
:10BD9000C0F3C420594300FB021374437343C4F33C
:10BDA000C45444EA4514DB0D44EAC320F0BD013914
:10BDB0000244904200D1704711F8013F00F8013B66
:10BDC000F7E70000F7B586680746007815460022B9
:10BDD000ADF8042000F01F020C46111F022916D8EE
:10BDE000344B104698473B68C0F3C700C3F38A231F
:10BDF00013FB05F310FB04F100FB031102222E4B91
:10BE0000314401A89847BDF8040003B0F0BD072AEB
:10BE100014D104F00703C3F107023B68C3F38A237C
:10BE20000733DB1005FB036303EBE4040121237AF2
:10BE300091400B401341ADF80430E4E7082A16D1D5
:10BE40003868C0F38A200330801005FB006304F0DB
:10BE5000030203EBA4045200237CC2F10602032177
:10BE600091400B4043FA02F2ADF80420CBE7092AD7
:10BE700011D13B68C3F38A2301335B1005FB0363D5
:10BE800004F0010203EB6404920094F84030C2F124
:10BE900004020F21E4E70A2A08D13B68C3F38A238E
:10BEA00015FB0343334493F80034C4E70B3A032AE9
:10BEB000A9D8C0E779750000AFBD0000F0B50B460A
:10BEC0000178856801F01F01052985B004460AD173
:10BED0000168C1F38A2112FB013303EB43032B44B6
:10BEE000987805B0F0BD0B2916D10068C0F38A2000
:10BEF0000730C01002FB005203F00706DB10C6F14A
:10BF00000706D35C0122B240134033410CBF4FF00F
:10BF1000FF300020C0B2E4E70C2918D100682049A6
:10BF20000091C0F38A200330801003F0030602FB67
:10BF300000529B107600D35CC6F106060322B24085
:10BF40001340334110336B4413F8100CC9E70D292B
:10BF50001BD1144EEC4606F1100E3068716867462E
:10BF600003C708367645BC46F7D12068C0F38A205F
:10BF70000130401003F0010602FB00525B10B600D6
:10BF8000D35CC6F104060F22D9E70E2903BF01686E
:10BF9000C1F38A2112FB0133FF2008BFE85CA0E750
:10BFA0000055AAFF43FE01002DE9F84FB0F9083013
:10BFB000DFF8EC801B024362B0F90A301B020A264C
:10BFC0008362B0F90C3093FBF6F51FFA85F904464D
:10BFD000C9F100004FF6F67700B215FB0737C047EE
:10BFE0000135ADB28246684200B2C0478346C9F10E
:10BFF0005A0000B2C047C5F15A05814628B2C04771
:10C00000F51B07FB0BF107FB00F305FB0A1205FB11
:10C01000093092FBF6F2204BE26290FBF6F02063CF
:10C02000A07C984794F8343060F3000384F83430EF
:10C03000A07C1A4B9847A37C1A1F022A8CBF0021B0
:10C040000121420042EA810294F8341002F0060213
:10C0500021F006010A4384F8342022682262A28873
:10C0600003F01F03C2F30A0243EA8223B4F9062055
:10C0700043EA4253A26902F440721343A361E28986
:10C080004FF48033B3FBF2F3E386FF23A375238AD7
:10C09000A382BDE8F88F00BF91750000A575000070
:10C0A00085E900002DE9F04F85B007465E4DBDF8EB
:10C0B000388002914FF00A094FF6F67B93FBF9F6B0
:10C0C000304616FB0B3B1446A8470390701C00B289
:10C0D000A847B6B2824606F15A0000B2A8470190BE
:10C0E00006F15B0000B2A847039B0199A9EB0B0680
:10C0F0000BFB0AF506FB03550F9B95FBF9F5B3F90E
:10C1000002C0B3F900E0CCF10002CEF1000308FB5D
:10C1100003F308FB02F20BFB00F043F30F2342F39F
:10C120000F2205FB02FA06FB010090FBF9F000FB71
:10C1300003F942436B439918C91311FA8CF109B200
:10C1400001910299A1EB0E0108FB01F141F30F21CE
:10C15000A4EB0C0400FB01FB08FB04F4A9EB0A06AA
:10C1600044F30F24ABEB0A0A6943F61365434FEA25
:10C17000EA3A16FA8EF61AFA8EFAA9EB050936B2E1
:10C180000FFA8AFA4FEAE939564500FB04F419FA26
:10C190008EF9ABEB05050FFA89F90A4423444FEAFF
:10C1A000E5350C443146A8BF5146494515FA8EFE87
:10C1B0000FFA8EFEA8BF49467145A8BF7146564585
:10C1C000B8BF5646B1454FEAE232B8BFB14612FA9F
:10C1D0008CF23980019912B2CE454FEAE333B8BFF1
:10C1E000CE4613FA8CF391421BB2A8BF1146E4135A
:10C1F000994214FA8CFC0FFA8CFCA8BF19466145D1
:10C20000A8BF614679800199A7F804E08A42B8BFC7
:10C210000A469342B8BF13469C45B8BF9C46A7F850
:10C2200006C005B0BDE8F08F85E900002DE9F04FAC
:10C2300090F83820D0F80080B0F93850B0F93A6062
:10C2400090F83A306F2A89B0044600F29380B0F932
:10C250003C90B9F1000FD4BF4FF000094FF0010935
:10C26000C9F10009803DEDB26F2B00F29880B4F95E
:10C270003E70002FD4BF002701277F42803EF6B2D8
:10C28000A38AADF80A30A37D019394F8343058079F
:10C2900040F1AA8094F84430216CDFF844A209FBF5
:10C2A00003110222414405A8D04794F84410A38802
:10C2B00011FB03F3216C07FB03110222414406A882
:10C2C000D04794F84420A388216C13FB02F309FBA8
:10C2D000021107FB03114144022207A8D04794F83A
:10C2E000343099076CD400200746834694F83430E4
:10C2F0009B0740F1C880019AC5F1FF0312FB05FCC2
:10C3000003FB0BCC4343CCF3072C15FB0733C3F3E0
:10C310000723C6F1FF0206FB0CF103FB0212121207
:10C32000BCF1050FA27500F2AA80052B40F2D48063
:10C330000026019B052B94BF00222A46BBF1050F66
:10C3400098BFFF22052F98BF0025052898BFFF251D
:10C35000002A40F09C80BDF81470002D40F0A480AD
:10C36000BDF81C10002E40F0AD80A182012009B064
:10C37000BDE8F08F902A0ED9B0F93C90B0F90410C6
:10C3800009F101098945ACBF4FF000094FF00109DF
:10C39000C5F17F0567E7FF254FF0000964E7902BA3
:10C3A0000BD9B4F93E70B4F9062001379742ACBFFF
:10C3B00000270127C6F17F0661E7FF2600275FE718
:10C3C000236C94F84410A288013B0B4409FB01390B
:10C3D00012FB01F27A4308EB020118F809B0CF5CB6
:10C3E000C84418F8020081E7A18FDFF8F8B0238A6B
:10C3F000B4F93E2004F1180A11FA89F109B2504645
:10C40000D847E28FB4F93C10ADF81400BBB212FA71
:10C4100087F2009312B2238A5046D847009BE28FDE
:10C42000A18FADF818001FFA89F81A444144238AF5
:10C4300012B209B25046D84794F83430ADF81C0017
:10C440009A077FF550AFB4F93C70B4F93E20DFF89D
:10C4500098900392B8440FFA88F841465046C8476E
:10C46000009B039A13441AB2394683465046009201
:10C47000C847009A074641465046C84736E7052B4D
:10C4800098BFFF2655E7FF23A3752A4660E7FF2ADA
:10C4900002D1BDF80A7060E7BDF81410BDF80A00BB
:10C4A0000E4B9847074658E7FF2D02D1BDF81810EC
:10C4B00058E7BDF81C10BDF81800084B2A469847ED
:10C4C00001464FE7FF2E01D1A7824FE7034B3246CB
:10C4D00038469847A08249E7002048E761BD000040
:10C4E000AFBD0000C5BD0000BDBE00002DE9F74F87
:10C4F000DFF89081B8F8004005460E465CB9524B13
:10C5000000935249524B534D44220220A8472046E3
:10C5100003B0BDE8F08F504B50481F6800233A46E7
:10C52000116A01338142A8BF01F1FF319BB2A8BF5C
:10C5300011629C4202F12402F2D1DFF84CB14FF0BB
:10C54000000A4FF02409B8F800101FFA8AF291424D
:10C5500039D807F124023C460123994256D8636832
:10C56000DFF8F080002B5AD03D4B204698473D4BDA
:10C570000093374B772235490120C0473A4B984703
:10C580004FF000092946394BC4F81490074632464B
:10C59000204698470546002846D1354B2B49009345
:10C5A00083222B4B334E0220C0472D4B2046984709
:10C5B00020462021B04720462421B0474FF00043B9
:10C5C00023622C46A3E71FFA8AF409FB04742A4B62
:10C5D0006068984780B96268AA4214D12189B2B2D2
:10C5E000914210D1236A62691344B3F57A7FC8BFC0
:10C5F0004FF47A7323628AE7012804D160682946E0
:10C60000D8470028EED00AF1010A9CE7176A206A91
:10C6100001338742B8BF14469BB224329DE7174BC3
:10C6200000937A220A4BA6E76369C4F82090002B96
:10C630007FF46DAF124B3846984708B1606166E7EA
:10C640000123636163E700BF9FFE01006AFE0100F2
:10C6500052FF010031E900006C86002002000080DA
:10C6600091D00000C6FE01008DDA0000C1CF0000AD
:10C6700028FF010061F0000011780000F7FE0100C2
:10C68000A1DA0000D085002059630100144B2DE988
:10C69000F7431F68134E144DDFF8508004464FF0E7
:10C6A000000932881FFA89F39A4202D803B0BDE824
:10C6B000F0831FFA89F3242000FB03704368A34230
:10C6C00000D04CB913B10190C047019801902021CE
:10C6D000A84701982421A84709F10109E1E700BF13
:10C6E0006C860020D085002061F0000091D0000011
:10C6F0002DE9F7431F4C236805462BB11E4B002044
:10C70000984720681D4B984724271D4B07FB05F0D1
:10C7100098471C4B20609847064660B91A4B1B4946
:10C720000093A82203201A4DA847226819481A49E5
:10C7300033468847FEE72368DFF8608023B9A8F80E
:10C74000003003B0BDE8F083DFF85490A8F8005043
:10C750000025B8F80020ABB29A42F2D92068AEB2F8
:10C760007E4320213044C847206824213044C847F4
:10C770000135EEE76C8600208DC600002DEB000031
:10C7800075EA00009517000065FF01006AFE0100D0
:10C7900031E9000002EE01009D170000D085002065
:10C7A00061F0000070B52C4B86B008460E46154669
:10C7B00098470446D8B93378C3F30403043BDBB28B
:10C7C0000A2B11D873886A883168C3F34A1363F35C
:10C7D0004F126A802B68214A23F01F1323F47C43F5
:10C7E0000A4013432B600124204606B070BD012887
:10C7F00025D11B4B0222314604A89847B8B9194EDF
:10C8000003AB0422294604A8B047174B064604A8E8
:10C81000984716B9039B042B09D0144B0093144B73
:10C8200040F221121349144C0220A04705E02B7856
:10C830001C3303F01F030A2BD6D90024D4E70228A7
:10C8400004D12B6803F478720C4BCAE70C4B0093AD
:10C850004FF49A72064BE5E7117800001FFC1F00A9
:10C86000E9E4000061E4000031E40000B2FF0100EF
:10C87000200102007BFF010031E900000B042000D1
:10C88000D6FF010070B5CC690D4684B12068084E12
:10C8900018B1084B98472068B047606800B1B047AE
:10C8A000A06800B1B0472046B0470023EB6170BDDF
:10C8B0002DEB000031E400002DE9F04F087B8DB036
:10C8C000984600F01E03042BBDF958A0179E0D4694
:10C8D000144603D000F01F03062B3DD195F80A90B3
:10C8E000B9F1010F35D1B34BD5F81CB000F01F00E2
:10C8F0009847E968B04BC1F38A2118FB01414143D5
:10C90000C91007460431DBF80000984748B1AB4B2B
:10C910000093AB4B40F22E22AA49AB4C0220A04719
:10C9200017E0C7F3C70717FB0AFA089008ABDBF854
:10C930000000A64D52463146A847089B9A4579D03B
:10C94000A34B00939F499E4B9F4D40F235220220FE
:10C95000A8474FF000096DE0A3F10B02032A00F293
:10C96000CE804FF47F43ADF81830A3F5AD03A3F5A7
:10C9700028530793974B08AA03F1100E174618681F
:10C9800059689446ACE80300083373456246F6D113
:10C99000298933464FEA112C002210B2824503F157
:10C9A000030314DC287B834B00F01F00984701230E
:10C9B0008340013B9BB204932B7B03F01F030B3B93
:10C9C0008146032B6AD8DFE803F008394D6003F88D
:10C9D000031C03F802CC0132DFE7EB68C3F34732F4
:10C9E00013F4E05F4FEAE4010CBF0FFA82FB02F19F
:10C9F000010BE4430BFB081104F0070406AFEB69DD
:10CA000003935846744B05919847AB7A0599804635
:10CA1000002B47D16B689B681944C9F108000023BB
:10CA2000023640B21AB292454BDC6C4B40469847F6
:10CA30004FF0010948460DB0BDE8F08FEB68A1103A
:10CA4000C3F3083213F4406F6FEA04040CBF0FFA0B
:10CA500082FB02F1010B04F003040BFB08116400DC
:10CA600007AFCCE7EB685905C3F3C9224FEA64016D
:10CA700054BF0FFA82FB02F1010B14F0010F0BFB04
:10CA800008110CBF04240024B9E7EA68C2F38A2124
:10CA90008B4618FB014100242746B0E700242146BD
:10CAA000A346F9E7039B04311868434B9847039862
:10CAB0005A4641460068DFF814B10023D847414682
:10CAC000ABE7049A91F800E002FA04FC0EEA0C02CB
:10CAD00095F80CC022410CF01F0CD2B2A4EB090453
:10CAE000BCF10E0F64B203EB430C18BFBA5C06F83E
:10CAF0000C20002CBCBF04460131013392E7073BF8
:10CB0000032B00F2AF802B4B00F01F00984701274A
:10CB10008740013FBBB203932B7B03F01F03073B0E
:10CB20008146032B00F28C80DFE803F0025A6D800F
:10CB3000EB68C3F3473213F4E05F4FEAE4010CBF44
:10CB400017B2571C07FB0818E44308F1080104F06A
:10CB50000704214B04913846D5F81CB09847AB7AAE
:10CB600004998046002B6FD16B689B681944C9F10A
:10CB7000080500206DB203B29A457FF756AF039ABD
:10CB80000B78A24013402341DBF80420DBB2A4EB76
:10CB9000090432F813203270120A7270DBF8082090
:10CBA00064B2002CD35CB370BCBF2C4601310130A1
:10CBB0000336E0E77975000097E40000FCFF010010
:10CBC0003D0102007BFF010031E9000061E400004B
:10CBD0001F00020065010200FDEE0000B1EB000045
:10CBE000EB68C3F3083213F4406F4FEAA4010CBFA3
:10CBF00017B2571CE44307FB081804F0030408F1BC
:10CC000010016400A5E7EB68C3F3C9225B054FEA96
:10CC1000640154BF17B2571C07FB081814F0010F2A
:10CC200008F140010CBF0424002492E7EF68C7F329
:10CC30008A2118FB01480F46002408F5806188E727
:10CC400000210C460F4684E7094BDBF80000094D34
:10CC5000043198474146DBF8000000233A46A847D4
:10CC6000414684E7044B00934FF4FE72034B53E6B6
:10CC700097E4000061E40000420002007501020038
:10CC80002DE9FF470646887A01280C4678D1486886
:10CC90008B4B98478B498C4B9847002840F0A980D4
:10CCA00061688A4B022202A8984738B1884B0093EA
:10CCB000884B4FF4A6728849022022E0E369DFF82E
:10CCC0003C92DFF83C8213BB0C20C847E061C047B0
:10CCD000054668B97F4B8049009340F25312032008
:10CCE0007E4EB047E2697E487E492B468847FEE784
:10CCF000E06948B97C4B00937749764B40F2551276
:10CD00000320764CA04774E0784B0C21984708200C
:10CD1000E769C8473860C047054668B96D4B6E493A
:10CD2000009340F25D1203206C4CA0473A686C48B7
:10CD30006C492B468847FEE73B684BB96A4B00932A
:10CD4000644B40F25F126449644D0320A8474CE0F5
:10CD500002AA03F1080112F8010B03F8010B8B4240
:10CD6000F9D1237B03F01F00021F022A11D8A37AF6
:10CD7000002B40F0878063689B682361012005E0F9
:10CD80000028EED14A689268002AEAD104B0BDE8D2
:10CD9000F087C21F032A00F2D480554BDFF85C9164
:10CDA000DFF85C819847E369074643BB0C20C8471E
:10CDB000E061C047054668B9464B474900934FF4C8
:10CDC000C6720320454EB047E269454845492B46A7
:10CDD0008847FEE7E56975B9434B00933E493D4BF3
:10CDE0003E4F4FF4C7720320B847424B21463046AE
:10CDF00098470020CAE73D4B0C212846984702205F
:10CE0000B840E569C8476860C047824668B9314B99
:10CE10003149009340F297120320304CA0476A68D2
:10CE20002F48304953468847FEE7012000FA07F7AC
:10CE30003846C847A860C047804668B9254B264990
:10CE4000009340F299120320244CA047AA6824487A
:10CE5000244943468847FEE76B680BB1AB682BB9A2
:10CE6000214B009340F29B121A4B6CE7A37A012BE3
:10CE70004AD12868204BDFF88C800421984700268F
:10CE8000BE4201D1002378E70023042202A92868CA
:10CE9000C0479DF809306A6899089DF80830DB089A
:10CEA00043EA41139DF80A10C90843EAC12322F856
:10CEB0001630AB689DF80B209A550136E0E700BFAD
:10CEC000B5E500007C00020059630100E9E40000C0
:10CED00080000200970102007BFF010031E90000A1
:10CEE00002EE01009D170000AB00020061F000009F
:10CEF0007975000085C8000097E4000075EA00001D
:10CF00009517000061E40000636899680020B8424A
:10CF100001F10401B6D011F8033C6A689E0811F8CB
:10CF2000043CDB0843EA461311F8026CF60843EAB6
:10CF3000C62322F81030AB6811F8012C1A540130C6
:10CF4000E5E7A0F10B03032B9CD9054B21463046A6
:10CF50009847044B009340F2D312034BABE600BF5B
:10CF600085C80000D4000200970102002DE9F843B3
:10CF70000B78DFF84480DFF844906FF347130B70B1
:10CF800007460C4B0C480E4698470024054615B939
:10CF90002046BDE8F8832C6834B13246394628462D
:10CFA000A04701280446F3D029464046C847054615
:10CFB000EDE700BFF1E6000054860020FDE600002A
:10CFC0002DE9F047224B0281044608460F46984758
:10CFD00000230128A072E3611DD11E4B38469847FB
:10CFE0001D4B013098471D4B6060394698471C48DF
:10CFF0001C4BDFF86C90DFF874A0984700260546BC
:10D0000004F10C084DB91EB9174B20212046984752
:10D010003046BDE8F0876760E9E72B689BB16A6836
:10D020008AB14246394628469847012806460AD121
:10D030000023A361236125606B6821462846984739
:10D0400001280646E4D029464846D0470546D9E798
:10D05000117800007D63010075EA00006D63010036
:10D0600054860020F1E6000061F00000FDE60000BB
:10D0700073B50568AC684CB1069ECDE90036134621
:10D080000A4601462846A04702B070BD2046FBE78D
:10D0900010B50446006858B1C3680BB121469847E3
:10D0A000A37A012B04D1034B606898470023636087
:10D0B00010BD00BF2DEB000073B50E4B0E48984716
:10D0C0000E4B04469847054660B90D4B0D49009339
:10D0D000C92203200C4EB0470C480D4922462B466E
:10D0E0008847FEE71CB10B4B10212046984720468D
:10D0F00002B070BD61E60000548600209517000064
:10D10000B40102007BFF010031E9000002EE0100E2
:10D110009D17000061F0000037B5154B1548102130
:10D120009847154B98470446B8B9144A0092022014
:10D130004722134B1349144DA847144A20469047E1
:10D1400098B90F4B0F49009348220320A847104875
:10D150001049002200238847FEE70F4B03600F4B66
:10D1600043600F4B83600F4BC36003B030BD00BF03
:10D170004DE6000054860020B9D00000FD000200FA
:10D18000CA0102007BFF010031E900009517000091
:10D1900002EE01009D170000A5C7000081CC000031
:10D1A000B9C8000085C800004368184710B4046877
:10D1B000A4465DF8044B60471FB51346044C0A466D
:10D1C00001A9A04708B1BDF8040004B010BD00BF1C
:10D1D000ADD1000003780A78934209BF4B78981AC2
:10D1E0004078C01A704703880A88934209BF4B8869
:10D1F000981A4088C01A7047531E10B5072B20D8C4
:10D20000DFE803F02404191B1F1F1F1D0323CC0894
:10D2100001F007010A44072A015D5BB218D92044D6
:10D22000C2F11002407800EB012080B240FA02F215
:10D230001340D8B210BD0723E9E70F23E7E7FF2328
:10D24000E5E701239340013BDBB2E0E71346DEE76D
:10D25000C2F1080241FA02F00340EAE7032B30B5BD
:10D2600004D1072A9CBF0B4B9A5C042301F00705ED
:10D27000C1F3CF04C5F108054FF0FF31ED1A01FAF3
:10D2800003F363F0FF03015DAB400B40AA401A4378
:10D29000025530BD170202002DE9F74F394CDFF877
:10D2A000E8A0D4F8009027794318804600934FF007
:10D2B000020B009B434502D103B0BDE8F08F6379B8
:10D2C000A3B9A66801933A4631464846D047054679
:10D2D00036B1227B019B824202BF637301236371DB
:10D2E0003E442573A66008F8015BE2E7012B31D1CB
:10D2F000A6681A4631464846D047637B0133DBB205
:10D30000711C01286373A16018D10B2B257BEAD116
:10D3100006224846D04707366073A66010B184F8ED
:10D3200005B0E0E7019031463A464846D0473E44D2
:10D33000019B20730546A6606371D4E73A464846D0
:10D340000191D0470199207339440546A1604FF0FF
:10D350000003F1E7022B12D1667B257B013EF6B27A
:10D360006673002EBFD1A16801913A464846D04766
:10D370000199207339440546A1606671B3E7002521
:10D38000B1E700BFD4850020F9D1000000880B88E8
:10D39000C01A7047F0B50C4685B021B10569AB697C
:10D3A000994247D1EC69204605B0F0BDAA6807FB59
:10D3B00003F6911992598888A21A8242039203F1C6
:10D3C000010339D88B7C2BB9C8881044C5E90640C5
:10D3D0000446E8E7012B04D1CB68985CCB8818445D
:10D3E000F4E7022B11D119480A8A00908968184F76
:10D3F00003A8B84708B90020E8E7AB681E44B36843
:10D40000C31AF08800EB5300E0E7032BF3D10F4B76
:10D410000A8A009389680E4F022303A8B8470028A0
:10D42000E9D0AB681E44B368C01A4008F368185CC2
:10D43000F388D4E7002314276A8A99B2C2F3090259
:10D440008A42B3D8AC610024EC61ACE78DD3000014
:10D45000ED0201002DE9F04F2DED028B0929684BFB
:10D4600005698BB008BF20219847074628B90020DE
:10D470000BB0BDEC028BBDE8F08F2B7DD5F804908E
:10D480009B0709EBC00809D1B8F1000FEFD059F89C
:10D4900030302868C3F313031844E9E798F80440D0
:10D4A00098F8051014FB01F4002CE0D0EB7CC3F3DA
:10D4B0008303013B032B05D8DFE803F002505353ED
:10D4C0000734E4084F4E504B30699847A0424BD385
:10D4D00059F837202B68ED7C98F80470C2F31302DA
:10D4E00013443269336008EE102A98F80520079239
:10D4F000C5F38302032A4FF0000B1146327108BFB7
:10D50000042186F805B0C6F808B086F80CB086F895
:10D510000DB038463D4E03920491B047044638465C
:10D52000B0473B4B0646394620469847B946A04689
:10D5300007EB040AD04531D1049B17FB03F3069394
:10D540009A464FF00108079B434532DC2046314C98
:10D55000A0473046A0472B4B186989E70334A4083D
:10D56000B0E701346408ADE721462B4B306998479A
:10D570002A4B30619847044660B9294B29490093EA
:10D5800072220320284DA84732692848284923469B
:10D590008847FEE73369002B9AD168E7039B18F8A8
:10D5A000012B244D594618EE100AA847049B9B44B2
:10D5B000C0E7174B494630469847631E0593F31959
:10D5C000B34608935146089B9B4506D1069B08F13C
:10D5D00001089A440FFA88F8B5E705981BF8012B63
:10D5E00010F8013F05905A400270039B114D0991BC
:10D5F00018EE100AA847049B09991944E3E700BFF5
:10D6000095D30000D485002095EB0000FDEE0000CE
:10D6100099D20000B1EB00005DEE0000951700000C
:10D620001F020200DF01020031E9000002EE0100EA
:10D630009D1700005DD20000092A2DE9FF47DFF8A1
:10D640003CA107690C46114608BF20218046994637
:10D650000CBF01260026D0470546002800F0868032
:10D66000FB683BBB002378683A8A00EBC50553434F
:10D670006A88C2F30B111B110A460EB10AB252009E
:10D68000083313441B0923806B79A3802B796380B3
:10D6900095F90620E28095F907202281FA7CC2F3F1
:10D6A0008302A272002E63D05B006380304604B018
:10D6B000BDE8F08749464046D0470028D2D0D8F888
:10D6C0001030D3F80C80DB7C5B063AD498F80B3032
:10D6D00013F003031BD1D8F80090D8F80820254B8D
:10D6E000009305EB0020ADF80C000223DFF890A0BA
:10D6F00022F07F42494603A8D04703460028B2D013
:10D70000A0EB09035B08D8F80420D356ABE7012B44
:10D71000A8D1D8F80090D8F80820174B009305EB53
:10D72000002003900423DFF858A022F07F424946EE
:10D7300003A8D0470346002895D0A0EB09031B0996
:10D74000E1E7D8F804305A5D002A8BD0D8F80830C9
:10D75000195C002986D0D8F8003098F80D00013AFD
:10D760000B4400FB023313F9013C7CE706469DE7BE
:10D7700001269BE7D5D10000E7D1000095D300003A
:10D78000ED02010010B5044C206918B1034B984715
:10D790000023236110BD00BFD48500202DEB0000C5
:10D7A00010B50D4B2C21044698470C4B0022C4E9C0
:10D7B00000322389E26023F47F6323F00F0343F4F4
:10D7C000027343F0010323814FF4FC63C4E9082290
:10D7D0002385626110BD00BF61F00000E00110010F
:10D7E000F8B504460D4617461E462421034B9847BC
:10D7F000C4E90057C4E90256F8BD00BF61F000005B
:10D800002DE9F3413B4B3C4E05463C4898470446C6
:10D8100098B9B04720B10024204602B0BDE8F0819D
:10D82000374B384900937C220320374CA0473748B8
:10D830003749002200238847FEE7364B4FF4B87182
:10D8400098472946344B354D2C2220469847344B77
:10D850004C2104F1300098470023C4F86C312B6848
:10D8600003B92C60234603221E212E48DFF8CC800A
:10D870002F682C60C047E062B047064660B9204B75
:10D88000204900938D2203201F4DA847E26A1F48BC
:10D890001F4933468847FEE7E36A002BBBD0B4F844
:10D8A0006831214E6FF309030021A4F86831C4F8F0
:10D8B0006C110846B0470021E0630846B0470021DC
:10D8C00020640846B047194E60640021206CB047C0
:10D8D000606C0021B047206C154E0021B047606C91
:10D8E0000021B047E06B134B9847E06A124B2F6062
:10D8F000984791E761E60000951700000C8600202C
:10D90000133F0200E03E020031E9000002EE010098
:10D910009D17000061F0000079EC0000E885002010
:10D920004DE60000E94F0000C5300000792E0000F0
:10D930000D1E0000392700009DFC00002DFC00009A
:10D94000014B1868704700BFE885002010B9074BED
:10D95000186838B1037A9B0754BFB0F90000B0F9DA
:10D96000020070474FF4F070704700BFE885002058
:10D9700010B9074B186838B1037A9B0754BFB0F948
:10D980000200B0F9000070474FF48870704700BF84
:10D99000E885002010B9044B186818B10089C0F35D
:10D9A0008900704782207047E885002008B501464D
:10D9B00010B90F4B196899B10E4B084698470246AB
:10D9C0000D4B084698470A235A43B2FBF0F01D2836
:10D9D00009D9312809D9462834BF0220032008BDBF
:10D9E0004FF4F072ECE70020F9E70120F7E700BF01
:10D9F000E88500204DD9000095D900004368002239
:10DA00009A61DA61704700000146034809B9034B87
:10DA10001847034B184700BF0C860020F1E60000B2
:10DA2000FDE60000406870474368186818B1586800
:10DA3000003818BF0120704708B5074B02469847C9
:10DA400040B150881388526813FB00F3D0681B1A4A
:10DA50005842584108BD00BF29DA0000014603487A
:10DA600009B9034B1847034B184700BF188600201D
:10DA7000F1E60000FDE60000034B00221A705A6830
:10DA800010445860704700BFEC850020034B586875
:10DA9000012119701A78002AFBD07047EC8500200C
:10DAA00010B5024B04469847001B10BD8DDA0000EC
:10DAB000D1E9083083421CBF800290FBF3F0D1E92A
:10DAC000062308BF4FF480609B1A584302EBA02046
:10DAD00000B2704710B5074C074801232370074B6D
:10DAE0009847074B014618B96068BDE810401847D1
:10DAF0000421F9E7F48500203C860020F1E60000CF
:10DB0000C9FB00002DE9F0474F48504D4E4C504E98
:10DB100090B0A847A0B94F4E4F4BB068DFF82881AE
:10DB2000DFF82C91DFF848A1984707464648A847F8
:10DB300004467CB9494B9847B06010B0BDE8F08707
:10DB400090F83C306FF3410380F83C3001462046AA
:10DB5000B047DFE70023337094F83C309A076ED467
:10DB600043F0020384F83C30636A002B05DCFB427F
:10DB700003D4A3680BB120469847636A3B44002B4B
:10DB800063622DDB226A2046934250F8103FC8BFE3
:10DB90006262214653B39847636813B101B22068AB
:10DBA0009847D4E908329A421ADB94F83C30E16A8B
:10DBB00013F0010323D1A28EDAB900293CD140220F
:10DBC00021466846D0472146254B40469847254B7D
:10DBD00020469847244B9847039B0BB168469847CB
:10DBE000337863B34046A8470446A2E71F4B9847E3
:10DBF000D2E74FF6FF70824204D0013AA286A28E8D
:10DC0000002ADAD0226B524262620029E8D013B9AE
:10DC1000A26A5242626283F0010294F83C3062F3DD
:10DC20000003D4E9060284F83C30DB0758BFA16B3F
:10DC30002162C4E90620D3E7002BE3D0BFE72146E9
:10DC40004046C847D0E700BF3C860020F1E6000010
:10DC5000FDE60000F4850020A1DA00008DDA000066
:10DC6000B5E700002DEB0000D5DA0000B1DA0000C6
:10DC700079EC000038B5402109480A4B0A4C0B4D9D
:10DC800098470B4B98470023A06004221E210948A7
:10DC9000A847094B606098470023237038BD00BF38
:10DCA0003C8600204DE60000F48500202DFC00009D
:10DCB0008DDA000005DB0000D5DA000010B50B4B53
:10DCC0000446402198474FF4FA73236200216423ED
:10DCD000C4E90613064B23610123A38694F836306A
:10DCE00043F0010384F8363010BD00BF61F000003E
:10DCF000B1DA00002DE9F84F144BDFF85490DFF84B
:10DD00005CA0DFF85CB0064611480D4698474FF01E
:10DD10000008044614B94046BDE8F88F214648463D
:10DD2000D0472368B34207460DD16368AB4200D0A9
:10DD30004DB921464846D847064B20469847064BE2
:10DD400098474FF001083C46E4E700BFF1E60000C9
:10DD50003C8600202DEB0000D5DA0000FDE6000037
:10DD6000B5E7000073B54168054611B100681D4B69
:10DD700098471D481D4B984720B11D4B98471D4B98
:10DD8000013898601C4B184898471C4B044698472C
:10DD9000064660B91A4B1B4900936A2203201A4DAC
:10DDA000A8471A481A49224633468847FEE7B4B1C5
:10DDB0002B6AAB634022174B29462046984794F8BC
:10DDC0003630DB0706D5636823B1206810B1B4F99B
:10DDD00018109847104B02B0BDE87040184702B0C9
:10DDE00070BD00BFF5DC00003C86002019E9000092
:10DDF0008DDA0000F485002061E600009517000030
:10DE0000583F0200283F020031E9000002EE010005
:10DE10009D17000079EC0000D5DA0000F8B5094B39
:10DE2000094E0A4F044608480D46984700B9F8BD08
:10DE30000368A34202D14368AB42F8D001463046A2
:10DE4000B847F3E7F1E600003C860020FDE600005D
:10DE5000891A0029B8BF49424FF47A725143B1FB85
:10DE6000F0F0012838BF01204FF6FF73984228BF19
:10DE7000184680B2704730B5B0F90430B0F90050A0
:10DE800040885B1B03EBD373121A5C10491BC3F36E
:10DE90004F03C91AD31A13FB03F3644311FB013177
:10DEA0008C42B4BF0020012030BD438801391944A1
:10DEB000C1807047B0F90030B0F90420D21AB0F92F
:10DEC0000630B0F90200181A013002FB000070475A
:10DED000B1F9003070B5B2F90050B1F90240B1F9B2
:10DEE0000460B1F906109D42B8BF1D46B2F9023078
:10DEF0000580A342B8BF2346B2F90440B2F9062018
:10DF00004380B442A8BF34468A42A8BF0A46A5420D
:10DF10008480C28004DC9342CCBF0020012070BD0D
:10DF20000020FCE7B2F9003010B5B1F90040A3427F
:10DF3000A8BF23460380B1F90240B2F90230A342E0
:10DF4000A8BF23464380B1F90440B2F90430A3428C
:10DF5000B8BF23468380B2F90630B1F90620934258
:10DF6000B8BF1346C38010BD2DE9F04FB1F9009042
:10DF7000B0F90040A14587B08846C0F28B80B0F967
:10DF800004300093994500F38580B1F902A0B0F9FF
:10DF900002B0DA457EDBB0F906309A457ADC002A19
:10DFA00003DC012007B0BDE8F08FBDF8000002904F
:10DFB000A6B20130801B9FB21FFA8BFCADF8104057
:10DFC0007D1CC0F3C03404FA80F0A5EB0C04C4F34C
:10DFD000C03505FA84F56D104410AC42A8BF2C463C
:10DFE000A242A8BF224616FA82F695B21CFA82F225
:10DFF000039314B293B2B6B2002204A80193ADF811
:10E000001460ADF812B0ADF81640FFF7ADFF039BFA
:10E01000024638B12E44ADF81460019B1D44ADF8A2
:10E02000165011E07F1BBFB2414604A8ADF8127034
:10E03000ADF81630FFF798FF024658B12E44ADF800
:10E0400014607D1BADF81250134B5246494604A88C
:10E050009847A7E7029B5E1BB6B2009BADF8106025
:10E06000414604A8ADF81430FFF77EFF024618B110
:10E07000761BADF81060E4E7414604A8ADF812B095
:10E08000ADF81640FFF770FF00288AD0761BADF878
:10E090001060C2E7002085E777DE0000B0F90020BD
:10E0A000B1F904309A4214DCB0F90420B1F900301F
:10E0B0009A420EDBB0F90220B1F906309A4208DC30
:10E0C000B0F90600B1F902309842B4BF0020012037
:10E0D00070470020704700002DE9FF41B0F9007043
:10E0E000B1F90030BB4205460C4624DCB0F9021001
:10E0F000B4F9023099421EDBB0F90410B4F90430CF
:10E10000994218DCB0F90630B4F906008342CCBF5E
:10E110000020012062B16B88164E019203A92046AF
:10E12000ADF80C70ADF80E30B047019A28B9002058
:10E1300004B0BDE8F0810020ECE7B5F90480ADF84B
:10E140000C8003A920460192B0470028EFD0EB884D
:10E15000019AADF80C7003A92046ADF80E30B04717
:10E160000028E4D0019AADF80C8003A92046B047FE
:10E17000DEE700BF69DF0000F0B544880588142A97
:10E180003FD8DFE812F015003B0045005A0061005F
:10E1900069007C00830085008C009300A600AD0020
:10E1A000B300C600CD00D200D700DC00DF00E200E3
:10E1B00082880F880132521BC2F3C03606FA82F6FB
:10E1C0008A880132D21BC2F3C03707FA82F252109A
:10E1D000C2EB66021A80C2880132121BC2F3C03041
:10E1E00000FA82F0CA8849880132521AC2F3C0315B
:10E1F00001FA82F25210C2EB600201E000221A80A2
:10E200005A801A8815445A881D8014445C80F0BDD9
:10E2100082880132521BC2F3C03000FA82F08A8831
:10E2200009880132521AC2F3C03101FA82F2521047
:10E23000C2EB60021A800022E2E70A888988521A3B
:10E2400081880A44521BF5E700221A804A88C9884F
:10E25000521AC1880A4447E082880F880132521B53
:10E26000C2F3C03606FA82F68A880132D21BC2F3A4
:10E27000C03707FA82F25210C2EB6602E5E78E88D9
:10E280000A88921B86883244521BDEE70022A1E7EF
:10E290008E880A88921B86883244521B9AE7002295
:10E2A0001A804A88C988013A521AA9E782880E88DA
:10E2B0000132521BC2F3C03000FA82F08A88013268
:10E2C000921BC2F3C03606FA82F25210C2EB600211
:10E2D000E6E70A888E888088921B0244521BDFE79B
:10E2E00000221A80C2880132121B89E7828801321B
:10E2F000521BC2F3C03606FA82F68A8809880132B8
:10E30000521AC2F3C03101FA82F25210C2EB660215
:10E31000E7E70A888988521A81880A44521BE0E795
:10E320000A888988013A521A84E70A888E88013A55
:10E33000921B4FE70A888E88013A921B85E78288F4
:10E3400001327FE782880132A7E7828801329BE7AA
:10E35000830710B58CB21CBF20F8021B02F1FF32FC
:10E3600004EB0443102A014600F1200004D801EB1D
:10E37000420291420AD110BD40E9083340E9063318
:10E3800040E9043340E90233103AEBE721F8024B4D
:10E39000EFE730B5C0F34513C1F1FF056B433F24F0
:10E3A00014FB013348F281046343C1EB4112C3F310
:10E3B000C55100F01F0305FB0323C0F3C4206343D2
:10E3C00005FB00206043C3F3C45343EA4113C00D6F
:10E3D00043EAC02030BDC1F1FF01C0F3451310B5C1
:10E3E0004B4348F281046343DA0D00F01F034B43B3
:10E3F000C0F3C420634348436043DB0D43EA421348
:10E40000C00D43EAC02010BD431C184613F8012B71
:10E410002AB13A2AF9D05C2AF7D02F2AF5D07047D2
:10E420000148024B44211847248600204DE6000095
:10E4300038B50446406860B1036963B12168984704
:10E44000064B0546206898470023C4E90033284658
:10E4500038BD0B25FBE70925F9E700BF2DEB0000D0
:10E460007FB51C460BB10023236045687DB1AE69C2
:10E470007EB10023039303AB009313460A46016861
:10E480002846B0470CB1039B236004B070BD0B203D
:10E49000FBE70920F9E7436810B40A463BB11C6A60
:10E4A0004CB10168184623465DF8044B18470B2011
:10E4B0005DF8044B70470920FAE7000070B5074B80
:10E4C000074D084E04460648984700B970BD0378CA
:10E4D000A342FBD001462846B047F6E7F1E600002C
:10E4E00024860020FDE6000000232DE9F341C0E969
:10E4F0000033044617460E46002943D00878234BC4
:10E500009847606028B920600325284602B0BDE81E
:10E51000F08183682BB1984718B9C4E90000012540
:10E52000F3E7636858881A4B98471A4B206098475E
:10E53000054660B9184B194900936F220320184E05
:10E54000B0472268174818492B468847FEE72168DC
:10E5500011B961600A25D8E7D4F80480D8F80C50C6
:10E5600095B1124B304698473B4602464046A84775
:10E5700005460028C9D00E4B206898470023C4E9FF
:10E580000033C2E70B25C0E70925BEE7BDE4000064
:10E5900075EA000095170000B13F0200703F0200CD
:10E5A00031E9000002EE01009D17000009E40000BF
:10E5B0002DEB000010B5094B0446984708B90848F0
:10E5C00004E0235C2E2B02D10130204410BD2F2B00
:10E5D000F5D05C2BF3D00138F0E700BF7D6301007C
:10E5E0001CF801000139031D11F8012F00F8012B5F
:10E5F0009842F9D17047000007B5019229B100682F
:10E6000008442AB1044B01A9984703B05DF804FB04
:10E61000024B04219847F8E7E5E5000061F00000AF
:10E6200007B5019231B10068043008442AB1054BA6
:10E6300001A9984703B05DF804FB034B04219847F8
:10E64000F8E700BFE5E5000061F000000023C0E945
:10E6500001338B071CBF21F00301043101607047B7
:10E6600070B5044600680D4B08309847054690B1D8
:10E670000146002220460A4EB04729466268094BEF
:10E6800020469847616811B12A462046B047A368E2
:10E69000656003B9A560284670BD00BF75EA00003B
:10E6A000F9E5000021E6000070B5044600680D4B56
:10E6B00008309847054690B10146002220460A4E90
:10E6C000B0472946A268094B20469847A16811B176
:10E6D0002A462046B0476368A56003B965602846AE
:10E6E00070BD00BF75EA000021E60000F9E50000FA
:10E6F00000B14068704700B18068704707B50023DB
:10E70000019328B103680433194401A8024B9847C8
:10E71000019803B05DF804FBE5E5000007B50023B0
:10E72000019320B1036801A81944034B984701984D
:10E7300003B05DF804FB00BFE5E500002DE9F04102
:10E740000E46044640B349B34368994203D1BDE83D
:10E75000F041134B18470068124B083098470546A4
:10E76000B8B1114BDFF848803146204698472A4619
:10E77000074601462046C0473A4629460B4F2046E9
:10E78000B8472A4631462046B847324629462046F1
:10E79000C0472846BDE8F0810546FAE70D46F8E790
:10E7A00061E6000075EA00001DE70000F9E50000E1
:10E7B00021E6000070B50D460446F8B14368994261
:10E7C0000CD12946174B204698470146606008B98E
:10E7D000A06070BD0022144B20460CE08368994273
:10E7E0000ED1124B98470146A06008B96060F0E76F
:10E7F0000F4B00222046BDE8704018470029E0D0AA
:10E8000029460A4B2046984729460646054B20468E
:10E810009847314602460546054B20469847324602
:10E820002946D8E7FDE60000F9E500001DE70000F5
:10E8300021E600002DE9F0410C461E461146164B1C
:10E84000DFF85C80154F1546984796B1002229469F
:10E850002046C047294662682046B847616811B122
:10E860002A462046C047A368656003B9A560BDE895
:10E87000F081A26829462046C047294632462046F4
:10E88000B847A16811B12A462046B8476368A56019
:10E89000002BECD16560EAE7B5E7000021E6000057
:10E8A000F9E5000091422DE9F84304460D4617466C
:10E8B00022D01AB3144B114698470646AE421BD0DD
:10E8C000124BDFF84C80DFF84C90294620469847E1
:10E8D0002A4631462046C047324629462046C84788
:10E8E0002A4639462046C8473A4629462046C04768
:10E8F00007B9A56006B96560BDE8F88308B1866808
:10E90000DCE70646DAE700BF1DE70000B5E70000D8
:10E9100021E60000F9E5000030B1436833B98068B2
:10E92000B0FA80F04009704701207047002070471E
:10E930002DE9F0431F46431EDBB2042BC5B004464D
:10E940000D46164617D84DAB0DF11009DFF8308093
:10E9500003934C9A4FF480714846C047074BD3F855
:10E960000080B8F1000F06D0CDF800903B4632464B
:10E9700029462046C04745B0BDE8F0838487002083
:10E9800069F800004FF4B47390FBF3F202FB13003C
:10E9900000B20028BCBFC01800B259280E4B02DCE0
:10E9A00033F91000704780B2A0F15A02592A03D8F7
:10E9B000C0F1B40080B2F3E7A0F1B40292B2592AD8
:10E9C00085BFC0F5B47080B233F8120033F8100080
:10E9D000404200B2704700BFCC3F020030B5000299
:10E9E0000023D41804FB04F5854298BF234652083F
:10E9F000F7D11A091B01DBB20A804B8030BD000041
:10EA0000074B1B6850B150F8042B00EB5200021D5D
:10EA100003F580439A4228BF00207047184670478C
:10EA2000888700208B0718BF21F00301026818BFF8
:10EA3000043110B50C1DB4EB520FC2F35E030BD0C2
:10EA40008B4204D0043B42185B1A5B00536003689E
:10EA500061F35F03036010BD1946F8E7034A044BF6
:10EA6000136047F6F8721A60704700BF888700206D
:10EA70009487002037B50146E0B1820718BF20F027
:10EA80000301124D18BF043100242046A847044654
:10EA900090B10378DB07F8D40368B1EB530FF4D8D7
:10EAA0000B4B9847037843F0010304F8043B2046DE
:10EAB00003B030BD074CFAE7074B00930749084BFA
:10EAC000084DD1220220A847F1E700BF01EA00006B
:10EAD00025EA00008C870020B1400200824002003D
:10EAE0009641020031E9000038B50E4B0E4C196812
:10EAF00001B938BD0846A0470B78DA070FD50146A3
:10EB0000F6E70378DB07FAD40B680568C3F35E0207
:10EB1000043202EB550262F35F030B60A04700284A
:10EB2000EFD1E6E78887002001EA0000164A131DAE
:10EB3000984270B5014610D078B110F8043C6FF3DC
:10EB4000000300F8043C138901339BB20F2B13819F
:10EB500014D80E4C0438A04700B970BD0378DB0709
:10EB6000FBD451F8043C0568C3F35E02043202EBA7
:10EB7000550262F35F0341F8043CECE70023138184
:10EB8000BDE87040024B18478887002001EA00006A
:10EB9000E9EA000040B1054B984204D050F8040C5B
:10EBA000C0F35E0070470020704700BF8C870020D4
:10EBB000164B1A68904213B50BD09A6890420AD14E
:10EBC000012203EBC2039A796FF300029A7102B03B
:10EBD00010BD0022F5E70E4A002352F8334084426C
:10EBE00002EBC30104D18B796FF300038B71EEE765
:10EBF0000133102BF1D1074B00930749074B084C09
:10EC000040F232220320A047E1E700BF4400002089
:10EC100074860020CA40020082400200A341020024
:10EC200031E90000114B9A796FF300022DE9F041B0
:10EC30009A719A7B0E4CDFF83C806FF3000200253E
:10EC40009A7327462E46206840B1C04707EBC5039C
:10EC500026609A7966F300029A71A6800135102D1C
:10EC600004F10804EFD1BDE8F08100BF44000020AA
:10EC7000748600202DEB000070B500F0030501F054
:10EC80000306B54204460B4640F09880002D40F044
:10EC9000A88005462B46202A1C4601F1200503F1D9
:10ECA000200300F2B080042A0E4640F29F8051F803
:10ECB000043B44F8043B043AF5E713F8201C04F83D
:10ECC000201C13F81F1C04F81F1C13F81E1C04F84A
:10ECD0001E1C13F81D1C04F81D1C13F81C1C04F842
:10ECE0001C1C13F81B1C04F81B1C13F81A1C04F83A
:10ECF0001A1C13F8191C04F8191C13F8181C04F832
:10ED0000181C13F8171C04F8171C13F8161C04F829
:10ED1000161C13F8151C04F8151C13F8141C04F821
:10ED2000141C13F8131C04F8131C13F8121C04F819
:10ED3000121C13F8111C04F8111C13F8101C04F811
:10ED4000101C13F80F1C04F80F1C13F80E1C04F809
:10ED50000E1C13F80D1C04F80D1C13F80C1C04F801
:10ED60000C1C13F80B1C04F80B1C13F80A1C04F8F9
:10ED70000A1C13F8091C04F8091C13F8081C04F8F1
:10ED8000081C13F8071C04F8071C13F8061C04F8E9
:10ED9000061C13F8051C04F8051C13F8041C04F8E1
:10EDA000041C13F8031C04F8031C13F8021C04F8D9
:10EDB000021C13F8011C04F8011C203A202A1D46ED
:10EDC000214603F1200304F120043FF676AF6B1EC9
:10EDD0000A44914200D170BD13F8014F01F8014B74
:10EDE000F7E7C5F1040505441E4612B9731E224417
:10EDF00030E013F8011B04F8011BAC42194602F184
:10EE0000FF32F1D146E755F8201C43F8201C55F895
:10EE10001C1C43F81C1C55F8181C43F8181C55F80A
:10EE2000141C43F8141C55F8101C43F8101C55F81A
:10EE30000C1C43F80C1C55F8081C43F8081C55F82A
:10EE4000041C43F8041C203A294624E713F8011F48
:10EE500004F8011B9442F9D1BDE700008B07F7B518
:10EE60000D4618BF21F00305044618BF043528B12C
:10EE700010F8043C13F0010F08BF0024164B204685
:10EE800098478542074604D005D2144B2946201FD7
:10EE9000984726460DE0124B28469847064658B933
:10EEA000104B00931049114B114C40F23F120220BD
:10EEB000A047304603B0F0BD002CFAD0002FF8D0A8
:10EEC000BD422A460B4B28BF3A46214698470A4B7B
:10EED00020469847EDE700BF95EB000025EA0000CB
:10EEE00075EA0000B140020082400200B741020012
:10EEF00031E9000079EC00002DEB0000F7B590B18E
:10EF0000102812D8364A937913F0010303D0937B6B
:10EF1000DE070AD4012302EBC300817941F001012D
:10EF2000817152F8330003B0F0BD2E4C00234FF036
:10EF3000FF32271D04EBC306B5792946ED0713D42C
:10EF400037F8335085420FD305D141F0010154F811
:10EF50003300B171E7E7561C01D15AB204E004EB6B
:10EF6000C2018988A942F8D80133102BE2D1551C7F
:10EF700008D004EBC20154F832008B7943F001034E
:10EF80008B71D0E7002504EBC50399790A46C907C0
:10EF900017D442F0010298809A710146124B54F83E
:10EFA0003500984744F8350040B9104B009310499C
:10EFB000104B114E4FF404720320B04754F8350043
:10EFC000B1E70135102DDED10C4B00930320094B26
:10EFD0000749094C40F21622A0470020A3E700BFD2
:10EFE00044000020748600205DEE0000F640020020
:10EFF00082400200C641020031E90000584102008F
:10F0000010F0030310B409D0C3F1040303442AB180
:10F0100000F8011B984202F1FF32F8D101EB012404
:10F0200004EB014404EB01640346202A184603F173
:10F03000200305D8042A0DD8084B5DF8044B184767
:10F0400043E9084443E9064443E9044443E90244EC
:10F05000203AEAE740F8044B043AEBE74963010041
:10F0600010F003030DD1034600222029184603F1B6
:10F07000200316D80023042908D940F8043B04399A
:10F08000F9E7C3F104030344002219B90A460A4B05
:10F090000021184700F8012B834201F1FF31F4D120
:10F0A000E1E743E9082243E9062243E9042243E970
:10F0B00002222039D9E700BF4963010010F00303A1
:10F0C0000FD103464FF0FF322029184603F12003E9
:10F0D00017D84FF0FF33042908D940F8043B04390E
:10F0E000F9E7C3F104030344FF2219B90A460A4BA6
:10F0F000FF21184700F8012B834201F1FF31F4D1C1
:10F10000DFE743E9082243E9062243E9042243E911
:10F1100002222039D8E700BF496301009A4238BF74
:10F120008854704770472DE9F74F1746DDE91162A3
:10F1300012F0020A8046DDE90C54DDE90F0C9DF85F
:10F1400038E01FD102F001094EB1B9F1000F06D02D
:10F15000BEF1000F02D112F00C0F00D0013E4FF0B3
:10F16000300B04E0202C04D005F804B00134A44591
:10F17000F8D84FF0300BB9F1000F03D0A64201D9F7
:10F18000202C37D112F0100F19D012F4806F36D125
:10F19000ACB3644501D0B44231D1B4F1010C2DD0EF
:10F1A00010286AD1023C900631D41F2C0FD8782049
:10F1B000285501341F2C0AD8302028550134202C22
:10F1C00005D0BEF1000F26D02D202855013492071E
:10F1D0003BD03A4625441444A2423AD1BAF1000F3A
:10F1E00004D0D51BB54205EB07043DD3204603B040
:10F1F000BDE8F08F05F804B00134BCE76446102880
:10F20000D1D00228D6D11F2CE1D86220D0E71F2C04
:10F21000DDD85820CCE7500701D52B20D5E71007C3
:10F22000D5D52020D1E72020CDE90013C047DDE966
:10F23000001309F101094E450BEB0902F3D8321B0B
:10F24000B44288BF00223A44C4E7A146A7EB040BAE
:10F25000F1E702F1010915F8010DCDE90013C047EE
:10F26000DDE900134A46B7E72246202001930091CA
:10F270000135C047DDE90013B4E70228644699D19F
:10F28000C3E700002DE9F04391B0189D1A9E1D9F21
:10F290000DB927F010077C0500D515B317F0200F26
:10F2A00014BF4FF0410E4FF0610EAC460DF1200837
:10F2B0000025AEF10A0EBCFBF6F906FB19C95FFA90
:10F2C00089F4B9F1090F94BF30347444E4B2B44501
:10F2D00008F8014BBCFBF6F405F1010501D3202D24
:10F2E00010D11C9C05941B9C0697CDE903649DF8E6
:10F2F0006440CDE9015408AC0094034CA04711B020
:10F30000BDE8F083A446D6E727F100002DE9F04FD1
:10F310002DED048B93B0DDE920659A4656EA05038E
:10F3200002BF289B23F010032893289B5B05DDE98F
:10F3300024B908EE100A08EE901A09EE102A02D538
:10F3400056EA05033FD0289B13F0200F14BF41233A
:10F3500061230A3B0DF12808002409931B4F5A46EC
:10F360004B4630462946B847D2B2092A8ABF099B84
:10F370003032D2185E45D2B275EB090308F8012B82
:10F3800004F1010401D3202C1AD1289B0693279B5A
:10F390000593269BCDE903B39DF88830CDE9014361
:10F3A0000AAB009319EE102A18EE901A18EE100A04
:10F3B000074C5346A04713B0BDEC048BBDE8F08F5B
:10F3C00006460D46CAE70024DFE700BF8D5F010057
:10F3D00027F100002DE9F04F91B01F460A92AC4B87
:10F3E000AC4A8946011E14BF92469A4600240A9BE5
:10F3F000187858B94C452CBF09F1FF3222464B46CC
:10F400000020D047204611B0BDE8F08F0A9B252888
:10F4100003F101030A9306D02246651C4B460B916B
:10F42000D0472C4617E2002506E02D2B16D0302BB6
:10F430000CD145F001050A920A9A12F8013B2B2BD8
:10F440000FD0F2D8202B0FD0232B10D0A3F13000F7
:10F4500009282CD84FF000080A2010E045F00205DA
:10F46000E9E745F00405E6E745F00805E3E745F080
:10F470001005E0E700FB0838A8F130080A920A9A64
:10F4800012F8013BA3F13006092EF3D90A9B1B7831
:10F490002E2B4CD10A9B581C5B78A3F13002092A11
:10F4A00045F480653AD800264FF00A0E13E02A2B67
:10F4B0000AD157F8048B0A92B8F1000FBCBF45F08F
:10F4C0000205C8F10008E1E74FF00008DEE70EFB97
:10F4D0000636303E1046024612F8013BA3F1300CCE
:10F4E000BCF1090FF3D9024612F8013B6C2B28D06E
:10F4F00020D8682B2CD06A2B33D00246134613F841
:10F50000010B0A93782887D861282DD8252883D025
:10F51000582881D145F0200510226BE02A2B07D115
:10F5200057F8046B0A9826EAE6760230DBE70A9879
:10F530000026D8E7742B01D07A2BDED145F48075F4
:10F54000DCE743786C2BF9D145F44075821CD5E794
:10F550004378682B02D045F08005CFE745F0C00521
:10F56000F4E745F40075C9E7A0F16203162B3FF6F6
:10F5700053AF01A252F823F0D5F50000F7F60000D2
:10F58000D5F5000019F4000019F4000019F400008A
:10F5900019F40000D5F5000019F4000019F400007A
:10F5A00019F4000019F4000019F40000D5F500006A
:10F5B0002FF8000019F4000019F400006DF70000A6
:10F5C00019F40000D5F5000019F4000019F400004A
:10F5D000D5F5000078289FD06F2800F03E81622882
:10F5E00000F03D81692825F010054FF00A0203D094
:10F5F000642801D025F00C056B0548BF25F00105F6
:10F60000692805F4007301D0642849D1FBB107379C
:10F6100027F00707BB4678685BF8083B0492002296
:10F620000592C20F0028CDE907850696029202DAFC
:10F630005B4260EB4000CDE9003022464B46164C61
:10F640000B915046A0470B9904465F46CFE6EB0569
:10F6500007F1040B12D53B68CDE90485CDE90226FC
:10F66000002B4FEAD3720192B8BF5B42009322464F
:10F670004B460A4C0B915046A047E4E715F0400F6B
:10F680003B6801D0DBB2E7E72F0648BF1BB2E3E7D8
:10F6900025F100001DF100000DF3000085F20000CF
:10F6A00073B1CDE907850023073727F0070B0696CE
:10F6B000049205930293FBE80223CDE90023BCE703
:10F6C000E80507F1040B06D5CDE90485CDE902264E
:10F6D00001933B68CAE715F0400F3B6807D0DBB2E7
:10F6E000CDE902260022CDE904850192BEE7280675
:10F6F00048BF9BB2F4E715F0020523D0012657F866
:10F70000040B0B914B462246C0B2D04704F1010BCB
:10F710000B994DB334465A461EE00B914B462020C0
:10F72000D0470B99A2190136B045F6D8B8F1000FB1
:10F7300008F1FF3308BF002308F101061C4408BF8D
:10F740000226DCE72E46EDE70B914B462020551CA8
:10F75000D0470B9901342A46A045F5D8A8EB0603FB
:10F76000B04538BF00239B445C4640E63B46002E34
:10F7700053F804BB0B9314BF33464FF0FF335B4485
:10F780005F463A780AB1BB4210D115F48063A7EB0B
:10F790000B070C9302D0B74228BF374615F002037F
:10F7A0000D9318D13B1B22460E9308E00137E8E782
:10F7B0000F914B462020551CD0470F992A460E9B8F
:10F7C000D3189845F4D8A8EB0703B84538BF0023F1
:10F7D00001371C441F445D46A4EB0B0B05E01E469D
:10F7E0000E914B462246D0470E990BEB050415F8B7
:10F7F000010B28B10C9B002BF2D0731E002EEED112
:10F800000D9B93B122463D1B06E00C914B462020F8
:10F81000561CD0470C99324653199845F5D8A8EB99
:10F820000703B84538BF00231C440B9FDFE50823BE
:10F83000CDE9036310220023CDE9013245F0210513
:10F84000059557F8043B009322464B46054C0B9117
:10F850005046A04704460B99C9E50822CAE6022291
:10F86000C8E600BF85F2000010B4024CA4465DF863
:10F87000044B6047D5F3000008B50548054B182137
:10F880009847054B00221A7001225A7008BD00BF2C
:10F89000008600204DE60000B4C70020F7B5364BC7
:10F8A000364898470546E0B1344E354C2B7D03F081
:10F8B0000703032B29462ED8324B30489847324B4A
:10F8C00004469847054608BB304B31490093DB227C
:10F8D0000320304EB0473048304922462B468847F7
:10F8E000FEE72F4B25489847274B04469847054687
:10F8F00060B9264B26490093D3220320254EB047FA
:10F900002548264922462B468847FEE7ECB90024C5
:10F91000204603B0F0BD3046A04705460028C5D1BB
:10F92000204B16489847184B044698470028EDD1BD
:10F93000164B17490093E5220320164EB047164890
:10F94000164922462B468847FEE74FF4FA73236098
:10F95000237D154D032262F30203002723754FF028
:10F96000FF3301262361A760104B2E709847E76094
:10F970006060AE70CCE700BFF1E6000000860020BA
:10F98000FDE600003DE7000095170000064202007A
:10F99000D641020031E9000002EE01009D1700008F
:10F9A00061E60000A9E60000B4C700208DDA00007F
:10F9B00070B501460446074B0748084D9847012695
:10F9C000074B2E7020469847064B1B68A34208BF82
:10F9D000EE7070BDB5E7000000860020B4C70020BF
:10F9E0002DEB00007086002038B5124B04464068AD
:10F9F0009847236898421BD30F4B104D984700231C
:10FA0000EB70AB70A368606043B92369002B0CDC1A
:10FA1000236943B90A4B2046984704E0204698479B
:10FA2000EB78002BF1D0012038BD013B2361EFE7DB
:10FA30000020F9E7A1DA00008DDA0000B4C7002049
:10FA4000B1F900002DE9F84FDFF874B19BF80440DC
:10FA5000012034B99BF801208BF804001AB98BF807
:10FA60000420BDE8F88F504DDFF84C91DFF84C8151
:10FA7000A847CBF80800002248468BF803208BF8F3
:10FA80000220C047DFF83CA1484FCAF80000DAF86E
:10FA90000010B9B1464B484698470646DAF80000D0
:10FAA000017D11F0070C0DD0A04203D1CAF800600F
:10FAB0000024ECE7BCF1050F3AD1B8479BF80210DF
:10FAC000002965D03B4CDBF80800A047DBF80C2090
:10FAD0001044CBF80C00DBF81400A047B0F5FA7F17
:10FAE00016D3DBF80C2064214A434FF4FA71B2FBC1
:10FAF000F1F2D2B2642A9ABFC2F16402D2B20022F9
:10FB00008BF810200022CBF80C20A847CBF814006B
:10FB10004FF0FF322848294BCBF818209847264E43
:10FB2000234F0546F5B9DBF818008BF8045098E729
:10FB30003CB194F814C001F007010CF0070C6145CA
:10FB4000BCD9B8470028B9D09BF802100029B9D118
:10FB50009BF803100029B5D1DAF800408BE7CAF80A
:10FB6000006094E72A7D53070DD06868A0472A6893
:10FB7000904238BF101ADBF8182028BF00208242BC
:10FB800088BFCBF8180029463046B8470546C9E774
:10FB90009BF80310002995D19BF800000028DED0C7
:10FBA0008BF800100C4666E78DDA0000E9F90000DA
:10FBB000FDE60000A1DA000000860020F1E600006A
:10FBC000B4C7002070860020F8B5037D03F007035A
:10FBD0008B4204460D4618D00F48104B0E4E104F66
:10FBE0009847024632B1137D03F007039D420DDBB7
:10FBF000A24203D008480B4B214698470A4B0122EA
:10FC00001A70237D65F302032375F8BD1146304653
:10FC1000B8470246E6E700BF00860020F1E6000094
:10FC2000FDE60000A5E80000B4C700202DE9FF4173
:10FC30001E46124B03920F4680469847104B0446CF
:10FC400098470399054668B90E4B0F4900934FF446
:10FC5000837203200D4EB0470D480E4922462B46B5
:10FC60008847FEE734B10C4BC4F808802760204673
:10FC70009847E660204604B0BDE8F0819DF800009A
:10FC8000951700001B420200D641020031E9000036
:10FC900002EE01009D170000C9FB000010B50446EC
:10FCA000034B98472368DB430344636010BD00BFE8
:10FCB0008DDA000090F900200378002A0EDA03F0B4
:10FCC000E002C02A0CD003F0F002E02A0AD003F0D0
:10FCD000F803F02B14BF0020042070470120704768
:10FCE000022070470320704773B50023019301B9C8
:10FCF00001A90A688556835C002D02F1010403DB2B
:10FD000018460C6002B070BD03F0E005C02D10D1A4
:10FD10000C60005D00F0C004802C01D00020F1E7F1
:10FD20009B0103F4F86300F03F00184402320A60BC
:10FD3000E8E703F0F005E02D17D10C60045D04F056
:10FD4000C005802DEAD1951C0D60455D05F0C00011
:10FD50008028E3D1180380B205F03F05A3012844B1
:10FD600003F47C6318440332E1E703F0F805F02D57
:10FD70000C60D3D1045D04F0C005802DCED1951C5C
:10FD80000D60455D05F0C006802EC7D1D61C0E6003
:10FD9000865D06F0C0008028C0D19B04200300F4DB
:10FDA0007C3003F4E0130343A80100F47C6006F008
:10FDB0003F06304418440432B9E700000B68F7B539
:10FDC000013B0D4F0B6006460C46042520683B683E
:10FDD00030449847236848B92BB1013D013B15F0E9
:10FDE000FF052360F2D1002003B0F0BD019301A90B
:10FDF0007B6830469847F7E7540000202DE9F04132
:10FE00000024DFF8288007460D462646AE4202D180
:10FE10002046BDE8F0813819D8F80030984701280D
:10FE200038BF012054FA80F40136EFE75400002077
:10FE3000F7B50024074F019406460D46019BAB42DF
:10FE400002D3204603B0F0BD7B6801A93046984735
:10FE50000134F3E75400002073B50024074E0194E9
:10FE60000546019BEB5C13B9204602B070BD736878
:10FE700001A9284698470134F3E700BF5400002049
:10FE80007F2882B013D9B0F5006F12D2830963F0D6
:10FE90003F0300F03F008DF8043060F07F00002346
:10FEA0008DF805008DF806308DF80730019802B006
:10FEB0007047B0F5803F12D2030B63F01F038DF83B
:10FEC0000430C0F3851300F03F0063F07F0360F05F
:10FED0007F008DF805308DF806000023E4E7B0F5CB
:10FEE000881FE3D2830C63F00F038DF80430C0F356
:10FEF000053363F07F038DF80530C0F3851300F000
:10FF00003F0063F07F0360F07F008DF806308DF8CE
:10FF10000700CBE7030612D5C0F30722030603EB65
:10FF20000243C0F3074203EB022303EB10600423F8
:10FF3000C2B202B9000A013B13F0FF03F8D17047C7
:10FF40002329024617D103781BB90123037001202E
:10FF500004E0012B4FF0000009D110701378012B41
:10FF600004D1202904BF0221117018467047022BCA
:10FF7000F4D11070EBE70020F0E700002DE9F04F1E
:10FF8000884685B017461E460546002400283ED008
:10FF9000002A3ED003948DF80B40002935D09DF8FF
:10FFA0003890DFF87CA009F00109DAF8043003A9E1
:10FFB0002846984783460398DAF80420002128440D
:10FFC00090470246B9F1000F11D1134B59463846FC
:10FFD000984703B2002B14DC039B9845E5D8002C0E
:10FFE00001DDA41B24B2204605B0BDE8F08F0190CE
:10FFF0000A4B59460DF10B009847019A0028E4D0AE
:020000021000EC
:10000000EAE73444204404B2E6E70C46EBE7044652
:10001000E9E71446E7E700BFB9D1000041FF00005F
:10002000540000202DE9F04F8FB099469DF86030C4
:10003000029104920393074698B1002900F0D28000
:10004000039B13F012030FD0002000E001303B5C53
:100050000A2B00F0C9800D2B00F0C680002BF5D1D3
:1000600080B20FB0BDE8F08F039A8DF82B3012F0FC
:100070000202059247F6184218BF91460B930B9B5C
:10008000009307EB030BFB5C002B00F08E80B9F1B3
:10009000000F40F38A80059A47F61843002A08BFEC
:1000A0004B460793514B00255A68CDE90C550CA9D6
:1000B000584690470C9B0D93039B019503F0010359
:1000C00080464FF0FF3A2E462A462C4608931BF8EE
:1000D000043043B9BAF1FF3F52D0009B002B6ED1E0
:1000E0001FFA8AF455E0414B0DA95B6858469847C2
:1000F000019B01330693089B024673B109903C4B68
:1001000041460DF12B009847099A30B1DDE90C43C7
:100110000C93069B01939046D9E7364B02980992BF
:1001200041469847064400B20028C8BF049B099A7C
:10013000B6B2C4BFF618B6B2BAF1FF3F36B205D1B7
:10014000049B0799F31A8B42C8BFA246B8F10A0F65
:1001500010D0B8F10D0F0DD027480023D9B2415C63
:1001600021B9BAF1FF3F08BF3546CFE7884503F113
:100170000103F3D1002CADD1BAF1FF3FADD135462B
:10018000019B23B1B8F10D0F02D10A2A00D10C9CBA
:10019000A4B2A9EB05090B9B0FFA89F994B95BB9D5
:1001A000124B0BA95B68384698470B9B23B90F4B42
:1001B0000BA95B6838469847BDF82C0051E700252D
:1001C0002C46E6E71C443B780B940A2BEDD00D2B14
:1001D000EBD03B5D0A2B02D00D2B7FF450AF0134E6
:1001E0000B94E2E702983CE7013039E75400002025
:1001F00041FF0000B9D100002A4202002DE9F04F72
:1002000089B0002598469DF85030BDF948B0BDF939
:100210004CA004930446164605804580039129B3FB
:1002200022B3049B13F0020F47F6184318BF9A46F7
:10023000B2F908300693138905935B440793039B37
:1002400003EB05095B5DA3B955B119F8013C0A2B15
:1002500001D00D2B04D1059B62885B44134463805D
:10026000B4F90230002B31D1069B638009B0BDE8A0
:10027000F08F049B0093424653463146154F484643
:10028000B847B4F90230079A1344B3F5004F01465A
:1002900005440BD3104B114C12931149114B712291
:1002A0000220A44609B0BDE8F04F60476380049B7C
:1002B000009348464346DFF830903246C847B4F9C9
:1002C00000309842B8BF18462080B8E7A3EB0B0374
:1002D000CBE700BF250001006142020031E90000C8
:1002E00032420200A14202007DFF00002DE9F047EA
:1002F000089D80460F46144699460CB9264612E0E2
:100300004FEA540A09FB0A7631464046A8470028BE
:1003100008DDE44304F00104AAEB040A06EB090734
:100320005446EAE7FCD13046BDE8F087014B18603F
:10033000704700BFD0C70020014B1B68D8687047CA
:10034000D0C70020014B1B681B681847D0C700208E
:10035000C0F3031310B500F0F001C4B2C0F30712EC
:10036000194300F00F0343EA041322F00F02890837
:1003700042EA1020C3F3C40343EA4113C0F3C400AC
:1003800043EAC02010BD000001392DE9F0470446C2
:10039000272934D8DFE811F028003900BB0082009B
:1003A00044004F004703B7000F01560239006F03A6
:1003B00020029503B700B7007100B7005101B700E4
:1003C000F701150285032A013B01EF016601D30104
:1003D000EB001B033703D700980084028E01B9019C
:1003E000F002C701BE02E502994B00219847994BE4
:1003F000002120469847984B1968984B984720460B
:10040000974BBDE8F047FF211847914B00219847D3
:10041000904B0021204698478F4B19680431ECE738
:100420008B4B002198478B4B0021204698478A4BE5
:1004300019681031E1E7884EDFF81492DFF8148272
:10044000864D0021C84700212046C047316804314D
:100450000746A847316818313846A8470121204689
:10046000C84701212046C047316804310746A847E4
:10047000316838460831A847C1E70021DFF8D0913C
:10048000DFF8D081744E754DC84700212046C04723
:1004900031680746A84731686831DDE7DFF8B08189
:1004A0006D4E6C4F6D4D0021C04700212046B8476E
:1004B00031682431A84701212046C0470121204648
:1004C000B84731682831D6E7DFF88481624E614F42
:1004D000624D0021C04700212046B84731682431D1
:1004E000A84701212046C04701212046B84731686E
:1004F0002831A84702212046C04702212046B8479C
:1005000031689C31B7E7524B0021984777E7DFF815
:100510004091514EDFF83C81504D0021C8470021E9
:100520002046C047316804310746A847316838463D
:100530002031A84701212046C84701212046C04755
:1005400031681C3197E7DFF80881434E414F434D36
:100550000021C04700212046B84731682031A84714
:1005600020460121C04701212046B847E8E73A4E1E
:10057000DFF8DC80374F394D0021C047002120468D
:10058000B847316824318146A847316848469431DC
:10059000A84701212046C04701212046B8473168BD
:1005A0002831A84702212046C04702212046B847EB
:1005B000316890315FE7284FDFF89480254E274D52
:1005C0000021C04700212046B04739684C31A84778
:1005D00040212046C04740212046B04739681031AD
:1005E0000646A84739683046503144E7184B1A4F41
:1005F0001A4E00219847174B00212046984739682A
:1006000004310546B04739687C3128467BE0DFF885
:100610004080114E0F4F114D4021C04740212046D0
:10062000B84731681831A84741212046C0474121C9
:100630002046B847316810311DE7054B0021984727
:10064000044B002120469847034B19686C31D4E6CF
:10065000F92400003D240000D4C7002015560000F6
:10066000392D0000DFF8A882A64EA74FA74D002124
:10067000C04700212046B84731680431A8474021CF
:100680002046C04740212046B84731681431A8476A
:1006900001212046C04701212046B84731688031FA
:1006A000A84702212046C04702212046B8473168AA
:1006B0008431E0E6964D934FDFF84C82934E002153
:1006C000A84700212046C0473968B047402120464E
:1006D000A84741212046A84741212046C047396804
:1006E000A831B04743212046A84743212046C047B0
:1006F0003968AC31B04742212046A8474221204604
:10070000C0473968A431B04779E6814D0021A84738
:1007100040212046A8477C4B402120469847794BF2
:100720001968B03169E60021DFF8E481754E764F33
:10073000764DC04700212046B8473168A7E7714E83
:10074000DFF8CC91DFF8C081704D0021C84700214F
:100750002046C047316804310746A847316838460B
:100760008831A84703212046C84703212046C047B7
:1007700031688C317FE6664B00219847624B00213F
:10078000204698473BE6624F5E4EDFF87C915F4D16
:100790000021B84700212046C8473168043180460F
:1007A000A847316840467431A84740212046B847E1
:1007B00001212046B84701212046C84731688031D1
:1007C00059E6534B002198474F4B0021204698474C
:1007D0004C4B1968783110E64A4EDFF834814A4FA5
:1007E0004A4D0021C04700212046B84731680431F6
:1007F0008146A847316848460831A84731684846CD
:100800001831A84740212046C04740212046B8471C
:10081000316804318146A847316848465431A847B9
:1008200041212046C04741212046B84731688031E8
:10083000A84742212046C04742212046B847316898
:10084000583118E62F4EDFF8C890DFF8BC802F4DE6
:100850000021C84700212046C047316804310746BF
:10086000A847316838464031A847316838461831C2
:10087000A84701212046C84701212046C0473168CA
:1008800018310746A847316838464431A847022145
:100890002046C84702212046C04731684831EAE572
:1008A000DFF86C80174E184F184D0021C04700210B
:1008B0002046B84731680431A84701212046C04787
:1008C00001212046B8473168A031A84702212046BF
:1008D000C04702212046B8473168A031A84703210C
:1008E0002046C04703212046B8473168A031A847B9
:1008F00004212046C04704212046B8473168A03172
:10090000B9E500BFD4C700203D2400001556000003
:10091000F9240000DFF800827C4E7D4F7D4D0021E0
:10092000C04700212046B8473168A84742212046E9
:10093000C04742212046B84731688031A84741214D
:100940002046C04741212046B8473168B031A8470A
:1009500040212046C04740212046B8473168A83191
:1009600089E56D4B00219847694B00212046984747
:10097000664B1968A43140E5DFF89C81634E644FF3
:10098000644D0021C04700212046B847316804313A
:100990008146A847316848461831A84720460421B7
:1009A000C04704212046B8473168B831A8472046DF
:1009B0000321C04703212046B8473168B431A84716
:1009C00020460121C04701212046B847F6E64F4E98
:1009D000DFF84491DFF838814E4D0021C8470021EF
:1009E0002046C047316804310746A8473168384679
:1009F0001831A84703212046C84703212046C04795
:100A00003168983137E5444B404F424E00219847BA
:100A10003F4B002120469847396804310546B047CE
:100A200039680831F1E5DFF8F080384E384F394D3C
:100A30000021C04700212046B84731680431A8474B
:100A400003212046C04703212046B84731682C3196
:100A5000A84701212046C04701212046B8473168F8
:100A60003031A84702212046C04702212046B8471E
:100A700031683431FFE4DFF8A080244E244F254D47
:100A80000021C04700212046B84731683831A847C7
:100A900001212046C04701212046B84731683C313A
:100AA000E9E41D4B194F1B4E00219847184B0021BC
:100AB00020469847396804310546B0473968703197
:100AC000A3E5124EDFF85080114F124D0021C047B0
:100AD00000212046B847316804318146A847316873
:100AE00048465C31A84701212046C04701212046E5
:100AF000B84731686031A84702212046C04702212B
:100B00002046B84731686431B5E400BFD4C700203F
:100B10003D24000015560000F9240000034B1B790A
:100B20000BB1034B1847034BFCE700BFD4C70020B1
:100B3000915700002D5500002DE9F0413A4D3B4BF7
:100B400028683B4E3B4C9C30984728683A4BFF2224
:100B50002C219C3098472868384B29211A88384B1B
:100B60009C309847286847F6FF7201219C30B047B7
:100B700000202F68A0473B2807F19C0747DD002095
:100B8000A04700F114026FF0270092FBF0F212B2BE
:100B900038461021B04700202F68A0473B2807F1B6
:100BA0009C0737DD0020A04700F114026FF02700FA
:100BB00092FBF0F212B238461121B04700202F68A4
:100BC000A0473B2807F19C0727DD0020A04700F144
:100BD00014026FF0270092FBF0F212B21221384695
:100BE000B04700202D68A0473B2805F19C0517DD84
:100BF0000020A04700F114026FF0270092FBF0F2F2
:100C000012B2284633461321BDE8F04118474FF091
:100C1000FF32BDE74FF0FF32CDE74FF0FF32DDE7A7
:100C20004FF0FF32EDE700BFD4C700201D0B0100DD
:100C30007558000095D90000155A0000B642020010
:100C4000455900002DE9F0416B4D6C4B28686C4E06
:100C50006C4C70309847286847F6FF72012170305D
:100C6000B04700202F68A04700EB80008000EF28ED
:100C700007F1700740F3B2800020A04750231421F1
:100C800000FB0132A02392FBF3F212B2384612218C
:100C9000B04700202F68A04700EB80008000EF28BD
:100CA00007F1700740F39C800020A04750231421D7
:100CB00000FB0132A02392FBF3F212B2384613215B
:100CC000B04700202F68A04700EB80008000EF288D
:100CD00007F1700740F386800020A04750231421BD
:100CE00000FB0132A02392FBF3F212B2384610212E
:100CF000B04700202F68A047C0EB00104000EF284D
:100D000007F1700770DD0020A04750231E2100FB73
:100D10000132A02392FBF3F212B238461421B047FD
:100D200000202F68A04700EB800000EB8000EF2838
:100D300007F170075ADD0020A0475023192100FB5E
:100D40000132A02392FBF3F212B23846C021B04721
:100D500028682D4FAA8999217030B8472868AA8938
:100D6000C9217030B8472868284B00F1700840F658
:100D700088009847CA2102464046B84700202F689D
:100D8000A04700EB80004000EF2807F170072FDD3F
:100D90000020A04750230A2100FB0132A02392FB30
:100DA000F3F212B290213846B04700202D68A047D8
:100DB000C0EBC000EF2805F170051BDD0020A04747
:100DC0005023072100FB0132A02392FBF3F212B261
:100DD00028463346C321BDE8F0411847012255E7B4
:100DE00001226BE7012281E7012296E70122ACE7AD
:100DF0000122D7E70122EBE7D4C700201D0B010039
:100E00007558000095D900004559000051030100B4
:100E10002DE9F041324C334B2068334E334F344D83
:100E20006C3098472068FF222C216C30B047206836
:100E3000A28929216C30B8472068022230216C3009
:100E4000A84720687F223C216C30B0472068294B9E
:100E500000F16C064C21A0899847392102463046A2
:100E6000B8472068244E47F6FF7201216C30A8472E
:100E70002368002003F16C08B047C0EB0010EF2896
:100E80002ADD0020B0470F21502300FB0130A022B3
:100E900090FBF2F212B250214046A8472068A28986
:100EA00059216C30B84700202468B04700EB80001F
:100EB000EF2804F16C0411DD0020B0475023052118
:100EC00000FB0132A02392FBF3F212B220462B4624
:100ED0005321BDE8F04118470122DCE70122F5E784
:100EE000D4C700201D0B0100155A00004559000011
:100EF0007558000093E3000095D90000C0F38522E7
:100F0000C0F3C40343EA4213C0F3C44043EAC02021
:100F1000704700002DE9F047434CDFF8349120681A
:100F2000424E434FDFF82C812430C847206847F6F3
:100F3000FF7201212430B0472068FF2224302C2189
:100F4000B847236A256813F0020F14BF39483A489E
:100F5000C0472435024629212846384DA847236832
:100F600003F1240A236A9A0758D53548C047024638
:100F700079215046A8472068A28949212430A847F2
:100F80002068E28940F249412430A84720680022C5
:100F90004C212430B84720687F224FF4137124304D
:100FA000B8472068032240212430B04720689622A9
:100FB000B0212430B04720684C22B7212430B047FC
:100FC00020682830C8472068FF222C212830B847E5
:100FD000206847F6FF7201212830B0472068A289B7
:100FE00029212830A8472068164B00F1280640F632
:100FF0008800984742F2290102463046A847236AF2
:1010000020689B0700F128060BD50F48C047024611
:1010100030462B467921BDE8F04718470B4B1A881C
:10102000A6E70A4B1A88F3E7D4C7002075580000DA
:10103000155A0000D9D7D4004D4945004559000044
:101040004F403100510301004F404100B6420200C1
:101050001D0B0100FD0E01002DE9F0417D4D7E4F7D
:1010600028687E4C9030B84728687D4BFF222C21A1
:10107000903098472B6A28689A0756BF794BAA89FF
:101080001A8890302921A0472B6A2E689B0706F109
:10109000900640F1CC807448744B98470246304625
:1010A0007921A0472868724E724C47F6FF720121E1
:1010B0009030B0472B68002003F19008A047C0EBA8
:1010C000C000EF2840F3B6800020A047072150233E
:1010D00000FB0130A02290FBF2F212B24046122136
:1010E000B0472B68002003F19008A047C0EBC00078
:1010F000EF2840F3A1800020A0470721502300FBE8
:101100000130A02290FBF2F212B240461321B04708
:101110002B68002003F19008A047C0EBC000EF2827
:1011200040F38C800020A0470721502300FB0130B2
:10113000A02290FBF2F212B240461021B0472B6879
:10114000002003F19008A047C0EBC000EF2877DD36
:101150000020A0470721502300FB0130A02290FB74
:10116000F2F212B211214046B04728689430B847D5
:1011700000202F68A04700EB80004000EF2807F117
:1011800094075FDD0020A04750230A2100FB0132B5
:10119000A02392FBF3F212B238461721B047002089
:1011A0002F68A04700EB80004000EF2807F194076C
:1011B0004ADD0020A04750230A2100FB0132A02372
:1011C00092FBF3F212B238461821B04700202F6884
:1011D000A04700EB80004000EF2807F1940735DDC1
:1011E0000020A04750230A2100FB0132A02392FBDC
:1011F000F3F212B215213846B04700202D68A047FF
:1012000000EB80004000EF2805F1940520DD002070
:10121000A04750230A2100FB0132A02392FBF3F2E6
:1012200012B2284633461621BDE8F04118470D4B4F
:101230001A8834E7012251E7012266E701227BE7A1
:1012400001228FE70122A7E70122BCE70122D1E7B3
:101250000122E6E7D4C700201D0B0100455900001C
:10126000155A0000B64202004F403100FD0E010049
:101270007558000095D900002DE9F047B54CDFF80E
:10128000F0822068B44DB54FDFF8E8A25C30C0476B
:10129000206800F15C0640F68800A84799210246C4
:1012A0003046B847206800F15C0640F68800A84741
:1012B000C92102463046B8472068A289CA215C305D
:1012C000B84700202668D04700EB8000EF28A946E9
:1012D00006F15C06554640F389810020D047052180
:1012E000502300FB0130A02290FBF2F212B23046F4
:1012F00090219B4EB0472368002003F15C0AA84769
:101300003B2840F375810020A8472822143090FB29
:10131000F2F212B25046C321B0472368002003F115
:101320005C0AA8471D2840F365810020A8471422C5
:101330000A3090FBF2F212B25046C221B047236845
:10134000002003F15C0AA84700EB80008000EF2832
:1013500040F352810020A8471421502300FB0130A4
:10136000A02290FBF2F212B250461221B04723683D
:10137000002003F15C0AA84700EB80008000EF2802
:1013800040F33C810020A8471421502300FB01308A
:10139000A02290FBF2F212B250461321B04723680C
:1013A000002003F15C0AA84700EB80008000EF28D2
:1013B00040F326810020A8471421502300FB013070
:1013C000A02290FBF2F212B250461021B0472368DF
:1013D000002003F15C0AA84700EB80008000EF28A2
:1013E00040F310810020A8471421502300FB013056
:1013F000A02290FBF2F212B250461421B0472368AB
:10140000002003F15C0AA847C0EB0010EF2840F36E
:10141000FB800020A8470F21502300FB0130A022B1
:1014200090FBF2F212B25046C021B047206847F656
:10143000FF7201215C30B04720686030C0472068EF
:1014400000F1600A40F68800C847992102465046DC
:10145000B847206800F1600A40F68800C847C921F3
:1014600002465046B8472068A289CA216030B84772
:101470002368002003F16009A8471D2840F3C680B7
:101480000020A84714220A3090FBF2F212B248461C
:101490009021B0472368002003F16009A8471D2868
:1014A00040F3B6800020A84714220A3090FBF2F2E5
:1014B00012B24846C321B0472368002003F16009F7
:1014C000A84700EB800000EB8000EF2840F3A280EB
:1014D0000020A8471921502300FB0130A02290FBD7
:1014E000F2F212B2C0214846B04720686430C047CB
:1014F000236803F16408236A9A0740F18D80194834
:10150000194B9847024640469921B8472368002066
:1015100003F16408A8471D2840F381800020A847F4
:1015200000F10A02142092FBF0F212B24046902120
:10153000B04720680D4BFF222C2164309847236868
:1015400003F16408236A9B076BD50648064B98474E
:10155000024611E0D4C700205103010045590000A4
:10156000755800005B4B4600FD0E0100155A000047
:101570001D0B010095D9000029214046B84720687D
:1015800047F6FF7201216430B04700202768A84762
:10159000C0EB00104000EF2807F1640744DD002095
:1015A000A84750231E2100FB0132A02392FBF3F237
:1015B00012B203213846B04700202468A84700EB48
:1015C00080004000EF2804F164042FDD0020A847CC
:1015D00050230A2100FB0132A02392FBF3F212B246
:1015E000204633461421BDE8F047184701227EE625
:1015F00001228FE601229FE60122B5E60122CBE619
:101600000122E1E60122F7E601220CE701223EE792
:1016100001224EE7012265E7054B1A8873E7012294
:1016200084E7034B1A88A7E70122C2E70122D7E724
:10163000B64202002DE9F047674D684F2868DFF891
:10164000B8914030B8472B6A2C6813F0020F04F1B0
:10165000400400F0B080624B40F6AA209847024652
:1016600048F289012046DFF894815E4CC047286823
:101670004430B84700202E68A047EF2806F1440602
:1016800040F39C800020A047A022503090FBF2F253
:1016900012B230469021544EB0472B68002003F11F
:1016A000440AA04700EB80004000EF2840F3888008
:1016B0000020A0470A21502300FB0130A02290FB0C
:1016C000F2F212B250469221B0472B68002003F18B
:1016D000440AA04700EB80004000EF2872DD0020A4
:1016E000A0470A21502300FB0130A02290FBF2F218
:1016F00012B250469321B0472B6803F1440A2B6A7B
:101700009B074CBF39483A48C84799210246504682
:10171000C04728684830B84700202F68A04700EB32
:101720004000EF2807F148074EDD0020A047502376
:10173000032100FB0132A02392FBF3F212B23846E0
:101740009021B04700202F68A0473B2807F14807A9
:101750003CDD0020A04700F11402282092FBF0F2AB
:1017600012B238460321B04700202F68A0477728DF
:1017700007F148072CDD0020A04700F12802502087
:1017800092FBF0F212B214213846B04700202D68C7
:10179000A047EF2805F148051CDD0020A04700F117
:1017A0005002A02092FBF0F212B2284633460121EB
:1017B000BDE8F04718470F48C84750E7012268E7DF
:1017C00001227FE7012294E70122B8E70122C8E75E
:1017D0000122D8E70122E8E7D4C700201D0B010051
:1017E0005103010095D9000075580000E3DDD600D3
:1017F000978A8000BDADA100FD0E01004559000093
:101800002DE9F04F2DED028BA04CA14F2068A14D8A
:10181000DFF8AC9283B0B8472068FF222C21A8479C
:10182000236A266813F0020F14BF9B489B48AB46FF
:101830009B4DA847BA4602469A4F30462921B847E1
:10184000236A266898074CBF97489848A84748F2EB
:10185000890102463046B847236A266899074CBF7B
:1018600091489248A847792102463046B8476269B4
:1018700020688F4E48F28E01C847626920687E2139
:10188000C84720680430D0472368002003F10408CB
:10189000B0471D2840F366850020B04714220A3067
:1018A00090FBF2F212B240460121DFF81882C047E5
:1018B0002068FF2204302C21D847236803F1040B51
:1018C000236A9A0754BF7B486FF07F40A8472921BD
:1018D00002465846B847236803F1040B236A9B0766
:1018E0004CBF75487548A847392102465846B84745
:1018F0002068A28940F239210430B8472068E28983
:1019000040F239410430B8472368002003F1040B4A
:10191000B047772840F329850020B047502228306F
:1019200090FBF2F212B258463021C04720680122E3
:1019300033210430C04720686269043048F28E01C8
:10194000C847236803F1040B236A98074CBF564825
:101950006FF07F40A84748F2890102465846B847D1
:101960002068626904307E21C847236803F10409B6
:10197000236A99074CBF4C486FF07F40A8477921F4
:1019800002464846B847236803F10409236A9A07C8
:101990004CBF45486FF07F40A84748F2A901024676
:1019A0004846B847236803F10409236A9B074CBFE4
:1019B0003D486FF07F40A847992102464846B84706
:1019C0002068DFF80491012290210430C047236889
:1019D0000020043308EE103AC84701284FF00000F9
:1019E00000F2D384B047C0EB0010EF2800F3C084AE
:1019F0004FF0010B0020B047772840F3D18400203E
:101A0000B0475023283090FBF3F080B20BEB00027C
:101A100012B218EE100A1221C047236800200433C6
:101A200008EE103AC84701284FF0000000F2C884C1
:101A3000B047C0EB0010EF2800F3B5844FF0010B66
:101A40000020B047772840F3C6840020B0475023D9
:101A5000283090FBF3F080B20BEB000212B218EECC
:101A6000100A1321C04723680020043308EE103AFF
:101A7000C84701284FF0000000F2BD84B047C0EB1A
:101A80000010EF2800F3AA8420E000BFD4C7002094
:101A90001D0B0100155A0000F3EFEA005A4B4400F9
:101AA000FD0E010045590000423E3B00ECE9E70015
:101AB00095D9000073625800E3DDD600978A800054
:101AC000E95A000075580000ADD900004FF0010B35
:101AD0000020B047772840F399840020B047502376
:101AE000283090FBF3F080B20BEB000212B218EE3C
:101AF000100A1021C04723680020043308EE103A72
:101B0000C84701284FF0000000F29084B047C0EBB6
:101B10000010EF2800F37D844FF0010B0020B04748
:101B2000772840F38E840020B0475023283090FB64
:101B3000F3F080B20BEB000212B218EE100A112182
:101B4000C0472368002003F1040BC84701284FF069
:101B5000000000F28584B047C0EB0010EF2800F3CE
:101B60007384012214215846C0472068DFF814937B
:101B70009622B0210430C04720683922B7210430B2
:101B8000C04720680C30D0472068AC4B011D0C309A
:101B90009847236A266898074CBFA948A948A847D0
:101BA0000C36024629213046B847236A2668990731
:101BB0004CBFA548A548A8470C36024639213046F7
:101BC000B847236A26689A074CBFA148A148A8478E
:101BD0000C36024648F289013046B847236A266827
:101BE0009B074CBF9A489B48A8470C360246792170
:101BF0003046B847236A266898074CBF94489548F2
:101C0000A8470C36024648F2A9013046B847236A75
